:10000000004000202571000065710000677100004C
:1000100000000000000000000000000000000000E0
:1000200000000000000000000000000069710000F6
:1000300000000000000000006B7100006D71000006
:100040006F710000AD520000A17500006F710000DB
:100050006F710000000000006F7100006F71000000
:100060006F71000071780000B53100006F71000001
:100070006F7100006F7100006F7100006F71000000
:100080006F710000097A00006F7100006F7100004D
:100090006F7100006F7100006F7100006F710000E0
:1000A0006F7100006F710000000000000000000090
:1000B0000000000000000000000000000000000040
:1000C00010B5064C2378002B07D1054B002B02D02E
:1000D000044800E000BF0123237010BD640200202B
:1000E0000000000038E40000044B10B5002B03D0E2
:1000F0000349044800E000BF10BDC04600000000F6
:100100006802002038E40000164B002B00D1144B8D
:100110009D46402292029A1A924600218B460F4633
:100120001348144A121A0BF017FA0F4B002B00D089
:1001300098470E4B002B00D0984700200021040068
:100140000D000D48002802D00C4800E000BF0BF065
:10015000C3F92000290007F041FA0BF097F9C046D7
:100160000000080000400020000000000000000027
:1001700064020020BC2F00200000000000000000EE
:1001800002000120104011D1042A0ED91368180969
:1001900080B2002809D001388000031D11180979A8
:1001A000002902D001309842F8D170470020FCE7C6
:1001B0000378002B03D05AB2002A01DB01307047CC
:1001C0003F229343C03B59424B41C01803789343AD
:1001D000802BF4D10130F9E710B500240378002B0F
:1001E00001D1200010BDFFF7E3FF0134F6E770B541
:1001F000002204000D00411C092003F005FB00282B
:1002000006D001236200134343600023A34200DBB6
:1002100070BD9A00A958821891600133F6E770B555
:10022000012803DC1C2001F047F870BD01230D6894
:1002300011201D42F7D04868184206D1042804D97D
:100240000F2302681340042B01D00E20EBE703F0CC
:1002500039F96D100400002D03DDFFF7BDFFA84242
:1002600006DA1220DFE72000FFF7A2FF0400013DBD
:10027000012DF8D120787F2809DDDF280BDCF82359
:100280003F22DB00800118406378134018430123AC
:1002900040001843C9E7EF280BDCFC226378120109
:1002A0009B0113403F220007000C0343A07810403D
:1002B000ECE7F72812DCFC22637892021B03134060
:1002C000E0228004520310403F221843E378134099
:1002D000FC220343A07812018001E8E7012040429C
:1002E000D5E7F8B54D680F00EB0706D4042D04D907
:1002F0000F232E683340092B03D00B2000F0DCFFC6
:10030000F8BD6B683609B6B25C10731EA3420FD8F5
:100310000321200008F0DCFF6421642803DC0100D5
:10032000032800DA03212800891903F09FFA050049
:100330002B6800201B099BB2013B9C42E0D23A682B
:10034000A31C9B005A510123013464001C436C60C0
:10035000D6E7F0B585B0012803DC1C2000F0ACFF27
:100360002CE001274B683A000093022806D08B68E6
:100370003B4203D05F10002F00DC17000124009BDC
:10038000234200D0B2E0042B00D8AFE01B680D6818
:100390000F2619003140042925D1254205D1042D0D
:1003A00003D92B681E40042E01D00E20D6E70098FA
:1003B000FFF7E6FEB84203DA0120404205B0F0BD87
:1003C000009803F07FF80600280003F07BF8010096
:1003D000781E30180BF076FC0028EDD0801B013021
:1003E00040002043EAE709293DD1009B5B685B1090
:1003F00001939F42E0DC25422CD1042D2AD92B68A1
:100400003340042B26D1280003F05CF803960290B9
:100410007E1C009AB300D058854201D17800E0E7F5
:1004200020420ED104280CD90368039A1340042BF0
:1004300007D103F047F8010002980BF00DFC0028EB
:10044000ECD0019B37009E42E2DDB5E71F00019B27
:100450009F42B1DC7B1C00999A008A58AA42F5D1D0
:1004600078000124BDE7032940D11A0992B25B0F3D
:1004700092000B40D31A01939F429DDC254229D163
:10048000042D27D92A681640032E19D1100980B2ED
:10049000520F800032402C1D801A019B26181B1A17
:1004A0000193009B781E0433019A904200DD83E79C
:1004B00022001918B2420FD316D101304000D0E704
:1004C000042E07D1280002F0FDFF04002800FFF7EA
:1004D00057FEE2E70F2041E70D78AC461578AC45B2
:1004E00002D101310132E5E70130DDE7212035E7B6
:1004F00010B502F0CBFF43000120184310BD0000EF
:10050000C30711D404280FD90F2302681340032B0B
:100510000AD119400133591AC0234907DB05194094
:10052000024B1A40114301607047C046FFFFFF9F16
:10053000F7B507000E001C20012F06DD4C680123D3
:1005400022001A40009203D10D2000F0B5FE53E0C6
:10055000022F02D08A681A42F6D0012335681D4264
:1005600000D0A9E0042D00D8A6E01C41002C00DC3E
:100570001C000F2029680840092828D16B685B10EF
:100580000093022F05D0B368009A5B109A4200DDF9
:100590000093009B01221D1B0135EB43DB171D401F
:1005A000691C092003F030F9071E09D001236D00F2
:1005B0001D4303003268083345600099A14201DA07
:1005C0003800FEBD0134A100515802C3F5E70428EC
:1005D00045D1280002F076FFFFF7FEFD0190022FC3
:1005E00004D0B3685B10984200DD0193019BA342E5
:1005F00004DA002003F07AF90700E1E7280002F0AE
:1006000061FF0700009BA34221DB2800009702F056
:1006100059FF05003800FFF7CBFD019B01340700AF
:10062000A342F7DA009BC41A200003F05FF9071E0B
:10063000C6D002F047FF0190306802F043FF22006D
:10064000009B591B411801980AF06AFFB8E738006F
:10065000FFF7AEFD009B070001330093D2E70328AC
:100660002AD10B099BB2490F9B000140591A022F56
:1006700004D0B2685210914200DD1100A14205DAA7
:1006800000220320110003F0BFF8B5E703200E1B82
:10069000331DD9170140C9188910002203F0B4F89E
:1006A000071E00D18CE7013631000334FFF728FF25
:1006B000381D29193200C7E7212046E7F8B5002880
:1006C00005DC1C2000F0F8FD05002800F8BD01261F
:1006D0000C6826400FD06410E343DB171C40E11C7C
:1006E00089100022032003F08FF8051EEDD02100B1
:1006F000FFF706FFE9E7042C01D80025E5E70F2303
:1007000022681340042B1BD12000FFF739FDC31CC6
:1007100007000320D9170140C9188910320003F0DF
:1007200073F8051ED1D03900FFF7EAFE200002F071
:10073000C9FE2B1D01003A0018000AF0F1FEC4E7C3
:10074000092BDAD10320636832005F10FB1CD91734
:100750000140C918891003F057F8051ECDD03900A3
:10076000FFF7CEFEFF20BE42AFDA0122B300E3184E
:100770009B68134208D01341FF2B00DD0300D943CF
:10078000C917AA190B4013710136ECE710B57F2980
:1007900002DC0170013010BD1A4B99420CDC402381
:1007A0008A115B42134303703F230B40802149426F
:1007B000194341700230EEE7134B994210DC2023BD
:1007C0000A135B4213433F24802203708B11524271
:1007D0002340214013430A43437082700330DAE719
:1007E0000A4B9942D7DCF0230370603B4370113B06
:1007F0008A11FF3B1A4382703F2211401943C17096
:100800000430C8E7FF070000FFFF0000FF0F0100F2
:10081000F0B50D0085B0002803DC1C2000F04CFD75
:100820000DE009680122080010400AD002AC114115
:100830002000FFF7ABFF011B200003F063F804006A
:100840001AE004293FD90F230C682340092B3AD121
:100850004B685B10019303239C46019B9A420EDD7B
:1008600003F044F8041E07D02E68012502F02AFE8A
:100870002F00019B9D421DDD200005B0F0BD01321F
:100880009300CC580123234001D10D20C6E764100A
:100890007F2C0DDD0D4E0223B44209DD0C4E634664
:1008A000B44205DD00270B4EE30FA6427B419B00BF
:1008B000C018D2E70135AB00F1583942E5D04910F4
:1008C000FFF764FFD5E72120A8E7C046FF07000037
:1008D000FFFF0000FF0F010010B5040001200840D9
:1008E00010D104290DD90F230A681340042B08D115
:1008F000080002F0E7FD010020000BF0ADF94342D3
:10090000584110BD0020FCE7F7B50F00012803DCBB
:100910001C2000F0D1FCFEBD01264D682E4006D102
:10092000042D04D90F222B681A40092A01D00B206C
:10093000EFE76A681B099BB25410A34200D85C1E03
:1009400039681E48FFF7C8FF01230190002813D122
:1009500039681B48FFF7C0FF002811D0002C0DD0CC
:100960000123621C013C9C409200535123436B6065
:1009700004E00136B200AB50B442FADA0020CAE714
:100980003B680D20DA07C4D55B10002B11DD9C42BB
:100990000FDB9B00A200291DEB1889180433994234
:1009A00009D10123013C9C40AA181C4353606C6090
:1009B000E4E71220ADE758681860EFE7EBCB0000E2
:1009C000EFCB0000002310B50C000B70C30705D55A
:1009D0000D49421020000BF003F908E00B490028F4
:1009E00002D0042804D10A4920000BF019F910BDE7
:1009F0000428FCD90F2302681340042BF7D102F01E
:100A000061FD04490200E5E7E8D50000F4CB0000F1
:100A1000FACB0000FFCB0000F0B593B006000291C6
:100A20001C20012E1DDD029B01251B681C002C4093
:100A300000D0ADE0042B00D8E6E01A680F231A407E
:100A4000092A4AD10394039A029992008A581700FE
:100A50002F4005D1042A03D910681840092806D070
:100A6000222000F029FC0190019813B0F0BD5268DB
:100A70005210A418039A013203929642E3D1611CEA
:100A8000012202F0C1FE0190002802D1002301934F
:100A9000EAE7019B6400190025435D600831029A72
:100AA000BB00D05802684368120992B25B109A42A8
:100AB00000D8531E0022934209DCDA43D2171340B8
:100AC0009B00C918039B01379F42E8DBCCE79400E9
:100AD0000519AD6801320D51EDE72700032A59D100
:100AE0000193029ABB00D3582B42B9D1042BB7D93A
:100AF000186801990140032939D1020992B2430FC4
:100B000092000B40D31A1C190137BE42E9D10320D1
:100B1000E31CD9170140C9188910002202F074FEA5
:100B200001900028B2D000252100FFF7E9FC019BCD
:100B30001E1D029AAB00D45801231C421FD1042C65
:100B40001DD90F2123681940032918D1180980B233
:100B50005B0F80000B40C01A0023834213DBC343AA
:100B6000DB17184001353618BD42E2DB7CE704296B
:100B700000D075E71800FFF703FB2418C4E7200036
:100B8000FFF7FEFAE8E7E2181279F2540133E4E7DE
:100B900000273C000F25029ABB00D35801221342C4
:100BA00034D1042B32D9186801002940042935D1E9
:100BB0001800FFF7E5FA24180137BE42EBD12000F8
:100BC00002F094FE0190002800D15FE7029FB6007A
:100BD000BB19041D029301233D681D4229D1042D38
:100BE00027D90F262B681E40042E37D12800FFF787
:100BF000C7FA0600280002F065FC01002000320060
:100C00000AF08EFCA41922E02700C3E7180005A90A
:100C1000FFF7D8FE05A80BF029F8CCE7032900D090
:100C20001EE7020992B2430F92000B40D31A1C191F
:100C3000C2E705A92800FFF7C5FE05A80BF016F8C6
:100C400005A90500020020000AF06AFC6419029B55
:100C50000437BB42BFD10023237005E7032EF6D132
:100C60001A0992B25B0F92001E40961B291DC5E720
:100C7000F0B50D0095B0002806DC1C2000F01CFB30
:100C80000400200015B0F0BD0C68012123000B40CA
:100C9000009306D1042C04D922680F331A40092A84
:100CA00001D00B20EAE7626852100392002A03DCAD
:100CB000009802F01BFEE3E73F4A019201280BD0A7
:100CC0006868084208D1042806D902681340042B3A
:100CD00002D102F0F7FB019001980AF0C7FF06006D
:100CE0000F27039B0834013B04935E43039B029050
:100CF0009B001B19059301232068184251D1042839
:100D00004FD903683B40042B52D1FFF739FA059BBA
:100D100004343618A342EED1300002F0E7FD041E81
:100D2000AFD02B680593029B002B03D0686802F0BC
:100D3000C9FB0190200002F0C5FB0500009B059A4D
:100D40009B00D3189F68380002F0BCFB012306000B
:100D50001F4201D1042F04D807A93800FFF732FE43
:100D600007AE30000AF082FF0700020031002800C1
:100D70000AF0D6FB029BED19002B0AD0049B009AC7
:100D8000934206DD2800029A01990AF0C9FB029BF2
:100D9000ED18009B01330093009A039B9342CDD141
:100DA0006FE707A9FFF70EFE07A80AF05FFFAEE79F
:100DB00002F088FBF9E7C0468CD0000010B5002493
:100DC000A04207DD0B6801341C4003D05C10E343F4
:100DD000DB171C40611C0122092002F015FD0028D0
:100DE00003D0012364001C43446010BD0A6870B541
:100DF00010000125284034D1042A32D90F24136869
:100E000049681C40092C17D154681B099BB22C411E
:100E1000A34200D85C1E844205DC022001339842C4
:100E200006DB00200FE085005519A9600130F2E7CC
:100E3000840011510130F2E7032C12D1294203D171
:100E4000132000F039FA70BD4910FF29F8D81B09AA
:100E50009BB204329B00D3189342E2D91170013245
:100E6000FAE70B2000F028FADBE700000123F7B5D2
:100E700000254E680F0033400093AB420ED11D0099
:100E8000042E0BD90F2233681A40092A10D1726838
:100E90001B099BB25510AB4200D85D1E3968CB07C9
:100EA00017D54C10002C01DDA5421DDA122032E0CE
:100EB000042A04D13000FFF763F90500EEE7009D36
:100EC000032AEBD11D09ADB25B0FAD001340ED1A43
:100ED000E4E72E48FFF700FD002814D00AF01CFEBE
:100EE000290008F0DBFA4C1C009B002B4CD1042E8F
:100EF0004AD932680F331340092B10D10134A400B2
:100F0000A4592000FEBD39682148FFF7E5FC2C00FC
:100F10000028E9D1113000F0CFF90400F1E7042BEB
:100F20002AD1300002F0CEFA0500FFF755F9A042B1
:100F3000BCDB012C1ADC300002F0C4FA009028005F
:100F4000FFF736F9461B300002F0D0FC041ED8D063
:100F500002F0B8FA0190786802F0B4FA009B32000F
:100F6000E91A411801980AF0DBFACAE72800FFF7EE
:100F70001FF9013C0500DCE7032B05D13419E478A7
:100F8000023B64001C43BCE70B20C4E7E4CB000039
:100F9000EFCB0000F7B54D680F002A0001210A4091
:100FA0002FD1042D2DD90F242B68BE681C40092C8D
:100FB00014D169681B099BB24C100192A34200D85E
:100FC0005C1E39682A48FFF787FC00282DD00F23C4
:100FD0002A681340092B1DD1012317E0032C10D1DF
:100FE0000E4203D1132000F067F9FEBD721001928A
:100FF000FF2AF7D81A0992B25B0F92001C40141B0B
:10100000DFE70B20EFE701339A00AE509C42FADA9B
:101010000020EAE7032BFBD12B0001335A1BA2422D
:10102000F6DC6A461279DA70F7E73968CB0706D53D
:101030004910002901DD8C4209DA1220D3E70D485E
:10104000FFF74AFC2100002801D11130CBE70F2324
:101050002A681340092B03D1013189004E51D7E78B
:10106000032BD5D16B461B796D18EB70D0E7C046CA
:10107000EBCB0000EFCB000010B501240868204244
:101080001AD1042818D90F2102681140092901D169
:10109000406810BD032908D113099BB2500F9B0073
:1010A0000840181A40002043F3E7042904D102F055
:1010B00009FAFFF791F8F5E70B2000F0FDF8E8E7F3
:1010C00010B5034A0B21034804F0E8F910BDC046EF
:1010D0008CCB000084CB00000020704704207047B8
:1010E0000120704710B5002002F000FC10BD002068
:1010F0007047002070470020704700207047002094
:1011000070470020704700207047002070470000A3
:1011100010B5034A0C21034804F0C0F910BDC046C5
:1011200074CC0000D4CC000010B50124044002D0DF
:101130004410200010BD042810D90F23026813406A
:10114000042B07D102F0BEF921000A220AF056FE54
:101150000400EEE7032B01D10430F5E70D22014B2B
:101160001A70E6E7A4020020012210B5024018D14F
:10117000042802D903681A0992B201230B4012D144
:10118000042902D90B681B099BB20024934206D1A3
:1011900004309B000431C318984206D30124200078
:1011A00010BD0022E9E70023EFE704780A78002C5D
:1011B00001D1002AF2D0013001319442ECD0002458
:1011C000EDE70000F7B50700009101933049314B7E
:1011D000002A02D002220A70013A00261A601B6817
:1011E000CE54BE4200DBF7BD009AB300D058294B65
:1011F000274D1C68C8239B0065191C1B012318423E
:1012000006D0254A4310210028000AF0B7FC09E067
:10121000224A002802D004281BD1214A210028009C
:101220000AF0ACFC1A4C20000AF020FD194A019B80
:101230001060002B0BD07B1EB34208DD194B984287
:1012400005D8431C1360202222540022E2540136A8
:10125000C7E7042819D90F2301680B40042B04D1D8
:1012600002F030F9104A0300CDE7092B03D143689F
:101270000E4A5B10C7E7032B08D10A0992B2490F47
:1012800092000B40D31A0A4ABDE70123094ABAE784
:10129000A5020020C8050020E8D50000F4CB00001E
:1012A000FACB00001F03000013DC000044CF000055
:1012B00053CF00005ECF0000014B18700020704734
:1012C000A402002070B501F063FE094C0100251D49
:1012D0001F2228000AF0E2FC28000AF0C7FC0423C1
:1012E00004308008000118432060200070BDC04613
:1012F00080020020C368F0B59D00836889B05D1945
:101300000300183306930369069A9F00069B029018
:10131000DF19436901939B00D3180393CD4B1B78CE
:10132000002B26D17F222B68CB491C1213409B0037
:101330005B58043501929F46029B587804F0CAFC22
:101340000023029A137027E0C24B1B78002B10D1A8
:101350002B68019A1C121340BF4A9B009B5804350E
:10136000E9E7069B3A1DD11ABA4BD82928DD1A2283
:101370001A70029BB74C9B6821780193EA1A029B72
:1013800092109B7812021A43029B587804F0AAFC30
:101390000023029A23701370029B069A9B680193A4
:1013A000ED1A029BAD10DD60069BFE1A029BB61083
:1013B0001E61039B9B1A029A9B10536109B0F0BDFA
:1013C0001B783C60002B01D01700D2E72B680199F5
:1013D0001C120B40A0499B005B5817000435AAE77C
:1013E000069B3A1DD11A9B4BD82902DD1A221A708E
:1013F000BFE728681B78291D3860002B02D0170032
:101400000D00B6E76B6801991C120B4092499B00D6
:101410005B58170008358EE7069B3A1DD11A8D4B95
:10142000D82902DD1A221A70A3E7A4001B782C1910
:101430003C60002B01D017009BE72B6801991C1220
:101440000B4085499B005B581700043573E7069BEA
:101450003A1DD11A7F4BD82902DD1A221A7088E76B
:101460007E49A40061581B783960002B01D0170019
:101470007FE72B6801991C120B4077499B005B5852
:101480001700043557E7043F744B3A68A400E25054
:10149000704B1B78002B00D06BE72B68019A1C1255
:1014A00013406D4A9B009B58043544E76B4BA400E6
:1014B000E058FFF739FE043F06003868FFF734FEB6
:1014C00036180120654B76000643E650614B1B78C9
:1014D000002B00D04DE72B68019A1C1213405E4A86
:1014E0009B009B58043526E7069B3A1DD11A594BA1
:1014F000D82902DD1A221A703BE70698039C0121C5
:10150000A04202D221000C3909681B783960002BF7
:1015100001D017002DE72B6801991C120B404E4992
:101520009B005B581700043505E7069B3A1DD11A4E
:10153000484BD82902DD1A221A701AE70699039837
:1015400081420FD203000C3B1B6845495B106418B5
:10155000E41AA40023583B603E4B1B78002B05D0B7
:10156000170006E7182119700023F4E72B6801998A
:101570001C120B4038499B005B5817000435DAE613
:10158000069B039A934219D213000C3B1B68344A02
:10159000043FA4185B10E31A039A39689B00995022
:1015A0002C4B1B78002B00D0E3E62B68019A1C1211
:1015B0001340294A9B009B580435BCE61822254B52
:1015C0001A70EDE7069B039A93422DD2244B3E1FDF
:1015D000E31814000C3C04932368049A5B10D31A9C
:1015E000039A9B009858FFF79FFD07903068FFF71C
:1015F0009BFD2468049B64101C1B079BA4001F1800
:1016000001207F00039B0743E7503700114B1B78F5
:10161000002B00D0ADE62B68019A1C1213400E4A35
:101620009B009B58043586E618220A4B1A70EDE79A
:10163000069B3A1DD11A074BD82902DD1A221A70CF
:1016400097E60399A40061581B783960002B09D0F4
:1016500017008EE6A402002044CD0000882D002053
:10166000FDFFFF3F2B6801991C120B40D9499B00DD
:101670005B58170004355EE6043F039B3A68A400FC
:10168000E250D54B1B78002B00D072E62B68019AF4
:101690001C121340CF4A9B009B5804354BE6039B1A
:1016A000A4001C192368043F38685E10FFF73CFD56
:1016B00036180120C84B76001B7806432660002BA5
:1016C00000D056E62B68019A1C121340C14A9B00B9
:1016D0009B5804352FE6069BA4003F1BBE4CBB4223
:1016E0000CD82378002B00D043E62B68019A1C12FB
:1016F0001340B84A9B009B5804351CE6B74801F0DC
:10170000D1FE2378002B00D033E62B68019A1C12FF
:101710001340B04A9B009B5804350CE6A300ED181B
:10172000002C00DA38E6AC4B1B78002B00D020E60A
:101730002B68019A1C121340A64A9B009B58043543
:10174000F9E5043F3B68042B04D1A300ED18002CFD
:1017500000DA21E6A04B1B78002B00D009E62B68AD
:10176000019A1C1213409B4A9B009B580435E2E5EA
:10177000043F3B68042B04D0A300ED18002C00DAD2
:101780000AE6954B1B78002B00D0F2E52B68019AF6
:101790001C1213408F4A9B009B580435CBE53A1F1F
:1017A00013685B10013B06D401215B00A4000B43CE
:1017B0002D191360F0E5884B17001B78002B00D023
:1017C000D7E52B68019A1C121340824A9B009B5854
:1017D0000435B0E53A00069B0C32D31AD82B03DD52
:1017E0001A227D4B1A70C4E5FF2361005B0019408B
:1017F000FE3BFF3B19433960029906988968241221
:1018000004916D1A0299AD1089782D020D43039948
:101810009D40091A891099401D430B43BB60029BF0
:101820007D609C70E4B26E4BE4000392E358029A30
:101830009360694A1278002A03D008331D00039F81
:1018400097E51D00019A9B680C351C121340614AF4
:101850009B009B58039F6EE53B1F1C68039A069BE9
:1018600093422DD10A20E3070CD4042C13D90F2363
:1018700022681340042B11D1200001F023FE0AF04E
:10188000F5F90630643003F043FE00280FD1043D23
:10189000069B039380E50720042CF3D02000431E11
:1018A0009841FA234042FF3318400730EAE7029B91
:1018B0002100587804F028FA0023029A1370E7E711
:1018C000039B039A0C3B1B6802995B109B00D31A85
:1018D0000C3B1C601F1D1300083B1B685A108A70CC
:1018E000D2B23F49D2005B0055589B0A029A9B0036
:1018F0009560ED18039B069A043B1B685B109B00E8
:10190000D3180393344B1B78002B00D031E52B68A0
:10191000019A1C1213402F4A9B009B5804350AE57C
:101920003B1F1868FFF700FCA40006003F1B1E28A1
:1019300027DC00280DDC284B1B78002B00D018E595
:101940002B68019A1C121340224A9B009B580435B5
:10195000F1E401F00BFB033E361801F007FB214BCD
:10196000801B9842F9D81C4B1B78002B00D000E557
:101970002B68019A1C121340164A9B009B58043591
:10198000D9E40123029A137001F0F0FA029B0A389D
:1019900086195E6000E53B1F1868FFF7C5FBA400D1
:1019A00006003F1B00280DDC0B4B1B78002B00D0E2
:1019B000DFE42B68019A1C121340064A9B009B58D7
:1019C0000435B8E4084B984210DD1D22024B1A7012
:1019D000CFE4C04644CD0000A402002070CF000038
:1019E000902500203F420F0080EE36000123029A2E
:1019F000137001F0BBFAFA239B005E43029B0A3E80
:101A000030185860C8E4A300FF1A002320001A0011
:101A10003900FFF7D7FBD44ED44C3168200001F0D9
:101A200071FFD34B31681860200004F021F8316851
:101A3000200004F070F9CF4B1B78002B00D098E405
:101A40002B68019A1C121340CB4A9B009B5804350B
:101A500071E4C84BA4001B783F1B002B00D088E426
:101A60002B68019A1C121340C34A9B009B580435F3
:101A700061E4029803F0B0FDBE4B1B78002B00D050
:101A800077E42B68019A1C121340BB4A9B009B58B9
:101A9000043550E43B1F1B68002B3ED13B000C3B40
:101AA0001B68DA072CD5390001225B105800083971
:101AB00002430A60002B44DD012259001143381F04
:101AC00001603900083909681141CB1A39000C3915
:101AD0000968114224D09B189340A4001343039A31
:101AE000A350A44B1B78002B00D042E42B68019A32
:101AF0001C121340A04A9B009B580435FFF71BFCA7
:101B0000042B06D90F211A680A40092A01D15B6803
:101B1000C9E71922974B1A702BE45B10013BC9E708
:101B2000042909D90F200A680240092A04D1023386
:101B30009B005B58A400D2E719228E4B1A70FFF766
:101B400018FC0435CDE7A300069AFB189B1AD82B86
:101B500013DC0122631E002C14DC864B1B78002B47
:101B600001D0FFF706FC2B68019A1C121340824A31
:101B70009B009B580435FFF7DEFB1A227D4B1A7041
:101B8000FFF7F7FB3A601C000437E3E7069A3B1DBA
:101B90009B1A784ED82B03DD1A233370FFF7E9FB2D
:101BA000069B039AA40093422AD23B1F1868FFF7B2
:101BB000BBFA011E21DD039B0C3B1A6852108242C6
:101BC0001BDB9007801A6D4B4018C018039B8000E8
:101BD000C2583B1B1A60674B3F1B1B780437002B16
:101BE00001D0FFF7C6FB2B68019A1C121340624A12
:101BF0009B009B580435FFF79EFB20233370EAE7D8
:101C00001823FBE75A4BA4001A683B1B1F001A60FD
:101C1000584B04371B78002B01D0FFF7AAFB2B6829
:101C2000019A1C121340544A9B009B580435FFF73D
:101C300082FB3B1F1A68042A11D1A4002D194D4BB9
:101C40001B78002B01D0FFF794FB2B68019A1C1224
:101C50001340494A9B009B580435FFF76CFB1F005B
:101C6000EDE73A1F1368042B04D0002313603A00F9
:101C7000A4002D193F4B1B78002B02D01700FFF753
:101C800078FB2B6801991C120B403B499B005B5869
:101C900017000435FFF74FFBA3009C46FE1A002CEB
:101CA00017DC1C22334B1A70002333606346FF1A83
:101CB000304B04371B78002B01D0FFF75AFB2B6801
:101CC000019A1C1213402C4A9B009B580435FFF7C5
:101CD00032FB002033685A108300F15801230B4077
:101CE00003D10D21234A1170DFE749108A4200DD3C
:101CF0000A0001308442EFDC012352001343D4E791
:101D0000A3009C46FE1A002C17DC1C22194B1A70EB
:101D1000002333606346FF1A164B04371B78002BF1
:101D200001D0FFF726FB2B68019A1C121340124AC0
:101D30009B009B580435FFF7FEFA002033685A10C9
:101D40008300F15801230B4003D10D21094A117082
:101D5000DFE749108A4200DA0A0001308442EFDCF2
:101D6000012352001343D4E7C8050020A502002038
:101D700008000020A402002044CD0000FCFFFF3F2B
:101D80003B00083B1868FFF7CFF93B1F06001868B7
:101D9000FFF7CAF90023864200DA0433A4003A1B95
:101DA00017001360E54B04371B78002B01D0FFF7B9
:101DB000E0FA2B68019A1C121340E14A9B009B58E1
:101DC0000435FFF7B8FA3B00083B1868FFF7ACF999
:101DD0003B1F06001868FFF7A7F9F30FC217B042C0
:101DE0005341A4003A1B17009B001360D34B0437E8
:101DF0001B78002B01D0FFF7BCFA2B68019A1C124C
:101E00001340CF4A9B009B580435FFF794FA3B00E0
:101E1000083B18683B1F1968A600BE1B04238142BB
:101E200002D0042802D80023336018E001239C4626
:101E30001842F8D10F2302681A40042AF3D16346EE
:101E40001942F0D10429EED90B680B321340042B50
:101E5000E9D1FFF789F9431E984180003060B74B04
:101E6000A4001B783F1B0437002B01D0FFF781FA39
:101E70002B68019A1C121340B14A9B009B580435F1
:101E8000FFF759FA3B00083B18683B1F1968A6008A
:101E9000BE1B0023814202D0042802D804233360F1
:101EA00018E001239C461842F8D10F2302681A401B
:101EB000042AF3D163461942F0D10429EED90B6804
:101EC0000B321340042BE9D1FFF74EF9434258413E
:101ED00080003060994BA4001B783F1B0437002B17
:101EE00001D0FFF746FA2B68019A1C121340944A5E
:101EF0009B009B580435FFF71EFA3B00083B18680F
:101F0000FFF712F93B1F06001868FFF70DF9F317EA
:101F1000C20F86425341A4003A1B17009B00136076
:101F2000864B04371B78002B01D0FFF722FA2B6871
:101F3000019A1C121340824A9B009B580435FFF7FC
:101F4000FAF93B00083B1868FFF7EEF83B1F060064
:101F50001868FFF7E9F80023864200DD0433A40087
:101F60003A1B17001360754B04371B78002B01D008
:101F7000FFF7FFF92B68019A1C121340704A9B006F
:101F80009B580435FFF7D7F93B1F1B68A400043B9F
:101F90005A1E93413A1B17009B001360674B04378E
:101FA0001B78002B01D0FFF7E4F92B68019A1C1273
:101FB0001340634A9B009B580435FFF7BCF93B0074
:101FC000083B1868FFF7B0F83B1F06001868FFF7DA
:101FD000ABF832180120A4003B1B1F005200024343
:101FE0001A60564B04371B78002B01D0FFF7C1F95C
:101FF0002B68019A1C121340514A9B009B580435D0
:10200000FFF799F93B00083B1868FFF78DF83B1F75
:1020100006001868FFF788F8321A0120A4003B1B5D
:102020001F00520002431A60444B04371B78002BF8
:1020300001D0FFF79EF92B68019A1C121340404A09
:102040009B009B580435FFF776F93B00083B186866
:10205000FFF76AF83B1F06001868FFF765F80200F3
:102060000120A4003B1B1F007243520002431A6070
:10207000324B04371B78002B01D0FFF77AF92B681D
:10208000019A1C1213402E4A9B009B580435FFF7FF
:1020900052F93B1F1868FFF747F8061E17D11F2398
:1020A000264A1370A4003B1B1F001E60234B0437FD
:1020B0001B78002B01D0FFF75CF92B68019A1C12EA
:1020C00013401F4A9B009B580435FFF734F93B002F
:1020D000083B1868FFF728F8310007F0F9F80126E7
:1020E00040000643DEE73B1F1868FFF71DF8061E99
:1020F00017D11F23114A1370A4003B1B1F001E6041
:102100000E4B04371B78002B01D0FFF732F92B68F8
:10211000019A1C1213400A4A9B009B580435FFF792
:102120000AF93B00083B1868FEF7FEFF310007F094
:10213000B5F9012649000E43DEE7C046A40200209F
:1021400044CD00003B1F1868FEF7EEFFC217801851
:1021500050400122A4003B1B1F00400010431860A8
:10216000F14B04371B78002B01D0FFF702F92B68E5
:10217000019A1C121340ED4A9B009B580435FFF74F
:10218000DAF8A300FE1A3068012C24D1FEF7CCFF48
:102190000494079009F0C0FC0799002900DC012194
:1021A00007F07CF9049BA400C918012349001943D6
:1021B000DD4B3F1B1B7831600437002B01D0FFF74C
:1021C000D8F82B68019A1C121340D84A9B009B58E0
:1021D0000435FFF7B0F8FEF7A7FF04907068FEF72C
:1021E000A3FF049B0130C31A0793D3E7A300FE1A91
:1021F00031002000049301F00BFD049B3060FF1AB6
:10220000C94B04371B78002B01D0FFF7B2F82B68BD
:10221000019A1C121340C54A9B009B580435FFF7D6
:102220008AF83B00083B1868FEF77EFF3B1F06005C
:102230001868FEF779FF02000120A4003B1B1F0075
:102240003240520002431A60B74B04371B78002B10
:1022500001D0FFF78EF82B68019A1C121340B34A85
:102260009B009B580435FFF766F83B00083B186855
:10227000FEF75AFF06003B1F1868FEF755FF3200B5
:1022800002430120A4003B1B1F00520002431A60BE
:10229000A54B04371B78002B01D0FFF76AF82B6899
:1022A000019A1C121340A14A9B009B580435FFF76A
:1022B00042F83B00083B1868FEF736FF06003B1F5C
:1022C0001868FEF731FF320042400120A4003B1B9A
:1022D0001F00520002431A60934B04371B78002BF7
:1022E00001D0FFF746F82B68019A1C1213408F4A61
:1022F0009B009B580435FFF71EF83B1F1868FEF73C
:1023000013FFC0430122A4003B1B1F0040001043E9
:102310001860854B04371B78002B01D0FFF729F894
:102320002B68019A1C121340804A9B009B5804356D
:10233000FFF701F83B00083B1868FEF7F5FE0600C2
:102340003B1F1868FEF7F0FE320082405100012268
:10235000A4003B1B1F000A431A60734B04371B7811
:10236000002B01D0FFF705F82B68019A1C121340CF
:102370006E4A9B009B580435FEF7DDFF3B00083B8F
:102380001868FEF7D1FE06003B1F1868FEF7CCFE6A
:102390003200024151000122A4003B1B1F000A43EE
:1023A0001A60614B04371B78002B01D0FEF7E1FF68
:1023B0002B68019A1C1213405C4A9B009B58043501
:1023C000FEF7B9FF3B000C3B1868FEF7ADFE3B0083
:1023D000083B06001868FEF7A7FEF1170200C317B6
:1023E000300007F0ADF83B1F049005911868FEF728
:1023F0009BFE02000498059907F056F8430001205F
:10240000A4003E1B37001843474B30601B7804374D
:10241000002B01D0FEF7ADFF2B68019A1C12134070
:10242000424A9B009B580435FEF785FFA300FE1A25
:10243000310020000493FEF7C1FC049B3060FF1ABA
:10244000394B04371B78002B01D0FEF792FF2B6825
:10245000019A1C121340354A9B009B580435FEF725
:102460006AFFA300FF1A39002000FEF7BFFC2E4BC5
:102470001B78002B01D0FEF77CFF2B68019A1C1201
:1024800013402A4A9B009B580435FEF754FFA300D3
:10249000FE1A310020000493FEF7E8FC049B306034
:1024A000FF1A214B04371B78002B01D0FEF761FF88
:1024B0002B68019A1C1213401C4A9B009B58043540
:1024C000FEF739FFA300FF1A39002000FEF762FD76
:1024D000154B1B78002B01D0FEF74BFF2B68019AA0
:1024E0001C121340114A9B009B580435FEF723FF32
:1024F000A300FE1A310020000493FEF7BDFD049BEB
:102500003060FF1A084B04371B78002B01D0FEF710
:1025100030FF2B68019A1C121340044A9B009B5801
:102520000435FEF708FFC046A402002044CD000099
:102530003B1F186800F0C6FF3A00083A1268030013
:10254000A400D10729D4042A0CD910680F22104006
:10255000013808280FD806F01DFE052026220E0E91
:102560000E0E2400EC49180009F076FB4342584156
:102570003B1B80001860E94B3F1B1B780437002B86
:1025800001D0FEF7F6FE2B68019A1C121340E44AB4
:102590009B009B580435FEF7CEFEE249E3E7E24993
:1025A000E1E7E249DFE7E249DDE7069B3E1DF31A7A
:1025B000DA4CD82B03DD1A232370FEF7DAFE00F085
:1025C000DFFC43000120184323783860002B02D041
:1025D0003700FEF7CEFE2B68019A1C121340D04A3A
:1025E0009B009B5837000435FEF7A5FE069B3E1D59
:1025F000F31ACA4CD82B03DD1A232370FEF7B9FE59
:1026000000F0B4FCCB4B4000184001231843237862
:102610003860002B02D03700FEF7ABFE2B68019A22
:102620001C121340BE4A9B009B5837000435FEF72E
:1026300082FE069B3E1DF31AB84CD82B03DD1A23ED
:102640002370FEF796FE00F09BFCBB4B1A68831AC2
:10265000904201D2B94A9B1801205B0003433B60C2
:102660002378002B02D03700FEF783FE2B68019AF7
:102670001C121340AA4A9B009B5837000435FEF7F2
:102680005AFE00F07DFCAC4BA4001860A34B3F1B2E
:102690001B78002B01D0FEF76CFE2B68019A1C12F0
:1026A00013409F4A9B009B580435FEF744FE0123CC
:1026B000A600BE1B20001A003100FEF783FDA04CCF
:1026C0002068643002F024FF002802D1043DFEF7A8
:1026D00063FE029B21685A789A4803F02AFB012383
:1026E000029A3700137000F041FC974B22681B6878
:1026F000063253431818029B5860FEF74DFEA600A1
:10270000BE1B2000012300223100FEF75BFD8C4C34
:102710002068643002F0FCFE0028D7D0894803F01E
:1027200097F8DCE7A4003E1BFEF7CCFD37007B4B9F
:1027300030601B780437002B01D0FEF71AFE2B689F
:10274000019A1C121340764A9B009B580435FEF7F1
:10275000F2FD724BA4001B783F1B002B01D0FEF74B
:1027600008FE2B68019A1C1213406D4A9B009B586F
:102770000435FEF7E0FDA4003E1B300000F02FFC06
:102780003700664B30601B780437002B01D0FEF712
:10279000F0FD2B68019A1C121340614A9B009B5864
:1027A0000435FEF7C8FDA4003E1B300000F019FC04
:1027B00037005A4B30601B780437002B01D0FEF7EE
:1027C000D8FD2B68019A1C121340554A9B009B5858
:1027D0000435FEF7B0FDA300FE1A3100200004937B
:1027E00000F002FC049B3060FF1A4C4B04371B784E
:1027F000002B01D0FEF7BDFD2B68019A1C1213407F
:10280000474A9B009B580435FEF795FDA4003F1BEB
:10281000380000F01BFC414B1B78002B01D0FEF769
:10282000A8FD2B68019A1C1213403D4A9B009B583F
:102830000435FEF780FDA300FE1A3100200004934A
:1028400000F02CFC049B3060FF1A344B04371B78DB
:10285000002B01D0FEF78DFD2B68019A1C1213404E
:102860002F4A9B009B580435FEF765FDA4003F1BD3
:10287000380000F055FC294B1B78002B01D0FEF7E7
:1028800078FD2B68019A1C121340254A9B009B5827
:102890000435FEF750FD0121200000F029FC1F4BFC
:1028A0001B78002B01D0FEF764FD2B68019A1C12E7
:1028B00013401B4A9B009B580435FEF73CFD00214A
:1028C000200000F015FC154B1B78002B01D0FEF703
:1028D00050FD2B68019A1C121340114A9B009B5813
:1028E0000435FEF728FDA4003E1B300000F03AFC42
:1028F00037000A4B30601B780437002B01D0FEF7FD
:1029000038FD2B68019A1C121340054A9B009B5806
:102910000435FEF710FDC04680CF0000A402002061
:1029200044CD000088CF00008FCF000096CF00007C
:102930009BCF0000FEFFFF7FD005002037894100BC
:10294000C8050020A502002004000020A4003E1BB2
:10295000300000F01BFC3700EE4B30601B78043772
:10296000002B01D0FEF705FD2B68019A1C121340C5
:10297000E94A9B009B580435FEF7DDFCA4003F1B91
:10298000380000F0DDFBE34B1B78002B01D0FEF795
:10299000F0FC2B68019A1C121340DF4A9B009B58E5
:1029A0000435FEF7C8FCA4003F1B380003F0DCFC34
:1029B000D84B1B78002B01D0FEF7DBFC2B68019A6B
:1029C0001C121340D44A9B009B580435FEF7B3FCFD
:1029D000A4003E1B300003F061FD3700CD4B30609A
:1029E0001B780437002B01D0FEF7C3FC2B68019A3B
:1029F0001C121340C84A9B009B580435FEF79BFCF1
:102A0000A4003F1B380003F05FFCC24B1B78002B77
:102A100001D0FEF7AEFC2B68019A1C121340BE4A8F
:102A20009B009B580435FEF786FCA4003E1B30003B
:102A300003F060FC3700B74B30601B780437002B85
:102A400001D0FEF796FC2B68019A1C121340B24A83
:102A50009B009B580435FEF76EFCA300FF1A39005B
:102A6000200001F015FCAB4B1B78002B01D0FEF7CA
:102A700080FC2B68019A1C121340A74A9B009B58AC
:102A80000435FEF758FCA300FF1A3900200001F0BE
:102A900013FAA04B1B78002B01D0FEF76AFC2B68C1
:102AA000019A1C1213409C4A9B009B580435FEF768
:102AB00042FCA300FF1A3900200001F021FB954BD6
:102AC0001B78002B01D0FEF754FC2B68019A1C12D6
:102AD0001340914A9B009B580435FEF72CFCA30041
:102AE000FF1A3900200001F033FB8A4B1B78002BC2
:102AF00001D0FEF73EFC2B68019A1C121340864A57
:102B00009B009B580435FEF716FCA300FE1A31000B
:102B10002000049303F05AFD049B3060FF1A7D4BA4
:102B200004371B78002B01D0FEF723FC2B68019A99
:102B30001C121340784A9B009B580435FEF7FBFBA0
:102B4000A300FE1A31002000049303F047FD049B0C
:102B50003060FF1A6F4B04371B78002B01D0FEF753
:102B600008FC2B68019A1C1213406B4A9B009B586F
:102B70000435FEF7E0FBA300FE1A310020000493A9
:102B800003F034FD049B3060FF1A624B04371B785E
:102B9000002B01D0FEF7EDFB2B68019A1C121340AD
:102BA0005D4A9B009B580435FEF7C5FBA300FE1A47
:102BB00031002000049303F03FFB049B3060FF1AB8
:102BC000544B04371B78002B01D0FEF7D2FB2B6847
:102BD000019A1C121340504A9B009B580435FEF783
:102BE000AAFBA300FF1A3900200001F09DF9494B10
:102BF0001B78002B01D0FEF7BCFB2B68019A1C123E
:102C00001340454A9B009B580435FEF794FBA300F4
:102C1000FF1A3900200001F0C3FA3E4B1B78002B4D
:102C200001D0FEF7A6FB2B68019A1C1213403A4A0A
:102C30009B009B580435FEF77EFBA300FE1A310073
:102C40002000049301F028FA049B3060FF1A314BF6
:102C500004371B78002B01D0FEF78BFB2B68019A01
:102C60001C1213402C4A9B009B580435FEF763FB53
:102C7000A300FF1A3900200001F0D6F9254B1B787C
:102C8000002B01D0FEF775FB2B68019A1C12134034
:102C9000214A9B009B580435FEF74DFB069B029A88
:102CA000FB1A9B101361A300FF1A3900200002F0E9
:102CB0000DFE184B1B78002B01D0FEF75AFB2B683A
:102CC000019A1C121340144A9B009B580435FEF7CE
:102CD00032FB069B029AFB1A9B101361A300FE1A9B
:102CE00031002000049302F0F1FD049B3060FF1AD4
:102CF000084B04371B78002B01D0FEF73AFB2B68FA
:102D0000019A1C121340044A9B009B580435FEF79D
:102D100012FBC046A402002044CD00000023F7B5FA
:102D20005A1E0192002B07DA01F0C8FA02F0FEFEEB
:102D300003F05EF81923019300263000194B19683F
:102D4000B14212DD184B1A6801328A420FDAF024C0
:102D50001A601D68154F6C43E35D002B1FD0E4190A
:102D6000022B06D12000FEF7C5FA019BD8E700220E
:102D7000EDE7012B0DD1002801D100F0F7F8F0228A
:102D80006A43BB185B680A49C31A8B4201D8022305
:102D9000BB54F0235D43054BEB5C022BE2D00136C4
:102DA000CCE7C046CC05002000000020301C0020ED
:102DB0003F420F00012200210A4B0B481A611950B3
:102DC00004301950A2210420C9005850C121C0204C
:102DD0008900800258501A60044BFC311960044B82
:102DE0001A70704700A000400405000000E100E0F8
:102DF000F705002004207047F8B550C901232200D0
:102E00001A40101E2DD03340181E2AD06410002006
:102E10001C2C26D81D4B761035009E4200DD1D006F
:102E20001B4F3B5D012B05D00121200004F06CFD00
:102E300001233B55174B1B78002B01D1FFF7BAFF3D
:102E40000023154A9E420DDCFF2514491448D65C28
:102E5000B44202D15E007052D5540133042BF6D136
:102E60000420F8BDD15C8C4203D10C4A5B009D521A
:102E7000F6E70133042BF5D10023D15CFF2901D102
:102E8000D454F2E70133042BF7D1E9E788130000AB
:102E9000D8050020F70500201C0000200E000020AF
:102EA000DC05000070B530C9012322001A40101E55
:102EB0001BD02B40181E18D064101C2C00D90024E5
:102EC000174E335D012B05D00121200004F01CFDBD
:102ED0000123335569100800124A1038124B9042F2
:102EE00004D9012252421A60042070BD1C600F48B0
:102EF00006F0EEF90E4B18800E4B1B78002B02D11A
:102F0000FFF758FFF0E701220B4B9A64A922D20089
:102F10009A588018A82280B2D2009850E4E7C046A0
:102F2000D8050020908601001800002020A107008D
:102F30000C000020F705002000A00040030010B5A1
:102F40000120002B02DC1B30FEF7B6F910BD042077
:102F5000704710B5002803DC1C20FEF7ADF910BD4A
:102F60000B680020DB07FAD40D30F6E70122034B93
:102F70001A64A822D20098587047C04600800040CA
:102F800010B5FFF7F3FFFA21890006F017F910BD1D
:102F900000487047F8CF00001D20704770B5054EFF
:102FA0000400335C0D008B4202D004F0ADFC3555BB
:102FB00070BDC046D805002070B50024064D635D85
:102FC000012B05D10021200004F09EFC0023635555
:102FD00001341D2CF2D170BDD805002070470D20A2
:102FE00070473B2070470000F8B501240B680600CD
:102FF0000D00234204D10D20FEF75EF92000F8BD3C
:103000005B102000052BFAD80E4A9B009C580E4FEF
:103010003B5D002B05D00021200004F075FC00234F
:103020003B55012E06DD6B68042B03D102212000E5
:1030300004F06AFC200004F015FB0124400020434A
:10304000DDE7C046E0CF0000D8050020F8B5012636
:103050000568354202D04468344203D10D20FEF7A2
:103060002BF9F8BD6D101C2DFBD80A4F7B5D012B91
:1030700004D03100280004F047FC7E550649641056
:103080008C4202DCE143C9172140280004F070FBA8
:10309000E7E7C046D8050020FF03000070B5012413
:1030A0000D68254204D10D20FEF706F9200070BD01
:1030B0006D101C2D17D80024012804DD4C68043C39
:1030C00063425C416400094E735DA34204D0210059
:1030D000280004F019FC7455280004F049FC030092
:1030E0000420012BE3D00020E1E7C046D8050020F2
:1030F00070B504000D001C280ED8084E335C012B5F
:1031000004D0012104F000FC0123335529002000E4
:103110004D1EA94104F016FC70BDC046D805002024
:10312000036810B5DA0703D40D20FEF7C5F810BD0B
:103130004168581004394A425141FFF7D9FFF6E778
:1031400037B569460A00064B30CB30C2036802200F
:10315000042B02D100F0D4FF37BD00F0F9FFFBE7EC
:10316000A8CF000010B5084C6379002B05D00021D2
:10317000052004F0C9FB00236371052004F0F8FB6F
:1031800043425841800010BDD805002010B5084CBE
:10319000E37A002B05D000210B2004F0B5FB0023BF
:1031A000E3720B2004F0E4FB43425841800010BD61
:1031B000D8050020F7B5304D304E6B6C002B15D084
:1031C000A8240023E40037596B642D4B18680028AD
:1031D0000CDB2C4B19784A425141C9B2197004F0EA
:1031E000B1FB294B1B88DF19BFB23751AB6C002BE9
:1031F00039D00021254B264FF458A9643A780C3475
:103200000193244D8A4206D02B68032B03D8224A0F
:10321000D05C04F097FB2B68204A0133134004D59F
:103220000422013B5242134301331B4900228C46C6
:103230002B60042B18D06046C05C591CFF2802D1BB
:103240000B000122F5E7002A00D02B60012104F0D9
:1032500079FB01233B702B68114A5B009B5AE418F1
:10326000019BA4B2F450F7BD01235B422B60002305
:103270003B700C4BF3E7C046FCA0004000A00040B0
:1032800018000020F60500200C0000204405000076
:10329000F5050020D40500201C000020030000805C
:1032A0000E00002050460000084B094AFF201A80FB
:1032B0005A809A80DA800023064A07491370074A29
:1032C000087048708870C870136070470E00002046
:1032D000DC050000F50500201C000020D4050020BE
:1032E0000122024B52421A607047C046180000206B
:1032F00010B5034A0621034802F0D0F810BDC046BD
:10330000B0CF00001AD70000E12170B5490219487A
:1033100003F0A0FF002401220320174B17491A6174
:103320005C50043158508018083158501A600630EB
:1033300004F092F9FF21124AA15401341D2CFBD153
:10334000012200200F4B01001A6004230E4A0F4D8A
:103350001468002CFCD02C680002013B2043116053
:10336000002BF5D101220A4B1A6004F02FF901F06D
:10337000F1F870BDB81B002000800040040500007B
:10338000D805002000D0004000D1004008D5004002
:1033900004D00040F8B50B4E070030000D0003F0DC
:1033A000A1FF0400A84200DD2C003D00EB1B9C4265
:1033B00005DD300003F0A0FF28700135F6E720009E
:1033C000F8BDC046B81B002010B50100014803F04D
:1033D00049FF10BDB81B002010B5054C200003F0BC
:1033E0004FFFE1212000490203F034FF10BDC04629
:1033F000B81B0020C3070CD4064B1B68834208D8B7
:10340000054B1B68984204D8031F1B68002B00D093
:103410001800704700060020FC0500200023012250
:1034200010B50A48990001334250642BFAD1084C78
:10343000084B00211A602000074A08F08DF8074B5E
:10344000074A6360074B1A6010BDC046882D0020F4
:103450000406002008000020D409000030270000E6
:1034600008060020F805002010B5044B044A1A6035
:10347000044B054A1A60FFF7D1FF10BD000600207B
:1034800004060020FC050020D80F0020044B1B6818
:103490001868000980B20238C343DB171840704730
:1034A000F805002000B59BB00200054901A808F00E
:1034B00097FB01A802F0E8F902F09AFCFCE7C0468D
:1034C0007CD000000B4BC20704D4042804D80A4B5C
:1034D00000D00A4B180070470F2203681A40031DE2
:1034E000042AF7D0064B092AF4D0064B032AF1D060
:1034F000054BEFE756D00000FACB0000F4CB0000FC
:1035000060D0000070D0000067D000000020064AA4
:103510000649131F186013681B099BB202339B00F6
:10352000D2188A42F5D3704708060020D80F002031
:10353000F7B50F240126314B314A1968314B324D12
:10354000186813681F002740072F26D813681B0927
:103550009BB202339B00D218AA42F2D300242B4E16
:10356000A500AD192868FFF745FF01342860642CD9
:10357000F6D1274C2068FFF73DFF2060254C2068DE
:10358000002802D0FFF736FF20600025224B1B6881
:103590000093009B9D4214DBF7BD1B099BB29B006F
:1035A000D3189A42D2D01F68374208D1B94206D206
:1035B000B84204D3043F3F68002F00D01F60043B93
:1035C000EFE7F0236B43154A9B181A78002A01D1C4
:1035D0000135DEE71F693C2300266B43DB199B00A6
:1035E00001930136BB1BF3D4019BB4001C1B0B4B96
:1035F0001C19A069FFF7FEFEA061F2E7000600209B
:1036000008060020FC050020D80F0020882D00208F
:1036100008000020D80F0020CC050020301C00201E
:10362000F7B50124204246D1234B1B689C469842A3
:1036300041D3224B1B68019398423CD8031F1B685F
:10364000002B38D10200036800941B099BB2002BA9
:103650000FD10099131F196090422CD015682B1FB1
:103660001B68990069180C68013B14600A602A0005
:10367000EDE79D0055192968009C214219D18C4520
:1036800017D8019C8C4214D30E1F3468002C10D123
:103690000F680F343C40072C08D92F60151F2B6092
:1036A0000B680A601B099BB20A00D0E700993160E1
:1036B000CDE7013BCBE7F7BD00060020FC0500206D
:1036C0000D4970B50A000D4D1368141F1B092668BB
:1036D0009BB2981C002E0BD000238A4200D00B0016
:1036E00023608300C91880001218AA42ECD370BD71
:1036F0001B011360F7E7C04608060020D80F002022
:10370000F8B5124C27000F223B681D09ADB21342D9
:103710000DD06E1CB600A74204D032003900200044
:1037200007F007FF0022A3190436A4191A60023516
:10373000AD00074B7F199F42E5D31B1B9B10013B3C
:103740001B012360034B1C60F8BDC0460806002027
:10375000D80F0020F8050020F0B59BB0FFF706FC5D
:1037600000240700214AA300D0580134FFF758FF76
:10377000642CF7D11E4B1868FFF752FF1D4B1868D9
:10378000002801D0FFF74CFF00261B4B1B689E4210
:1037900017DBFFF795FFFFF7CBFEFFF7B1FFFFF752
:1037A000E5FB164BC21B1B6815491B6801A81B09CA
:1037B0009BB2023B08F014FA01A802F065F81BB0B6
:1037C000F0BDF02575430F4BED182B78002B01D180
:1037D0000136DAE72B695C1E002CF9DBA300EB183D
:1037E0009869FFF71DFF013CF6E7C046882D0020D1
:1037F00008000020D80F0020CC050020F80500208C
:1038000036D00000301C0020F7B5174D4F1C2B6838
:1038100006001B680C001B099BB201929F420BDB48
:10382000FFF79AFF2B681B681B099BB29F4203DBC3
:103830000A20FDF741FDFEBD2868A71CBA00DB1B6E
:1038400081181B010B6029600021031F19600F23E1
:103850001E4003002401264340C3083A9A189A42A6
:10386000E9D9019902C3FAE7F8050020F7B503008A
:103870000122134004000D000193002B2BD1174BA4
:103880001B68834227D8164B1B68834223D90F231A
:10389000144F386000681840FFF7B6FF019B3C6882
:1038A000061E3B6017D0236804301B099BB29D4263
:1038B00000DD1D00AA00211D251F07F031FEFFF7C6
:1038C00025FE2E60FFF734FE00232B602268064B96
:1038D0001340236034002000FEBDC04600060020D7
:1038E000FC050020D80F0020F0FF0F000323043058
:1038F00010B5C11719400918891000220420FFF7DC
:1039000083FF10BD70B5050008000C00FFF7EEFF47
:103910000023002804D170BDE95CC2181171013385
:10392000A342F9DBE343DB171C4000230419237196
:10393000F1E7F0B50C009BB0022804DC1C20FDF779
:10394000BBFC1BB0F0BD01230868184206D1042857
:1039500004D90F2601683140042901D00E20EEE77A
:1039600061680D001D40F9D10429F7D90A68324079
:10397000042AF3D1A2681A4201D10D20DFE7FFF734
:10398000A1FD06006068FFF79DFDA768010001AC7E
:103990007F103000257003F008F8390064232200FE
:1039A00003F068F8200008F061F901002000FFF73B
:1039B000A9FFC6E710B51C4CA544041E02D1FFF7B1
:1039C00095FF0BE002F00AFF0138062828D805F021
:1039D000E1FB090911182904240000208023DB00E1
:1039E0009D4410BD200002F075FF011B2000FFF771
:1039F00089FFF3E7200002F01BFF4300012018437A
:103A0000ECE780226946D200200002F028FF6846D9
:103A100008F02CF901006846E9E704210348E6E7CD
:103A20000020CCE70420D9E700FCFFFFC4D0000051
:103A300070B50C00022803DC1C20FDF73DFC70BDB6
:103A400001230868184206D1042804D90F2501680B
:103A50002940042901D00E20EFE761681942FAD10C
:103A60000429F8D90A682A40042AF4D1A2681A4223
:103A700001D10D20E1E7FFF725FD05006068FFF7A4
:103A800021FDA46801006410280002F08EFF2100CF
:103A900002F0CBFFFFF78EFFD1E770B50D000128D4
:103AA00003DC1C20FDF708FC70BD012408682042DF
:103AB00006D1042804D90F2102680A40042A01D043
:103AC0000E20EFE76A682242FAD1042AF8D9136877
:103AD0000B40042BF4D1FFF7F5FC06006868FFF7F4
:103AE000F1FC0100300002F060FF02F0E2FF400054
:103AF0002043D9E7F8B507000C001C20012F0BDD8F
:103B000001250868284206D1042804D90F2102683B
:103B10000A40042A03D00E20FDF7CEFBF8BD6268F0
:103B20002A42F8D1042AF6D913680B40042BF2D1AB
:103B3000FFF7C8FC06006068FFF7C4FC0100022F15
:103B400014D0A4682C4211D06410300002F02DFF74
:103B5000050002F043FE012811D1002C02DD0135E1
:103B6000012C06D12800FFF725FFD7E70124644286
:103B7000EBE7280002F0BAFE013C0500F0E702285E
:103B8000F0D1002CEEDD0135012CEBD00022280015
:103B9000110002F0DDFE02F0A9FE013C0500F3E792
:103BA00010B501240868044016D04410200005F028
:103BB00023FE154905F0EEFC07F0D4FB04F01CF8D9
:103BC0000022124B06F088FD03F0BEFF07F05AFBFF
:103BD00043000120184310BD042810D90F230268A8
:103BE0001340042B07D1FFF76DFC21000A2208F0D7
:103BF00005F90400DAE7032B01D10430F5E70D20C5
:103C0000FDF75AFBD2E7C046D30237390000D04057
:103C1000086870B501240500254006D1042804D9A0
:103C20000F2302681340042B03D00E20FDF744FB42
:103C300070BDFFF747FC03782900233B5A425341EC
:103C40001022C01808F0DAF880239B05C218044B34
:103C50009A4201D91420E9E740002043E8E7C04632
:103C6000FFFFFF3F10B5034A0621034801F016FC91
:103C700010BDC04694D000008DD0000000207047D9
:103C800010B51E20FDF718FB10BD10B51E20FDF766
:103C900013FB10BD10B51E20FDF70EFB10BD10B5B7
:103CA0001E20FDF709FB10BD10B51E20FDF704FB1B
:103CB00010BD10B51E20FDF7FFFA10BD10B51E2077
:103CC000FDF7FAFA10BD10B51E20FDF7F5FA10BD8C
:103CD00010B51E20FDF7F0FA10BD10B51E20FDF73F
:103CE000EBFA10BD10B5034A0B21034801F0D6FBD7
:103CF00010BDC04600D1000058D100000120034B88
:103D00001860034B1B68834018437047FC0F00206A
:103D1000DC0F0020F0B5EFF310810123194083F38D
:103D20001088134C134AA4461268134E013A93406C
:103D3000124F134A002B17D0146803420FD03D686E
:103D40002C60C046C046C046C046C046C046C046BD
:103D5000C0460C4C1568246825605B08EAE7654698
:103D60002C6014683460F8E781F31088F0BDC04619
:103D700008050050200000200C050050E80F00202E
:103D8000F00F0020E40F002030B585B001AD0C220B
:103D90000649280007F0C4FB0024285D01210134F6
:103DA000FFF7FCF80C2CF8D105B030BDEDD10000C8
:103DB000F7B56A46394B01AD13801C239370384B1D
:103DC0002B800A23AB70FFF7D1F8364B364CC01866
:103DD0002368984201D2002323602668002E3DD13B
:103DE0006B469F5D01213800FFF7D8F801360021AE
:103DF000380003F0A7FD032EF2D10026AF5D0121AC
:103E00003800FFF7CBF801360121380003F09AFDA6
:103E1000032EF3D1C8200138C046C046C046C04674
:103E2000C046C046C046C046C046C046C046C04662
:103E3000F1D100212878FFF7B1F868780021FFF769
:103E4000ADF8A8780021FFF7A9F8FFF78FF8FA235B
:103E500000251B01C01820602800FEBDFFF786F872
:103E6000236800259842F7D3032003F0FBFB0600EC
:103E7000042003F0F7FB36180A2003F0F3FB0B4B8A
:103E80009B1B181A0A4BA84206DB18600023094A3C
:103E9000236013600125DFE71D60F7E71A1B0000B0
:103EA0000304000010270000F40F0020E3030000CB
:103EB000DC0F0020FC0F00200022054B10B51A601B
:103EC000044B1B68934201D002F028FC002010BD77
:103ED000F80F0020DC1A002010B5041E10DA0024B0
:103EE0000A4BA400E25801239340094A0949136090
:103EF000094A1160094A0A4911600A4A136010BD53
:103F0000FFF74AF8A042EADDEAE7C046F0DE00002B
:103F1000F00F002008050050E80F0020E40F0020FB
:103F20000C05005018050050F0B53B4B85B01B68E0
:103F30000C00002B03D101204042FFF7CDFF246885
:103F400001222700174028D0FF2360121840334970
:103F50006714661040431F401E4005F0B9F9050480
:103F600038002E49784305F0B3F9000205433000CC
:103F70002A49704305F0ACF9294B28431B68202BD4
:103F800006D16400A40E274BA400E3580002184396
:103F9000FFF7C0FE002005B0F0BD042CFAD90F23B6
:103FA00021680B40092BF5D1636803925B100193E4
:103FB000019B9F42EEDABB00E3189E68039B1E4202
:103FC00028D0FF237012184072101A40134975143C
:103FD00040431D40009205F07BF9030428000F497F
:103FE0006843029305F074F9029D000205430098AE
:103FF0000A49404305F06CF9094B28431B68202B04
:1040000006D17600B60E074BB600F55800022843DD
:10401000FFF780FE0137CBE7F00F002059060000C4
:1040200020000020D4D300000200086810B5C307A8
:104030000FD540101823012A03DD4A68042A00D155
:104040000833054A1360FEF7C9FFFFF745FF00205C
:1040500010BD01204042EDE72000002010B50124F2
:10406000044002D04410200010BD042810D90F23B2
:1040700002681340042B07D1FFF724FA21000A221B
:1040800007F0BCFE0400EEE7032B01D10430F5E796
:104090000D20FDF711F9E6E70868F8B5C3071AD552
:1040A000FFF7DCFF0300203B5E2B25D805204343B0
:1040B00001221D180020114E9D4219D00521102407
:1040C000F75C3C4200D0801801395200641000298E
:1040D000F7D10133F0E704280ED90F2203681A4004
:1040E000042A09D11B099BB2002B05D00379DAE71A
:1040F000012340001843F8BD0120FCE7F9D100007E
:1041000070B508680D00FFF7A9FF04006868FFF7A5
:10411000A5FF621E0100042A14D8451E042D11D8E3
:1041200005236B439B18012215009D402B00064878
:1041300005682B430360054B1B68002B02D0200051
:1041400002F0EDFA002070BDF80F0020DC1A00200C
:1041500070B508680D00FFF781FF04006868FFF77D
:104160007DFF621E0100042A13D8451E042D10D8BD
:1041700005236B439B1801229A4007480368934329
:104180000360064B1B68002B03D00022200002F0C6
:10419000C6FA002070BDC046F80F0020DC1A0020CF
:1041A000F0B5050089B008680C00FFF757FF0690CE
:1041B000022D36DD6068FFF751FF0190A068FFF720
:1041C0004DFF04000127231D661E0793731C0293F5
:1041D000079B9E4235D0052373430593019B019DA8
:1041E00005330493049BAB421ED0042E16D86B1EDD
:1041F000042B13D80122059B2349013B5B199A40EC
:104200009446224A0B681068069A3A4003920DD0F1
:1042100062461A430A60012200280DD17F00013551
:10422000E0E701240194CDE7029ECFE76246934385
:104230000B600028F2D0039A0299280002F06FFA6E
:10424000ECE7019B1E1D042E1AD8012C18D1002565
:1042500005273B0021006B439B1999400B000A4A3C
:10426000013511689943094B11601B68002B05D07B
:10427000019B0022581D290002F051FA052DE8D1BA
:10428000002009B0F0BDC046F80F0020DC1A002065
:10429000086810B5C30703D5FFF7E0FE054B1860AB
:1042A000054B1B68002B03D0024B186802F038FA4C
:1042B000002010BDF80F0020DC1A00207FB5A04CB4
:1042C0002368002B0AD19F4A1268002A06D19E4B10
:1042D0001B68002B01D0FFF76BFD7FBD9B4D2A684B
:1042E000002A26D1984A1268002A1BD0FFF760FDE9
:1042F0000028F2D0FFF748FD924B24681A681C6032
:10430000002A16D0002C14D101AD0C2290492800AF
:1043100007F006F9285D00210134FEF73FFE0C2C62
:10432000F8D1DAE7874A1268002AE5D1002BE3D0FA
:10433000E0E700211A2003F005FB00211B2003F019
:1043400001FB00211C2003F0FDFA2E68012E5CD039
:10435000022E00D1A2E0002E50D101363100794C5E
:1043600003202368994303F0EDFA042021680140FB
:104370004B42594103F0E6FA102123680A20194004
:104380004B42594103F0DEFA8021236809011940AC
:104390004B425941062003F0D5FA802123680902D7
:1043A00019404B425941072003F0CCFA8021236881
:1043B000490219404B425941092003F0C3FA8021B8
:1043C0002368890219404B425941192003F0BAFA77
:1043D00080212368C90219404B425941182003F03B
:1043E000B1FA802321681B0319404B425941172021
:1043F00003F0A8FA31001A2003F0A4FA2B68032175
:10440000581C05F04BF8296067E702214D4C172036
:10441000236819404B42594103F094FA082123685C
:10442000182019404B42594103F08CFA802123682F
:10443000C90019404B425941042003F083FA8021FE
:104440002368490119404B4259410A2003F07AFA86
:1044500080212368C90119404B425941032003F0D0
:1044600071FA80212368890319404B425941092080
:1044700003F068FA802321681B0419404B4259411C
:10448000192003F05FFA3100062003F05BFA3100D7
:10449000072003F057FA31001B20ADE72021294CFB
:1044A0001720236819404B42594103F04BFA402131
:1044B0002368182019404B42594103F043FA8021E8
:1044C0002368192019404B42594103F03BFA8021DF
:1044D0002368490019404B425941092003F032FA40
:1044E00080212368890019404B425941072003F07D
:1044F00029FA80212368890119404B42594106203D
:1045000003F020FA80212368490319404B425941A6
:104510000A2003F017FA80212368C90319404B428F
:104520005941032003F00EFA802321685B041940EF
:104530004B425941042003F005FA01211C205BE79E
:10454000F80F0020EC0F0020FC0F0020E00F0020EF
:10455000EDD10000012010B54042FFF7BDFC10BDB9
:1045600010B5034A0921034800F098FF10BDC0466A
:10457000D4D400001CD500008023F0B502255B05D3
:104580001A690A4C0A4BA1261D5103278025F60003
:10459000ED00BA43884202D300221A51F0BD5F59A0
:1045A000002FFCD098518018F4E7C04604050000A5
:1045B00000E0014010B5002806D1C020B021400223
:1045C0008902FFF7D9FF10BDB02080218002C90207
:1045D000F7E7000043425841064B40421840B023E1
:1045E0009B02C018036800201A0E532A01D11B0237
:1045F000180A704700C0FEFF30B501248025054B26
:10460000054AED009C505C59002CFCD00160002153
:10461000995030BD00E0014004050000434258417C
:10462000074B40421840B0239B02C018A62310B588
:104630000902DB05090A1943FFF7DEFF10BDC0467A
:1046400000C0FEFFF0B5012480260D4B0D4DF60095
:104650005C51002902DC00225A51F0BD57781478D1
:104660003F022743947824042743D4780432240655
:104670003C439F59002FFCD010C00139E9E7C046E8
:1046800000E001400405000070B505004B680A0019
:104690009C1C2100A400FFF7D5FF281970BD000065
:1046A000134B1B68002B0CD08022B023D2029B023C
:1046B00000280BD11A1D5B681B0E522B00D1100075
:1046C0007047B022C02392025B02F1E782420DD90B
:1046D00003681B0E522B09D1436802339B00C0189C
:1046E000824203D903681B0E522BE9D00020E7E772
:1046F00000110020F0B50020B7B00024FFF7D0FF74
:10470000270005002600002D2ED1284D2868FFF730
:1047100061FF32003B0001900094254904A807F096
:104720005FFA04A801F0B0F8224B64201C682B68E3
:10473000A0215A425341204A5B421340B0229202C8
:104740009B18E41A6043490204F0C2FDA022520201
:10475000030000921949220004A807F041FA04A8B6
:1047600001F092F837B0F0BDFF226B6829689C46D3
:104770000233FF180B12013613409C4200DA1C0072
:10478000FF200A1402400392624601400192009108
:10479000039A0B4904A807F023FA04A801F074F85F
:1047A0002800FFF77DFF0500ADE7C046001100209F
:1047B00026D600000411002000C0FEFFD0D5000066
:1047C00012D6000070B50020FFF704FF040001209E
:1047D000FFF700FF844200DA04000A4B1D686A42BA
:1047E000554128001D60FFF7E5FEA0226B425202F2
:1047F0001340054A28009B18044A611C1360FFF708
:104800000DFF70BD00110020048001000411002084
:10481000F8B50020FFF7DEFE07000120FFF7DAFE03
:104820003E00204D0643204C0DD18021C020C902FE
:104830004002FFF7A1FE01213000FFF7EFFE1B4B06
:104840002E6023601DE0874209DD0023B0212B602C
:10485000164B8902236023680020012517E00123FD
:1048600080212B60124BC9022360F4E7120E522AFA
:1048700008D0002800D023600E4801F005F8FFF7AB
:10488000A1FFF8BD28005A68023292009B188B42A3
:1048900005D21A68561CE9D10028F2D0D1E7216070
:1048A000EFE7C04600110020041100200480010041
:1048B00004C00200EBD5000070B50020FFF7F0FE49
:1048C000FF260500002801D1280070BD03681C14D4
:1048D0003440FFF7E5FEDA2CF4D10500F2E70000E2
:1048E0008022F0B55200A1B00021674806F034FEE6
:1048F000802200215200654806F02EFE644BFF27FF
:104900001B681A00049353425A4110000592FFF7A6
:1049100051FE049C0020631E9C415E4B64421C407F
:104920005D4BE418FFF7C8FF0600002E2DD1049858
:10493000FFF750FE411C0598FFF770FE059A574D92
:10494000534B2C601A60FEF747FD514B64201B68E7
:10495000A0215A4253414F4A5B421340B0222C6877
:1049600092029B18E41A6043490204F0B1FCA022B1
:104970005202030000924A49220007A807F030F9CA
:1049800007A800F081FF21B0F0BD326813141212A5
:104990003A403B4003921A000A3A092A49D83A4B56
:1049A000039A995C002931D110223E4806F0D4FDCB
:1049B00035002B6803991A123A40914209D11A1412
:1049C0003A400B2A27D0132A2DD00A2A01D1354B81
:1049D0001D602800FFF764FE051EEAD1314B1968FF
:1049E00000290FD02000FFF74FFE04002D4B5B196C
:1049F0005968002903D02000FFF746FE0400043563
:104A00000C2DF3D1204B0121039A99543000FFF76C
:104A100047FE060089E73B40022BDADC214A9B0077
:104A2000D3185D60D5E7102200211E4806F094FDE2
:104A3000CFE71A00153A082AE8D8144A0399525CBD
:104A4000002AE3D13500152B00D015003000036893
:104A50001A143A40152A0FD01D2A00D10025FFF75D
:104A60001FFE0028F3D1002D04D020002900FFF7FD
:104A70000BFE0400054BC6E7039A1B123B409A420B
:104A8000EDD10500EBE7C046001000200811002022
:104A90000011002000C0FEFF04C00200041100202D
:104AA000B5D50000182F002010B5FFF719FF10BD75
:104AB000F0B585B0039203220333DC17294D14406F
:104AC000E4182B68284F5A42534180225B42D2029D
:104AD000A4103B409B18A21C0291244E910000910F
:104AE0000190316800980A18934215D2FFF7F8FE3A
:104AF0002B685A42534180225B421F40D202BF18AA
:104B00003368009A9B189F4206D2194800F0BCFEF9
:104B10000025280005B0F0BD029B356819066B46DC
:104B20001A7BA423DB051343FF222F00090C194332
:104B3000019B12041B04134019432800FFF75CFD7E
:104B40000837281D21003760FFF756FD002C04D0E0
:104B50000A9A21003800FFF775FD009B083BFF18FB
:104B60003760D6E70011002000C0FEFF04110020CE
:104B70008FD5000070B59AB0FFF74AFEFF221E4C99
:104B8000D2000021200006F0E7FCFF25FFF794FE8D
:104B90000026002814D10200C300E3580130591E3A
:104BA0008B41D218FF28F7D1144901A807F018F853
:104BB00001A800F069FE124800F066FE1AB070BD50
:104BC00003681A142A400A2A0AD11A122A40FF2A14
:104BD00003D0D200A1180B71A050FFF761FDD8E7F8
:104BE000132AFAD11B122B40FF2BF6D0DB00E21860
:104BF0001671E650F1E7C046902500205BD6000014
:104C00006FD600000021094B094A596001315160FB
:104C100059680029FCD00021196101239360022208
:104C2000044B8131FF315A501A607047FC1000402C
:104C30000010004000E100E00222064B0121DA678B
:104C40000022054B5A61054A11615A69002AFCD0BD
:104C50007047C04604E100E0FC1000400010004036
:104C600010B5044C2378002B01D0FFF7E5FF00209E
:104C7000207010BD09120020802301205B055B6EAF
:104C80005B001843704700000120024B1B685B006B
:104C9000184370478C1200200120024B1B685B00F8
:104CA00018437047240000200120024B1B685B0062
:104CB000184370479012002070B504000D001600D4
:104CC000FEF75EF9802301215B055A6E26700026EF
:104CD00053006170E1706272010A5A0A6071A17139
:104CE000A272010C5A0C000E5B0EA6702571E171C8
:104CF0002072E272237370BD10B5044C200006F0E0
:104D0000B5FF01002000FEF7FDFD10BD951200204B
:104D10000E4B10B51B680E4C5A1C0FD00D4C002BBF
:104D20000CD00D4C012B09D00C4C022B06D0094C99
:104D3000042B03D00A4C052B00D1074C200006F0B1
:104D400095FF01002000FEF7DDFD10BD28000020CA
:104D500000D7000088CF00000BD700008FCF0000E5
:104D600005D7000070B5214C2278002A3DD1204B98
:104D700001215A608022D20511605A68002AFCD0B5
:104D8000002207201B4B1C4901255A50043958505A
:104D900008315A5019481A4958501A491A485A5055
:104DA0001A495A50A622D2009D50082218495A503A
:104DB0000431585002201749585017491748585085
:104DC000174804395850182016495850C1218900F5
:104DD0005A500539FF395858921802435A5012490F
:104DE000124A9950FFF70EFF257070BD091200207E
:104DF000FC000040001000400C0500007469627562
:104E00001C05000024050000200004022C05000001
:104E100014050000340500003C050000FFFF000001
:104E200021100100540500000A12002004050000B2
:104E300070B50E4B06001B78002B01D1FFF792FFD7
:104E400000200B4D2C7884420ED00A4B202219787A
:104E50000323091B1940084B4901C918300006F00B
:104E60005FFB0120013C2C7070BDC0460912002080
:104E700094120020081200200A120020002370B5AE
:104E800088B0984235DD0D6801262C0034409C42E4
:104E90002FD12300042D2CD90F222B681A40230078
:104EA000092A26D16A683F2A23DD6846FFF7C0FF3A
:104EB000230000281DD06B4619783300A14203DB84
:104EC0006B461B5D5B003343A200AA18013493605C
:104ED000202CF2D1092169444A780B7812021A4336
:104EE0008B781B041A43CB781B061343024A1360CA
:104EF0000423180008B070BD9012002070B5454B17
:104F00008AB01B78002B01D1FFF72CFF02AC2000E8
:104F1000FFF78EFF002802D100200AB070BD237871
:104F20000B2BF9D96378012BF6D1E378012BF3D160
:104F300000231120384E394D33602B70684423799B
:104F4000374A4178136002780902114382781204CB
:104F50001143C27812060A4332490A60002B0ED16F
:104F6000152169444A780B7812021A438B781B0486
:104F70001A43CB781B0613433360002318E0012B40
:104F80001AD1152169444A780B7812021A438B789A
:104F90001B041A43CB781A211B06134333600E23DC
:104FA000627C6944934200DD130000229A422CD1B6
:104FB00000220420EA54B0E7022B03D1627B1033B5
:104FC0001621EEE7042B0DD115210822694468460D
:104FD00006F0A6FA0098019902F026FD06F052F9B3
:104FE0003060CAE7052BC8D11521082269446846FC
:104FF00006F096FA0098019902F016FD06F042F9C3
:105000003060627D0A231E21CBE7885CA854013200
:10501000CCE7C046091200208C1200209512002017
:10502000280000209012002010B5134B04001B78BC
:10503000002B01D1FFF796FEFFF7FEFD00200F4A7F
:105040000F49104B545058600130106058680028C8
:10505000FCD0002018610130906018690028FCD055
:10506000094B0A481B785B011B185350FFF7E4FDFE
:10507000FFF7C8FD10BDC046091200200010004017
:1050800004050000FC100040081200200A12002055
:1050900010B588B000281DDD0A68012113000B40FF
:1050A00018D1042A16D90F2014682040092811D1DC
:1050B00050683F280EDD98001018806800240842D0
:1050C00001D04010C4B26846C4540133202BF2D141
:1050D000FFF7AAFF002008B010BD000010B500289F
:1050E00013DD0C68E30710D56410532C0DD8084B62
:1050F0001B78002B01D1FFF735FEFFF79DFDA123A3
:10510000044ADB00D450FFF77DFD002010BDC046EF
:10511000091200200010004010B500280EDD0C68B8
:10512000E3070BD56410FF2C08D8054B1B78002B28
:1051300001D1FFF717FE034A034BD450002010BDE6
:1051400009120020001000402405000013B50028BB
:1051500014DD0C68E30711D5094B64100093094B6B
:105160000193072C0AD8084B1B78002B01D1FFF7BD
:10517000F9FD6B46054A1957054BD150002016BD65
:10518000E2ECF0F4F8FC00040912002000100040EA
:105190000C05000070B588B0002820DD01240868E7
:1051A00004401CD104281AD90F2302681340042B91
:1051B00015D1FEF787F9060006F058FD0500122804
:1051C00000D912252A0002210D326846FFF774FD2E
:1051D0006B465D73A54205DC6846FFF725FF00209E
:1051E00008B070BD2300325D6B449A730134F1E75F
:1051F000F0B50D008BB0012832DD086801220400F3
:1052000014402DD104282BD90F2301680B40042B07
:1052100026D16B68134223D0FEF754F96E6807005D
:105220007310019306F022FD05000E2800D90E250B
:105230002A000121113202A8FFF73EFD6A461279C9
:1052400002AB5A7302AA73129373019B76141B0E5E
:10525000D67313745574A54205DC02A8FFF7E4FE6B
:1052600000200BB0F0BD3A5D02A963189A740134B6
:10527000F1E730B589B0002814DD0C68E30711D5DB
:10528000102268460021FFF717FD6B466A4665103D
:105290005D73684663122D0E64149373D473157492
:1052A000FFF7C2FE002009B030BD0000174B184ABE
:1052B0005968002903D000215960013191601969B2
:1052C00000291FD0002018618023DB00D35811492A
:1052D000012B18D1A923DB00D3585B420B600E4988
:1052E0000B78032B01D801330B7003200B490B788B
:1052F000013303400B700A495B015B1809495350A5
:105300000123936070470860FAE7C046FC10004034
:1053100000100040240000209412002008120020F9
:105320000A1200200405000010B5034A10210348AA
:1053300000F0B4F810BDC04680D6000077D600005B
:10534000044A05491368C85401339B059B0D13603B
:105350007047C046C4160020C412002070B5114C1E
:10536000114A2368834202DC0023236016E0155CA7
:10537000411C2E00FA3E012E05D899420FDA555CE9
:10538000013D1F2D01D90800ECE70100151A565CFC
:105390006E5401318B42FADC181A206070BD157012
:1053A000FAE7C046D01A0020D016002010B5FDF74D
:1053B000DDFD064B1A68824201D900221A601B6883
:1053C000C31A034898428041404210BDC0120020D9
:1053D000204E000010B5094C094A23681268934218
:1053E00000D110BD074AD05CFDF7EEFF0028F8D0D1
:1053F000236801339B059B0D2360ECE7C816002052
:10540000C4160020C412002010B50400064B074A41
:105410001B6812689B1ADB439B059B0DA34200DBB4
:1054200010BDFFF7D7FFF1E7C4160020C816002013
:10543000F7B5050056680191B000441C063017000E
:10544000FFF7E2FFFB20FFF77BFF1C20FFF778FF51
:10545000E8B2FFF775FFE0B22412FFF771FFE0B288
:10546000FFF76EFF6B461879FFF76AFF0025AE4223
:1054700000DCF7BDAB00FB189C680135E0B2FFF71C
:105480005FFF2012C0B2FFF75BFF2014C0B2FFF72E
:1054900057FF200EFFF754FFE9E7000070B5074EF5
:1054A00033680B2B08DC0C255D43054C0133285178
:1054B00064196160A260336070BDC046CC160020E4
:1054C000282F002010B5FBF7FBFDFFF749F8FBF78D
:1054D0001FFEFDF70DFFFEF7C5FBFEF703FCFFF710
:1054E00023FF00F015FF01F01DF901F067FB10BD6F
:1054F000962210B512010021034806F02DF8002273
:10550000024B1A6010BDC046301C0020CC050020A4
:10551000064B074A1B6812689B1ADB439B059B0DD1
:105520000122834200DC002210007047C4160020D4
:10553000C8160020F8B505000C0016001F1E0ED17D
:105540000320FFF7E5FF002808D0FA20FFF7F8FE58
:10555000E8B2FFF7F5FEE0B2FFF7F2FEF8BD501D2E
:10556000FFF7D6FF0028F9D0FB20FFF7E9FEE8B2ED
:10557000FFF7E6FEE0B2FFF7E3FEF0B2FFF7E0FE72
:105580003012C0B2FFF7DCFE3C00E31B9E42E5DDBB
:105590002078FFF7D5FE0134F7E7000070B500244E
:1055A000F0250B4B1B68A34202DCFFF7A1FF70BD87
:1055B0002B006343074A9B181A78002A05D05978B4
:1055C000002311201A00FFF7B5FF0134E9E7C046B8
:1055D000CC050020301C0020F8B507000024F02581
:1055E0002B0063430C4A01349E18B74211D0317826
:1055F00000290BD00133D15C002311201A00FFF7E2
:1056000099FF2A000021300005F0A6FF0A2CE7D1FF
:10561000F8BD024B1C60F9E7301C0020CC050020CF
:10562000F0B5150001222F00754C1740A5440190DC
:105630000291002F11D005AB1A706A105A70120E29
:105640001A710522691299706D140299DD70FFF7C5
:1056500071FFCF239B009D44F0BD042D1ED90F2068
:105660002A681040042826D1022304AA28001371B6
:10567000FDF728FF040006F0F9FA624B984200D9C2
:105680001800B84204DC421C05AB02990198DEE721
:1056900001377B1EE35C05AAD355F2E7042D00D049
:1056A000A9E0032304AA043D13716B425D4105ABDD
:1056B00055710222E9E709287ED1042205AB1A7050
:1056C0006A68511000916946521209789A70009ADE
:1056D00059701F2A01DD202200926A46127806AC1A
:1056E000DA70009BBB4202DC05ABE21ACDE7012673
:1056F000BB00EB189868064006D1042837D90F2163
:105700000368194002290CD10123237043106370F0
:1057100042121B0E4014A270E07023710534013751
:10572000DFE7042921D102232370FDF7CBFE03908C
:1057300006F09CFAA31C0C2809D86070864201D19F
:105740009C19ECE7039A925D9A550136F6E70C2214
:105750006270039A925D9A550136092EF9D12E2373
:10576000E372237363730E34D9E7012907D103234E
:10577000043823704342584160700234CFE709294E
:1057800009D10423237043685A1062705B12A3701E
:10579000E6700434C3E703290BD1052323700068A6
:1057A000020992B2430F92000B40D31A63701B128E
:1057B000EDE726700134B2E7032800D049E7052160
:1057C00005AB1970110989B2520F890002408A1A7B
:1057D000111299705A701100642A00DD64210420AE
:1057E000D970C9B2041FA14201DC04324DE72C5C20
:1057F0001C540130F6E7002D00D02AE751E7C046DF
:10580000C4FCFFFF2303000070B502000024F02158
:105810000D4E0800604380194578954203D001344D
:105820000A2CF6D170BDF022002105F095FE074A42
:105830001368013BA34200D11460002329001A0021
:105840001120FFF777FEEDE7301C0020CC0500208B
:1058500010B5B2B002236A460400137006F006FACF
:10586000C72800D9C7200023984207DC421C6B469A
:10587000FE211420FFF75EFE32B010BD69460133F1
:105880005A1EA25CCA54EFE730B5B3B002236A4691
:105890000500137006F0EAF90400C72800D9C724F0
:1058A00000239C420BDC20003230FFF7ADFD621C70
:1058B0006B46FF211420FFF73DFE33B030BD694633
:1058C00001335A1EAA5CCA54EBE70000F0B5BBB026
:1058D00004900C00012803DC1B20FBF7EDFC51E0D9
:1058E0002A4B08680293C30709D4042807D90F2359
:1058F00002681340042B02D1FDF7E4FD0290234B14
:1059000060680393C30709D4042807D90F230268EA
:105910001340042B02D1FDF7D5FD039000271C4B4B
:105920001B680693069BBB420BDC039B194A009342
:10593000C821029B08A806F021F908A8FFF7A4FFD8
:10594000CAE70C267E43144B0299F618306806F01D
:1059500083F9051E05D17368B6680793079B9D42BE
:1059600001DB0137DEE730680399059606F074F92C
:105970000836002808D121000498059B0831023818
:105980005B6898473BB0F0BD0135E7E78CD000007D
:10599000CC160020DCD70000282F0020F7B5234BC1
:1059A00006001B68F02100930023009A9A4211DC44
:1059B0000024F0231A006243019201991C4A5518F1
:1059C0002F78002F12D001340A2CF3D11948FFF799
:1059D0005BFF29E00A005A43154882185078B0420C
:1059E00002D11278002A1FD10133DEE7F0223900FC
:1059F000280005F0B1FD02230D4A0199EB605354D4
:105A00000D4AF1008A58009B6E70AE70AA602F613B
:105A10006F61A34202DC054B01341C60002331009E
:105A20001A001020FFF786FDF7BDC046CC05002008
:105A3000301C002025DC00009025002010B5FFF769
:105A4000ADFDFF24084AE3005B429B18074AD35C84
:105A5000043B012B03D8E043C0B2FFF79FFF013C9A
:105A6000002CEFD110BDC046FC070000902500209F
:105A7000F7B50F00FF247F2501901E4AE300D31ADB
:105A80001D4A9A181278062A01D0032A20D1FF2233
:105A9000D2009B18186883682B401C2B18D1C36850
:105AA0001A002A40042A13D102692A40192A0FD168
:105AB0001B0A01339B000C30C018FDF703FD03786F
:105AC0000600002B10D006F0D1F80023B84209D010
:105AD000013C002CD1D1F7BD019AF15CD25C91421E
:105AE000F6D101339F42F7DCE043C0B2FFF756FF27
:105AF000EEE7C04690250020FC07000070B50500C9
:105B0000FF24084AE3005B429B18074AD35CAB4280
:105B100003D1E043C0B2FFF741FF013C002CF0D1BC
:105B200070BDC046FC07000090250020F7B5FDF7CA
:105B30001DFA514B1A68824201D900221A601A6874
:105B40004E49821A8A4200D883E01860FDF718FA9D
:105B5000071E00D101370020FDF704FB0190002053
:105B6000FDF714FB019B0090454C464D002B14D0D3
:105B70002368002B00D07AE02B682760002B00D12F
:105B800071E0414B01261B78002B63D10920FFF700
:105B9000B5FF3E4B1E703C4B1E70009B002B12D07D
:105BA0002B68002B0FD123682F60002B1ED0374BA2
:105BB00001261B78002B52D10920FFF79FFF334BA2
:105BC0001E70314B1E702368002B0FD02F4E327881
:105BD000002A0BD19F4200D227602368FB1A312B89
:105BE00004D90720FFF78AFF012333702B68002BAD
:105BF0000FD0254E3278002A0BD1BB4200D92F603E
:105C00002B68FF1A312F04D90820FFF777FF0123F3
:105C100033702368002B0CD0019B002B09D11B4E45
:105C20003378002B02D10720FFF768FF00232360A1
:105C300033702B68002B0CD0009B002B09D1124C29
:105C40002378002B02D10820FFF758FF00232B6098
:105C50002370F7BD0720FFF751FF0C4B9CE708208E
:105C6000FFF74CFFADE7009B002B9CD1ABE7009A00
:105C7000002A95D1AAE7C046BC1200200F270000D9
:105C8000AC120020B4120020B8120020B012002084
:105C900037B500240500FFF781FC01A80194FDF74A
:105CA0004FFA21002000FEF707F9FEF707FBFDF78A
:105CB000FBFAFDF715FBFEF74DFCFDF77DF9A5425C
:105CC00004D0FDF7ABFB0248FFF7DEFD37BDC04651
:105CD00016DC0000002310B501001A001120FFF7A8
:105CE00029FC10BD07B56B46197069465A7013122E
:105CF0008B701314120ECB700A716B4601000522D3
:105D00001320FFF717FC07BD10B50A000100122091
:105D1000FFF786FC10BD70B5050008000C0032309E
:105D2000FFF772FB2B00220000211B20FFF702FC73
:105D300070BD10B50C000300110014202200FFF705
:105D4000F9FB10BD012370B5FF24084A41185B42DE
:105D5000884201D3D84370BD06781D0A23407340A2
:105D60009B009B5801306B40F2E7C046F8D700001B
:105D700013B50400FE2813D80A4BC200D0580028DF
:105D80000ED0436808309900FFF7DCFF019009202E
:105D9000FFF73AFB01AB042221001720FFF7CAFBF3
:105DA00013BDC04690250020F7B50190FEF784FD95
:105DB00001250400FF276D42002C01D12800FEBD03
:105DC000266833143B40152B0DD121000198083172
:105DD00005F042FF002801D135123D402000FEF7BA
:105DE0005FFC0400E8E71D2BF8D101256D42F5E7C3
:105DF000F0B580279DB0FFF7EDFAA54CA54D2068C2
:105E0000FF00391A4019FDF7C5FA23680600C318C8
:105E10002360002B0ED11DB0F0BD2068391A281860
:105E2000FDF7B8FA236806001B182360FDF79EF8FB
:105E3000994B1860002EF0DC2B78FA2B00D037E15C
:105E40002368022B07DCFFF7B1FA0028E3D001201A
:105E5000FFF784FADFE76878AC78023818282BD887
:105E600003F0A2F919002C00300034003700400084
:105E70002A004A007C0086008A00A000F10002018E
:105E80002A002A002A002A002A002A002A002A00C2
:105E90002A002A001001FF2C0ED02000FFF7B4FCCE
:105EA00000227E4BE100CA505B181A71210000925B
:105EB00013001320FEF7FCFD0320C9E72000FFF7C5
:105EC0006DFDF9E72000FFF79FFCF5E7FFF7B6FD52
:105ED000F2E7FFF763FB0020FFF7DAFE7048FFF7F9
:105EE000D3FCE9E7632CE7D86E4BA200D25821001F
:105EF0001520FFF795FBDFE7FEF7DEFCFF27040028
:105F0000002CD9D025682B143B40152B04D0200041
:105F1000FEF7C6FB0400F3E72000083005F0A6FEFC
:105F200006000530FFF770FAFB20FFF709FA2D1283
:105F30001D20FFF705FAE8B2FFF702FAF0B2FFF70B
:105F4000FFF93012C0B2FFF7FBF925002B1B9E4270
:105F5000DDDD287AFFF7F4F90135F7E700211D2090
:105F600000910B000A00FEF7A3FDFDF757FAA3E727
:105F70002000FFF7FDFE9FE7FDF70AF803AC4A4A51
:105F800064210090494B200005F0F8FD0223200019
:105F9000237005F06BFE2300020000211620FFF79E
:105FA000C9FA89E700243D4AE300D558002D27D0DF
:105FB0006B689E00701DFFF727FA2B00002532004A
:105FC000083321000120FFF7B5FA2F00FEF774FC1B
:105FD0002E00002818D1002F04D03A000121200003
:105FE000FFF726FA002D04D02A0002212000FFF737
:105FF0001FFA002E04D0320000212000FFF718FA0B
:106000000134FF2CCFD157E7FF2103681A120A4051
:10601000A24209D11A140A400B2A08D10B400CD015
:10602000012B0CD0022B0CD0FEF73AFBD1E7132A40
:10603000FAD100252F002E00F6E70600F4E707004E
:10604000F2E70500F0E70024FFF7A8FA220021009C
:1060500000942300DA20FEF72BFDFF222100D2005E
:106060000E4805F079FA80E7012C02D1FEF742FBD9
:1060700022E7022C02D1FEF717FD1DE70120FFF7F2
:1060800007FE19E7002321001A001A2087E7C046FF
:10609000D01A0020D0160020C01200209025002029
:1060A000F8DB0000882D00200FDC00000ADC000077
:1060B000FB2B00D0CBE62268042A00DCC3E62E7955
:1060C000E878574B360206439E4200DDBFE6331D9B
:1060D0009A4200DCB7E6EB5CFE2B00D0B7E66B78AB
:1060E000AC78771E1B2B61D019D8072B47D0082B13
:1060F0001CD0012B18D1FF2C16D02000FFF784FBF9
:106100006D79484AB31E009221002A000A20FEF74A
:10611000CFFC454BE400E0501B191D7104E01D2B22
:1061200056D048D31E2B6AD0701D91E6632CFBD845
:106130006A79022A13D0032A1BD0012AF4D1E97903
:10614000AB79090219432B7AA4001B0419436B7A1B
:106150001B060B435B001343344AA350E4E7002FB4
:10616000E2DDB11E2F48FDF7CDFB304BA400E0501F
:10617000DAE7AB79A4005A1E93419B00ECE7632F4A
:10618000D2DC03AD3A002A49280005F0C9F9002302
:106190002800EB55FFF708FE0028C5DB234B8000E5
:1061A000C25821001520FFF73BFABDE7390020480F
:1061B000FFF75EFCB8E7FF2CB6D06A79022AB3D8A5
:1061C00018490B2000912100B31EFEF771FCABE7CC
:1061D000632F00DD6327002303A99F420ADCFB43F2
:1061E0000022DB173B40CB181A70152000917B1C56
:1061F0002100EAE7EA185279CA540133EDE7012C8D
:1062000092D1002F90DD6B79002B03D01C00322B34
:1062100000DD322464235C43064B1C6084E7C046E7
:10622000F6030000D616002090250020882D0020BF
:10623000D5160020040000200122094B1A60094AEB
:106240001368002BFCD00322074B1B68D8171040A3
:10625000C018012380100638400018437047C0461C
:1062600000C0004000C1004008C500400120704748
:1062700010B5064C200000F0D7FD0549200000F0C5
:10628000FBFD0122034B1A6010BDC046001B00201D
:10629000801A0600D41A002010B501210D20FCF749
:1062A0007DFE01210E20FCF779FE00210F20FCF776
:1062B00075FE044C200000F0F3FC1021200000F0DB
:1062C0000BFD10BDE01A002010B504680D20E30797
:1062D00003D56410FF2C03D91720FAF7EDFF10BD8A
:1062E000FFF7DAFFE1B2024800F018FD0020F6E700
:1062F000E01A002010B5FFF7CFFF0021034800F09F
:106300000DFD43000120184310BDC046E01A0020D7
:1063100010B5034A08210348FFF7C0F810BDC04676
:106320003CDC00007CDC00000D4B70B51B680400F9
:106330000E001500002B01D1FFF79AFFE1B2094CC6
:10634000200000F030FEF1B2200000F033FDE9B291
:10635000200000F02FFD200000F090FE70BDC04630
:10636000D41A0020001B002010B50124036823422A
:1063700005D04168214202D08268224203D10D201B
:10638000FAF79AFF10BD5810802801D91520F7E7B9
:106390004910FF2901D91620F2E75210FF2A01D92E
:1063A0001720EDE7FFF7C0FF0020EBE7F7B501226C
:1063B0001400904222DD0D682A421FD01D4B15416A
:1063C0001B684C68002B01D1FFF752FFE9B201278F
:1063D0002500194E3D40300000F0E5FD002D0FD0A6
:1063E0003C413000E1B200F0E5FC300000F046FE38
:1063F0000024A04202D02320FAF75EFF2000FEBD59
:10640000042CF2D90F2322681340092BEDD16368C5
:106410005B100193019BAB42E7DDAB00E318996889
:10642000394204D04910C9B2300000F0C3FC013534
:10643000F0E7C046D41A0020001B0020154B70B5B1
:106440001B6805000E00002B01D1FFF711FF124C55
:10645000EDB22900200000F0A6FDF1B2200000F00E
:10646000A9FC0021200000F0A9FD002801D0404235
:1064700070BD72B601222900200000F08FFD62B6C7
:10648000200000F088FC0028F2D0200000F088FCFA
:10649000EEE7C046D41A0020001B002010B50124EE
:1064A0000368234202D04168214203D10D20FAF74C
:1064B00003FF10BD5810802801D91520F7E74910B7
:1064C000FF2901D91620F2E7FFF7B8FF400020436B
:1064D000EFE7000010B50D211D20FFF7AFFF164CB0
:1064E0005A2809D101222A2122703D38FFF71CFFCA
:1064F0000122124B1A6010BD0F211920FFF79EFFD9
:10650000332805D102235F22237020211A38EDE7BA
:106510000D211E20FFF792FFC7280AD10323002276
:106520002A21A9382370FFF7FFFE1B222A211E20F3
:10653000DCE700232370DBE72C000020D81A0020C2
:10654000204B10B51B680400002B01D1FFF7C2FFE0
:106550001D4B1B785BB2022B0AD0032B29D0012BD9
:106560002CD121001D200124FFF768FF644205E0C3
:10657000012C13D129211920FFF760FF7F2801DDAD
:106580000138FF3803007F3301DA7F204042C823FF
:106590007F21584302F09CFE604310BD032C0BD1B9
:1065A0002B211920FFF74AFF043CE7E72D21192092
:1065B000D9E721001E20D6E7052CF7D001240020C2
:1065C0006442E4E7D81A00202C00002010B5012016
:1065D000FFF7B6FF43000120184310BD10B503209C
:1065E000FFF7AEFF43000120184310BD10B5052092
:1065F000FFF7A6FF43000120184310BD144B70B5F0
:106600001B68002B02D10120FFF79AFF114B1B786A
:106610005BB2013301D1FFF75DFF0120FFF790FF6F
:1066200004000320FFF78CFF05000520FFF788FF1B
:106630006D43644340436419201804F059FE01F08F
:1066400023FB04F01FFE43000120184370BDC04629
:10665000D81A00202C000020F8B501231C00984215
:106660002BDD0F683B4228D04E6835001D4024D1F9
:10667000042E22D90F2231680A40092A1DD17368DD
:106680005C10202C00DD2024144B1B68002B01D152
:10669000FFF7EEFD72B67F10F9B2114F22003800FD
:1066A00000F07CFC62B6A54214DA380000F073FBFF
:1066B000002804D101246D002C432000F8BD3800CF
:1066C00000F06EFB0122AB004000F318104398600D
:1066D000AD18E8E764000125EEE7C046D41A0020B3
:1066E000001B0020002070470120704700207047E9
:1066F000002070470120704700207047002070473D
:10670000002070470020704700207047002070472D
:106710000020704700207047002070477047704786
:106720007047000010B5034A0E210348FEF7B6FE7D
:1067300010BDC046CCDC00003CDD00000378013B0E
:106740001F2B00D970470130F8E710B5FFF7F6FFAF
:106750000378002B0BD00130222B11D10378002BB2
:1067600003D0421C222B03D11000FFF7E7FF10BD1E
:106770005C2B03D14378002B00D0821C1000EDE786
:106780003A2BF2D02C2BF0D07B2B0BD1FFF7D6FF7E
:106790000378002BE9D07D2B01D10130E5E7FFF72D
:1067A000D4FFF5E720225B2B14D1FFF7C7FF037856
:1067B000002BDAD05D2BF0D0FFF7C7FFF7E7202BD7
:1067C000D3DD2C2BD3D0190091435D29CFD0222BC0
:1067D000CDD001300378002BF1D1C6E7002210B5EF
:1067E000904216D0FFF7AAFF03780422222B10D084
:1067F000023A7B2B0DD0013A5B2B0AD019003039BD
:106800000232092905D92D2B05D1417830390929C2
:106810000AD8100010BD0522742BFAD00132662B65
:10682000F7D001326E2BF4D0581E83415A42F0E764
:1068300070B5FFF783FF037801222D2B01D180185B
:10684000023A00230A2502E06B430130CB1801789D
:106850003039CCB2092CF7D95A43100070BDF8B5C5
:106860000C001500FFF76AFF0378222B02D00023EB
:106870002370F8BD0D236A1E210008250C260A2767
:106880009C4601300378222B02D100230B70F0E7E5
:10689000002BFAD0441C5C2B0BD14378841C622B58
:1068A0000ED0662B0ED06E2B0ED0722B0ED0742B0A
:1068B0000ED0002AE9DD0B70013A01312000E1E73A
:1068C0002B00F6E73300F4E73B00F2E76346F0E71E
:1068D0000923EEE710B50400FFF737FFA04202D905
:1068E0000378202B00D910BD0138F7E710B5002838
:1068F00015D00378002B13D0FFF720FF2021037859
:1069000002008B4300205D2B09D01000FFF71DFF14
:1069100003782C3B5A425341C018FFF70FFF10BDBC
:106920001800FCE70300002070B50C0081420EDD6A
:106930001A785B2A0BD1581CFFF700FF0125AC42E7
:1069400005D0FFF7D3FF002801D00135F7E770BD70
:1069500070B50C001500002901D000230B70002831
:1069600020D00378002B1ED0FFF7E8FE0378060046
:106970002C2B03D10130FFF7E1FE06003378002015
:106980007D2B0FD0844204D02A0021003000FFF775
:1069900066FF3000FFF7D9FE03783A2B02D10130B1
:1069A000FFF7CCFE70BD1800FCE7F0B50D00040049
:1069B0009DB02E78002E35D02E21280005F03EF90E
:1069C000071E14D0431B0193303E092E14D8280013
:1069D000FFF72EFF01002000FFF7A4FF0400002CAA
:1069E00020D0002F1ED0019B0133ED18E1E72800D5
:1069F00005F03CF90190E7E723787B2B11D1601C6F
:106A0000642203A9FFF7A4FF041E0BD0019A2900FA
:106A100003A805F032F90028E1D02000FFF795FE29
:106A2000EEE7002420001DB0F0BD70B50500002089
:106A30000C0081421DDD2800FFF7D0FE0300681C1A
:106A4000012B14D00020022B13D10022681C11004E
:106A5000FFF77EFF012C0CD0FFF748FF002211004A
:106A6000FFF776FF013CF5E7FFF740FF013C012C03
:106A7000FAD170BDF8B5050000200C0016001F000B
:106A800081420DDD2800FFF7A9FE03000020022B44
:106A900006D1681C3A003100FFF75AFF012C00D1E3
:106AA000F8BDFFF723FF3A003100FFF751FF013C2B
:106AB000F4E710B50024A04218D0FFF73FFE03789A
:106AC0007B2B0AD1013000221100FFF741FF002883
:106AD0000CD0FFF73AFE0134F5E75B2B06D101300D
:106AE000FFF704FF002801D00134F9E7200010BDB2
:106AF000F8B5002816DD0D68EB0713D56D10013DC4
:106B00000124FDF7D9FE0026FF27644200280CD19E
:106B1000002E21D0300005F0A9F801003000FCF76C
:106B2000F1FEF8BD01256D42EAE703681A143A4008
:106B3000152A0BD11B123B409C4200DA1C009D42DF
:106B400001D106000836FDF7ABFDDFE71D2AFAD1BB
:106B5000012400266442F6E701200134640020434A
:106B6000DFE7000010B508680C00FCF7ABFCFFF78E
:106B70001BF9002803DB6268024B8000C250002032
:106B800010BDC046882D002010B50868FCF79AFC9F
:106B9000FFF70AF90123002802DB024B8000C358EB
:106BA000180010BD882D002010B50868FCF78AFC7D
:106BB000FFF7FAF8C043C00F800010BD10B5034ABC
:106BC00004210348FEF76AFC10BDC046CCDD00007E
:106BD000C5DD000010B5FCF797FBFCF745FCFEF7A0
:106BE00071FC0448FEF750FEFDF7C4FFFEF726FFD8
:106BF00010BDC0461BDE000010B5FCF78FF810BDBD
:106C000070B5002504AC24780573A94205D10A4B60
:106C10000A4A23210A4804F015FC01600949920040
:106C200052589B0002715B58A400837163588560C1
:106C300043710223C37170BD33DE000092DE000099
:106C400041DE0000F0DE0000037B002B04D1437323
:106C50008373036101330373704700001FB5019113
:106C6000A02100240068C900D2B24450012A10D0EB
:106C7000A24209D0032A0AD0074A8350074B019A3F
:106C8000C250012343501FBD02221343F4E70422E4
:106C9000FBE70622F9E7C046540500002405000082
:106CA00010B50400FFF7D0FFA1222368A179D2001C
:106CB00099506179064A20009950217904329950FF
:106CC000044B19685A689B68FFF7C8FF10BDC0469F
:106CD0000C050000F41A00204BB2002B0FDB8023C0
:106CE0003F290FD81F290FD80F290FD807290FD8F0
:106CF00003290FD81B060168074A8B507047802371
:106D00009B04F8E7DB04F6E71B05F4E75B05F2E715
:106D10009B05F0E7DB05EEE7240500000368074A62
:106D200099501A00FC32D1680029FCD0A321C90077
:106D300058580023C0B2D3607047C0461C050000FD
:106D400007B58022074BD2051A6000229A600232F2
:106D50001A710F230C3200930349023B0348FFF7DB
:106D60004FFF07BDF41A002000300040E01A002059
:106D7000F8B505000E0017000024BC4208D02B68AF
:106D8000315D1B6828009847002801D00134F4E7E2
:106D90002000F8BD704710B51C3000F0A9F910BDF7
:106DA00010B51C3000F096F910BD10B51C3000F085
:106DB000A5F910BD70B5437E0D00002B01D1002058
:106DC00070BD6430040000F0A2F90028F7D1200063
:106DD000290000F070F90120F2E70000F7B50193F7
:106DE000FA23002504009B0083600D4B45600833A7
:106DF00003601C300F00160000F052F920006430D0
:106E000000F04EF9074A2761B600B35820006375B9
:106E1000019B9B009B586576A576A375FEBDC04679
:106E2000D0DE0000F0DE00000123A022C375837DC8
:106E30000E49C133FF33D2059B009950437DC133C6
:106E4000FF339B009950CC220169094B5204CA5070
:106E500005220169243BCA50827D01690833CA506A
:106E60000269417D034BD1507047C0460C060000BB
:106E7000240500000C050000A022002310B50469C1
:106E8000D200A3500A4CA1420FD90A4C8C425B415C
:106E900009495B420B40CD21C9045B1804690749CD
:106EA000635005210369995010BDCC235B04F5E7BD
:106EB000A086010090D00300000098FD240500008A
:106EC000F7B5040000200D000193824265D0160042
:106ED000402A00D9402627001C37380000F0F6F879
:106EE000B1232269DB00D550802201232169920061
:106EF0008B50A27E002A03D122691362226913609B
:106F00000025731EAB4207D1019B002B04D08022C9
:106F10000221236992009950012223691A62236990
:106F2000FC33DA68002A02D19A6A002AF9D09A6AF8
:106F3000002A0BD1DA60A3232269DB00D158380084
:106F4000C9B2013500F0B7F8B542DAD3019B226926
:106F5000002B0FD11300FC339B6A002B0AD10133A5
:106F6000A376D3612369FC33DA6C002AFCD00022BB
:106F7000DA640AE000230121A37651611A00236933
:106F8000FC3399680029FCD09A602369FC339A6A23
:106F9000002A01D000229A62E8B2FEBD10B501239A
:106FA000FFF78EFF10BD0300AC3310B5040019705D
:106FB000643000F08BF80123637610BD00230200DB
:106FC00070B5AC3243760D001178B122040000692F
:106FD000D20081508022216992008B5022690133B6
:106FE00013622269936026006436300000F080F856
:106FF000002812D0300000F06DF81E4B2269D050EE
:107000002369FC331A6A002A02D19A6A002AF9D04D
:107010009A6A002A01D11A62E5E723690122002D4C
:107020000DD11900FC31896A002908D1DA61236980
:10703000FC33DA6C002AFCD00022DA6407E05A61E3
:107040002369FC339A68002AFCD000229A60002051
:107050002369FC339A6A82420BD098622169064AFE
:107060008B588B501800022B03D0181F431E9841D9
:10707000033070BD1C050000C404000010B50121E0
:10708000FFF79CFF10BD000010B513231422024926
:107090000248FFF7A3FE10BD00400040001B002087
:1070A00010B540220021040004F056FA002320000D
:1070B0002364636410BD10B53F24026C531C23404D
:1070C000446C9C4201D08154036410BD00230364CE
:1070D00043647047436C026C934206D03F21C25C0C
:1070E00001330B4043641000704701204042FBE72E
:1070F000036C406C181A00D540307047436C026C2A
:10710000934201D0C05C704701204042FBE73F2220
:10711000036C406C01331340181A43425841C0B20B
:107120007047000003210A4802680A4302600948C8
:1071300002680A4302600849084A094B9B1A03DDAA
:10714000043BC858D050FBDC00F012F8F8F7DCFF25
:10715000240500405405004044E4000000000020E5
:1071600064020020FEE7FEE7FEE7FEE7FEE7FEE73B
:107170002D4B10B51A68D2B2012A0FD12B4A1268D2
:1071800012070BD12A4AE0241168F02208001040AF
:1071900021422DD12749096811422CD01A68D2B258
:1071A000012A12D12149096809070ED1F02020498E
:1071B00009680140402908D11E490968014204D1EB
:1071C0008020C121C005C90042501B68DBB2012BE1
:1071D0000DD1164B1B681B0709D1154B1A68F023FC
:1071E0001A40A02A0FD1134A12681A420ED010BDBD
:1071F0003028CFD0D2E7104A104911608021104AC0
:1072000009021160CAE7D02AF1D1ECE70D4B1A68E8
:10721000012A04D00C4A1A601A68012AFCD1C02243
:107220000A4B1A60E3E7C046E00F00F0E40F00F0FD
:10723000E80F00F0EC0F00F004050040DFFF07C08E
:10724000186C004000EC06407593000014EC0640FA
:107250000120704710B503681322DB69984710BD01
:1072600070470000054B0269D1500369FC331A6A6C
:10727000002AFCD0002201201A6270471C05000081
:10728000030010B55C331A781F231A401E3B190007
:107290009140114AD167C222042104699200A15091
:1072A000026953600269D360A02300220169DB00F8
:1072B000CA5001230169094A5B428B500169084A9F
:1072C0008B5001690C3A8B50016908328B50143095
:1072D000FFF7FCFE10BDC04604E100E00C05000015
:1072E0001405000010B51430FFF702FF10BD10B5F3
:1072F0001430FFF703FF10BD10B51430FFF7EAFE9E
:1073000010BD0000030070B55E331A780469724B3B
:10731000E25003005D331A780469704BE2500300B9
:1073200061331C7802696E4B012C00D09EE0050091
:107330005F352E78A225ED00565102006032157897
:10734000A1220669D200B5500269D4509623DB0011
:10735000994200D88CE096231B01994200D88AE01C
:1073600096235B01994200D888E096239B019942BD
:1073700000D885E0E1239B01994200D882E0962362
:10738000DB01994200D880E0E123DB01994200D87B
:107390007DE096231B02994200D87AE0E1231B028C
:1073A000994200D877E096235B02994200D874E0B6
:1073B000E1235B02994200D871E0E1239B029942EC
:1073C00000D86EE0474B994200D86CE0E123DB0225
:1073D000994200D86AE0E122002312038A425B410D
:1073E000414A5B421340802252059B1801693F4A83
:1073F0008B50A02304220169DB00CA5000210369DD
:10740000FC33D9600369FC331962012301690B6005
:1074100001698B60C1210469890062501F215C30C1
:1074200002780A4093406231314AFF3153500021C3
:10743000415600293CDA0F230B40083B2D4C9B089A
:107440009B001B1903242140A140FC348C40DD69C2
:10745000A5432C00C0258D4029002143D9611F235D
:10746000017819401E3B8B40136070BD00246CE70F
:107470009E23DB02BAE79D231B03B7E71E4BB5E74C
:107480001E4BB3E7EC239B03B0E71D4BAEE71D4B50
:10749000ACE71D4BAAE71D4BA8E71D4BA6E71D4B0C
:1074A000A4E71D4BA2E78023DB049FE71B4B9DE76E
:1074B0008C080F4BA400E41803230B40FF21C025C8
:1074C000DB009940AD0066598E433100C0269E40D6
:1074D00033000B436351C2E70C05000014050000A4
:1074E0006C05000090D0030000D0BEFE2405000013
:1074F00000E100E000ED00E000B0130000502700C4
:1075000000A04E0000F0750000509D0000F0EB0060
:1075100000903A0100E0D70100B0AF0300705F07B0
:10752000F7B5009308AB1B7800250193FA230400FC
:107530009B0083600E4B45600833036014300F00DE
:107540001600FFF7ADFD23005C3327611E70009B22
:10755000084A9B00995823005D331970019B200055
:107560009B009A5823005E33DD701A70FEBDC04642
:1075700074DF0000F0DE0000036910B51A00FC3271
:10758000D2680400002A0AD0A322D20099581430ED
:10759000C9B2FFF790FD00222369FC33DA6010BD09
:1075A00010B50248FFF7E8FF10BDC046B81B002029
:1075B000162307B5022200930249013B0248FFF758
:1075C000AFFF07BD00200040B81B002010B5002809
:1075D00001D004F07DFA10BD7047000010B500F036
:1075E00011F8FFF7F9FF012000F000FAFFF7F2FAB7
:1075F000FFF702FB024B002BFAD000E000BFF7E7D9
:1076000000000000C420114B80001A58104911409E
:10761000C02212020A431A50C0218022490092025D
:107620005A501A608023A3220021DB05D200995012
:107630000122F9309A60074BFF301950C120023106
:1076400080001950403019501A60704700E100E086
:10765000FF00FFFF00100140014B18607047C0465B
:1076600078000020F7B5002320285AD8384B800036
:10767000C258042A5BD007D8022A54D055D8042314
:10768000012A09D000234CE0062A54D051D31A2AEB
:1076900053D002231B2AF5D12E4A116808294ED94E
:1076A00009294FD00A240226A02001252A4AC00019
:1076B00015502A482A4D07681C20BF00074029485A
:1076C000019700685759009027481B0207401F4345
:1076D000C02300989B020340FF20575157590002D6
:1076E00007401F43019B1F43009B58016023184024
:1076F00007433E43565101251C4B1560586800282E
:10770000FCD000205860A1230125DB00D358556030
:10771000A025ED0050511BB2A14202D015D2611A32
:10772000CB401800FEBD0823B6E71023B4E72023A2
:10773000B2E74023B0E78023AEE70123ACE708249B
:107740000026B1E70C000126AEE7091B8B40E8E7F5
:10775000F0DE0000740000200070004030000020C7
:107760000405000034000020FF00FFFFFC70004013
:10777000F0B520285BD8364B8000C258354B1E68C8
:10778000002E30D1C227344BBF00D859334C0325CB
:107790000440C02000022043D851C024802064004F
:1077A000800018512E4F18602E4B803CD859FF3C5A
:1077B000A043D8510437D859A8432043D85108379B
:1077C000D8590C35A8438446072065462843D8512C
:1077D000A820C0001E50C1208026800076021E50C6
:1077E0001C601C4B1C60142500202B001E4C2E001E
:1077F00046433659771C1BD14343E250A02303254F
:10780000C132FF329200DB05D550184B1A68082AA6
:1078100014D114234343E3189A6812485132FF32BB
:10782000920059601150DA68C1239B00C250F0BD2C
:107830009642E1D001300328D9D1F8E7082A02D9CD
:10784000083AD140E5E708239A1A9140E1E7C0469B
:10785000F0DE00001C1C002000E100E0FF00FFFF44
:10786000040500000090004038000020780000204F
:107870002149F0B54A6C2148002A14D0A025A12640
:1078800000230124ED05F600C258571C06D0C71886
:107890007F68002F02D027009740AF5114333C2B54
:1078A000F2D100234B64A0230121DB0500260F0049
:1078B0009C4614234B43C3181A1F1268104C0E4DDC
:1078C000920014195219526C002A10D01A00143A5E
:1078D0001268551C09D0103B1B68FF2B05D03B00DC
:1078E000934065461A00074BEA50FC346664013148
:1078F0000429DED1F0BDC046FC90004038000020D5
:10790000009000400C05000000B5202810D80C4A5B
:107910008000835803290BD8A0220800C133FF330D
:10792000D2059B0001F036FC020905070021D15069
:1079300000BD0C21FBE70421F9E70321F7E7C0466E
:10794000F0DE000020280AD8074B8000C25801232F
:107950009340A022D205002902D104495350704718
:10796000A121C900FAE7C046F0DE00000C050000C6
:1079700003000020202B0AD8A021A222C905D20092
:107980008858034A9B009B58D840012318407047F1
:10799000F0DE0000F7B506000D000C008B18019317
:1079A000019B671B9C4207D0336821781B6830001D
:1079B000984701340028F3D13800FEBD0849094A30
:1079C000094B10B51B688858FA22190A1B06184380
:1079D0009200002301F0B4FD4904C00B084310BD20
:1079E0000010014004050000201C002070B5041E9A
:1079F00009D0FFF7E3FF050000F014F8FFF7DEFF02
:107A0000401BA042F8D370BD0022044B9A60044A88
:107A100013680133DBB213607047C046FC100140AD
:107A2000201C002070470000F0B5C64600B5CB0F03
:107A30009846404A4B005B0D9A1882B00D00040036
:107A4000132A2FDC002A49DB3B4F17413E000E4032
:107A5000064323D07F08390029400C430AD0374918
:107A6000BD438C4663445C425C418023DB0213418E
:107A7000E4071D434146CE0031492B008E192200F8
:107A8000346875682000290001F000FF0090019122
:107A90000098019922002B0003F090F802B004BC7A
:107AA0009046F0BD332A08DD8023DB009A42F5D1F1
:107AB00002000B0001F0EAFEF0E7224A94460122A0
:107AC00063445242DA400242E8D052080242D1D026
:107AD00094438022D2051A411443CBE74B005B0844
:107AE0000343DBD00B031B0B1C4363422343802463
:107AF0004D0C24031B0B23406D042B4319004346FC
:107B0000DA000F4B9B181C685D6802000B00200018
:107B1000290001F0BBFE009001910098019922001C
:107B20002B0003F04BF842464B005B08D60733436B
:107B30001900B3E701FCFFFFFFFF0F00EEFBFFFFA3
:107B4000A8DF0000EDFBFFFFF8B5274A4B005B0DF7
:107B50009A180C000700132A10DC002A36DB234B8E
:107B600013410B423AD080242403144100206418AE
:107B70009C430600250030002900F8BD332A0EDDA5
:107B800080230600DB000D009A42F4D102000B00B6
:107B90003800210001F07AFE06000D00EBE7144DDD
:107BA0000600AC46012563446D42DD40AC466346A9
:107BB0000D000342DFD033239A1A323B934018184A
:107BC000874200D94C1C63469843D2E7C90FCC07C3
:107BD0000020531CCDD1074B1C43CAE706000D0003
:107BE0000028C0D1C7E7C04601FCFFFFFFFF0F0020
:107BF000EDFBFFFF0000F03F30B5214A4B0087B09E
:107C00005B0893421EDD1F4A934205DD02000B0014
:107C100002F0D4FF07B030BD02AA00F095F80323AC
:107C20001840049A059B012813D002281DD0002873
:107C300014D00298039900F06FFB80231B069C462A
:107C40006144E7E7002300220093002301F0DEF8FF
:107C5000E0E70298039900F05FFBDBE7012402985C
:107C60000399009401F0D2F8D4E701240298039913
:107C7000009401F0CBF880231B069C466144C9E7C1
:107C8000FB21E93FFFFFEF7FF0B54746CE4680B5C9
:107C90008DB004000D0000F067FA294B06001B7838
:107CA0000F005BB29846013310D022002B00200059
:107CB000290003F0CBFA8146002807D100220023D7
:107CC0002000290001F014FC002806D13000390002
:107CD0000DB00CBC90469946F0BD01230293194BA0
:107CE0000694079503934B460A93434604940595DF
:107CF000002B15D0002300221900100002F0E2F83A
:107D0000434608900991022B0ED103F0B9FB2123C1
:107D100003600A9B0193002B0CD1089E099FD5E7B5
:107D2000002300240893099402A801F0C1F9002857
:107D3000EFD1EAE703F0A4FB0A9B01930360ECE7B1
:107D40007C000020B8DF0000F0B54E464546DE4618
:107D50005746E0B5E14B4C008FB090468946640829
:107D60009C4200DC87E0DE4B9C4222DCDD4A00299D
:107D700000DC92E0DC4B02F021FFDB4B06000F0041
:107D80009C4200D17EE1D94AD94B02F017FF020094
:107D90000B00414630000A604B60390002F00EFFD4
:107DA000D34BD24A02F00AFF434601259860D960BE
:107DB0006BE0D04B9C4200DC8FE0CF4B9C4200DD5F
:107DC00055E1CE4A231592469A4451460905631A55
:107DD00019001D00040003F055FA03F089FA0200AF
:107DE0000B00200029000892099302F0E7FE002210
:107DF000C34B02F071FC0F00060003F043FA03F0DE
:107E000077FA04000D0002000B00300039000A94DC
:107E10000B9502F0D3FE0022B94B02F05DFC00226C
:107E200000230C900D9101F05DFB002800D192E140
:107E3000002300222000290001F054FB434243416B
:107E40000133B04A41460192022208A800925246EC
:107E500000F07CFB4B460500002B16DA80224346DF
:107E60001206944642465B68454263445360D368B9
:107E70006344D36009E00B00020041460A604B6096
:107E80000022002300258A60CB6028000FB03CBC94
:107E900090469946A246AB46F0BD934B01F0F6FCE6
:107EA000914B06000F009C4200D13DE18F4A904B60
:107EB00001F0ECFC02000B00414630000A604B6010
:107EC000390002F07BFE894A894B01F0DFFC012575
:107ED00043466D429860D960D7E701F049F88A4A75
:107EE0008A4B06000F0002F0F7FB0022884B01F0DE
:107EF000CDFC03F0C7F9050003F0FAF9794A7A4B93
:107F00000490059102F0E8FB02000B0030003900FC
:107F100002F054FE754A06000F0004980599744B50
:107F200002F0DAFB029003911F2D00DCC7E0029AF9
:107F3000039B3000390002F041FE83468A465346D7
:107F40005B0024155B0DE31A102B6CDD049805997A
:107F5000D322674B520502F0BFFB02000B0030003A
:107F600039000292039302F029FE0A000100130077
:107F70000691079202003900300002F01FFE029ABB
:107F8000039B02F01BFE06000F0004980599614A4E
:107F9000614B02F0A1FB32003B0002F00FFE069E97
:107FA000079F0B000200390030000292039302F099
:107FB00005FE4B005B0D83468A46E41A312C32DD08
:107FC00004980599B822544B920502F085FB0300F2
:107FD0000C000200029303940B000698079902F02C
:107FE000EDFD02000B0006000F000698079902F055
:107FF000E5FD029A039B02F0E1FD484A02900391DD
:1080000004980599464B02F067FB029A039B02F025
:10801000D5FD02000B00300039000292039302F0FC
:10802000CDFD83468A465A465346414630000A6093
:108030004B60390002F0C2FD029A039B02F0BEFDC4
:1080400044460B000200A260E3604B46002B00DBBD
:108050001BE75B46236080231B0653446360802339
:108060001B069C466144A060E1606D420DE70B0079
:10807000020002F0A3FD434600259860D960186015
:10808000596002E7D3221A4B520502F097FD214AAC
:10809000214B0D00040002F091FD02000B0041464F
:1080A00020000A604B60290002F088FD1A4B194A33
:1080B00002F084FD434601259860D960E5E60200A0
:1080C0000B003000390002F079FD6B1E154A9B0051
:1080D0009B5883468A46A342A5D130E7FB21E93F5E
:1080E0007BD9024000004054FB21F93F3163621A02
:1080F00061B4D03DFB213941FFFFEF7FEAFBFFFF79
:108100000000704140E0000083C8C96D305FE43F6B
:108110000000E03F7370032E8A19A33BC14920255C
:108120009A837B39C0DF0000D3220C4B520501F04B
:10813000ADFB0B4A0B4B04000D0001F0A7FB020046
:108140000B00414620000A604B60290002F036FD1A
:10815000034A044BB9E6032373E6C04661B4D03D3D
:108160007370032E8A19A33BF8B54746CE46674B7A
:1081700080B50A000F00190005003940994200D16E
:108180009BE004000100002F69DD3F1500D1B4E041
:108190005F4B12039C468023120B5B0313435B006F
:1081A000CA0F67449B184A00F80703D5D20F5B003B
:1081B0009B188A0079108C4600218020162489465D
:1081C00080030D189D4202DC29185B1B8144D50FEA
:1081D0005B00013C5B1952004008002CF1D10020EB
:1081E0008046802020250027000609E08B425CD0D5
:1081F000D40F5B00013DE31852004008002D16D05B
:10820000C4198B42F2DD27180E00002C49DB5B1AE3
:10821000A242894149425B1A121BD40F5B00013D07
:1082200080443100E31852004008002DE8D1134388
:108230004ED143465B0837494A4688464946521064
:108240004244C90702D5802109060B4361460F0548
:10825000BD18180029000CBC90469946F8BD7B005B
:108260005B0803433900002BF5D0002F3CD1E30A13
:10827000153A6405002BFAD08020400303423FD119
:10828000002700E00F005B00791C0342FAD02500B4
:1082900020208D40401A2900D71B2200C2401A43DB
:1082A00076E7FE43F60F8E19B1E79442A0D827185F
:1082B000002CF6DB1E000023AEE702003B00280086
:1082C000390002F009FA2A003B0001F0DFFAC2E7A8
:1082D0004346013303D0434601335B08ABE7012338
:1082E00098460023C144A6E73B00020002F066FC6A
:1082F00002000B0001F0E6FDADE713000022BBE732
:108300000127210020207F42C6E7C0460000F07F01
:1083100001FCFFFF0000E03FF0B54746CE4680B5C8
:1083200087B000920193754B4F00814688467F08C5
:108330009F4263DC02F0A6FF002800D1D4E04A4649
:1083400043464846414602F0C7F904000D006C4A16
:108350006C4B02F0C1F96C4A6C4B01F097FA2200A9
:108360002B0002F0B9F96A4A6A4B02F027FC22009E
:108370002B0002F0B1F9684A684B01F087FA22003D
:108380002B0002F0A9F9664A664B02F017FC2200A6
:108390002B0002F0A1F9644A644B01F077FA220045
:1083A0002B0002F099F9029003910022604B20000B
:1083B000290002F091F9029A039B06000F002000A9
:1083C000290002F089F9009A019B04000D0048463B
:1083D000414602F081F902000B002000290002F062
:1083E000EDFB02000B003000390002F0E7FB020059
:1083F0000B0000204F4902F0E1FB70E002000B008F
:1084000002F06AF904000D003D4A3E4B02F064F9A7
:108410003D4A3E4B01F03AFA22002B0002F05CF993
:108420003B4A3C4B02F0CAFB22002B0002F054F9FD
:10843000394A3A4B01F02AFA22002B0002F04CF99B
:10844000374A384B02F0BAFB22002B0002F044F905
:10845000354A364B01F01AFA2B00220002F03CF9A3
:10846000354B029003919F429FDD344B00229F4287
:108470003DDC334900207B182E4916001F0002F016
:108480009DFB049005910022294B2000290002F059
:1084900023F932003B0002F091FB029A039B060095
:1084A0000F002000290002F017F9009A019B040038
:1084B0000D004846414602F00FF902000B00200073
:1084C000290002F07BFB02000B003000390002F0B3
:1084D00075FB02000B000498059902F06FFB07B0D2
:1084E0000CBC90469946F0BD00201249F7E7154BA9
:1084F000002604920593144FC5E7C046FFFF3F3E98
:10850000D43888BEE9FAA8BDC4B1B4BD9EEE213E00
:10851000AD529C804F7E923E9015CB19A001FA3E41
:108520007751C1166CC1563F4C5555555555A53F11
:108530000000E03F0000F03F3233D33F0000E93F4E
:108540000000E0FF0000E73F0000D23FF0B5DE464C
:108550004E4645465746E0B5DC4CA5440D91140007
:108560001900A49A0993DA4B9200D6584D1E039035
:108570001821E01E0696029500F0AAFEC3430100F2
:10858000DB1719404B1C9A009B1ADB001B190B913F
:1085900005934C1B771918D4A59BA5009C463F1941
:1085A00022AE6544013707E0286802F0A1FE0134DD
:1085B00003C60435BC4208D0002CF5DA00200021A7
:1085C000013403C60435BC42F6D1069B002B01DA08
:1085D00000F0FDFB069B03990133DB009A46099BE3
:1085E000DA00944600920022914672AA0492B94A97
:1085F0006144934688469AAB63449B44029B002B9C
:1086000000DABCE15D4600260027039C4D442A6841
:108610006B6803CC02F060F802000B0030003900F8
:1086200001F034F9083D06000F004445EFD1049BEA
:108630004B441E605F6008239C46E144D145DDD178
:108640000EA804218446494261448C46069A930050
:108650009C44614684460A910399083B63448C46D6
:108660000C93009B009263449B46009A0498D100AF
:1086700003008C46634408911E685F68002A33DD5E
:10868000954980468C466244D300984470AB9A4624
:108690000EAB99460022914B3000390002F01CF8D5
:1086A00002F0F0FD02F024FE00228D4B04000D00CC
:1086B00002F012F802000B003000390002F07EFADE
:1086C00002F0E0FD4B4601C39946434620001A687C
:1086D0005B68290001F0DAF808235B429C46E0441D
:1086E00006000F00D045D5D1059B30001A00390097
:1086F000984600F0DFFCFF2300229B0504000D00DC
:1087000001F0EAFF00F038FC0022764B01F0E4FFB4
:1087100002000B002000290002F050FA0D000400B6
:1087200002F0B0FD814602F0E3FD02000B002000E4
:10873000290002F043FA060040460F00002800DC42
:10874000EEE0009B18215A1E92000EAB9B58091AAE
:108750001D000D41A9448D405D1B0EAB9D5017239C
:108760001B1A1D41002D2DDD01239C46009BE14479
:10877000002B00DC1CE20E9C0123002C00D0B5E095
:10878000009A012A09D099000EAA54580133002CEE
:1087900000D0ACE0009A9A42F5D1059B002B0EDD8B
:1087A000012B00D1A8E1022B09D1009B0EA95A1E72
:1087B00092000EAB9B5807939B029B0A8B50022D95
:1087C00000D1C1E0002300223000390000F08AFE11
:1087D000009B002800D194E2069A591E8A4210DCC0
:1087E000414A0A9894460EAA6344944600229B008C
:1087F00063441C68043B22438342FAD1002A00D020
:10880000C0E0069B0EAA013B9B00D358002B00D072
:10881000B3E001220C9B043B596801320029FAD0D5
:10882000009B9C466244110007921A0001338B4260
:1088300046DC0B9863468046A59C4344A046099CB1
:108840009B00A1464A449844D30022AA9146049A28
:1088500099449446089BA59A63448446614494468F
:108860009A468B00634400934346586802F040FDEB
:108870004B4618605960029B002B24DB4D46039C3D
:108880000026002701E0286869680CCC01F024FF6D
:1088900002000B003000390000F0F8FF083D060030
:1088A0000F005C45EFD153469E60DF6004239C4679
:1088B0000433E0449C46009BE144E2449845D3D114
:1088C000079B0093D1E600260027ECE794FDFFFF0D
:1088D00088E1000018FEFFFFFFFFFF1F0000703E51
:1088E0000000704100002040FFFFFF3F0021802278
:1088F0005204141B0EAA5450009999420EDD0EA882
:1089000084469B000EAA8900D25861446344CF4834
:1089100000E01A68821A04C38B42FAD101243CE7B2
:10892000059B002B06D1009B0EAA013B9B00D5584E
:10893000ED1517E70022C64B300000F0F7FD0028C8
:1089400000D024E100253DE732003B000020C14972
:1089500002F034F906000F00002C00D132E7059A2E
:108960000020BC4900F0A6FB02000B0030003900DB
:1089700002F024F906000F0024E7012250E7002648
:10898000002754E64B46059A079388468B000EA9AC
:10899000CB58183A08950592002B0DD18C464146CC
:1089A000AD4B43449B006344043B58680139183A7B
:1089B0000028F9D088460592059A0020A54900F0C4
:1089C00079FB434604000D00002B00DA05E29E000F
:1089D0000EAB9C464346DB0066449C46059370AB59
:1089E0009946049F67440097306802F081FC22009A
:1089F0002B0001F071FE002238607960974B200057
:108A0000290001F069FE083F04000D00043EB9454D
:108A1000EAD14AAB03939B4600239A46069B424603
:108A2000994643460132029204934B46002B00DAEA
:108A3000AAE080208A4B009D9846C00589490026FF
:108A40000027002408E008239C460835E0445445EC
:108A500011DC4346186859682A686B6801F03CFECF
:108A600002000B003000390000F010FF0134060056
:108A70000F00A145E7DA5B46C0C39B4601239C4635
:108A8000009BE244083B0093029B9A45CDD1049B96
:108A90009846A49B022B00DD8EE0002B37DC1FD113
:108AA000059B00271D00039B00249C461E00654477
:108AB000083E2A686B683800210000F0E7FE083D98
:108AC00007000C00AE42F4D1089B002B03D080239A
:108AD0001B069C4664443A0023000D990A604B60D3
:108AE0000720079B18409B239B009D443CBC90465D
:108AF0009946A246AB46F0BD009B0EA95A1E9200B5
:108B00000EAB9B5807935B025B0A8B5057E64346BC
:108B1000002B00DA70E100200021DB004AAAD61801
:108B200048AF32687368083E00F0B0FEB742F8D133
:108B3000089B002B00D025E10B0002004A984B99BE
:108B40000D9C2260636002F039F8434607000C0078
:108B5000002B13DD01254CAEB14638002E0021005C
:108B60004C4601360CCC00F091FEA146B045F7DA38
:108B7000089B07000C00002B00D015E13A002300F1
:108B80000D998A60CB60ABE70026002773E70123CD
:108B90009C46009BE1440225002B00DDEBE5320002
:108BA0003B0000202B4902F009F806000F0009E6FF
:108BB0000024F2E54AAB0393A49B032B00D08FE77C
:108BC0004346002B00DC14E1039ADB009B461300B4
:108BD00091465B441E685F68234B43440293DB006D
:108BE000994448AB9A464B465C681B6818002100C4
:108BF00032003B000090019100F048FE04000D009F
:108C000002000B000098019901F0D8FF3B003200F0
:108C100000F03CFE4B469860D9601C605D60082304
:108C20005B429C46E14426002F00CA45DBD1434607
:108C3000012B00DCE3E0039A13005B441E685F68CD
:108C4000029BDB0099464A44904610E0FFFFFF007C
:108C50000000E03F0000F03FFFFFFF3F0000703EDC
:108C600048E10000FB21F93FFFFFFF1F9846434604
:108C70005C681B681800210032003B0000900191E5
:108C800000F004FE04000D0002000B0000980199A2
:108C900001F094FF32003B0000F0F8FD4346039AD8
:108CA0009860D9601C605D60083B26002F009A42E6
:108CB000DCD14D46944600260024474608356544DD
:108CC0002A686B683000210000F0E0FD083D0600D6
:108CD0000C00AF42F4D1039B4A9F5D689968D86845
:108CE000089B002B65D08022120694460D9B65449C
:108CF000604464441F605D609960D8601E615C617F
:108D0000EEE69A464B460793059B30005A423900DF
:108D1000089500F0CFF900223A4B06000F0000F052
:108D200005FC002824D0384B00223000390001F027
:108D3000D3FC02F0A7FA52460400950002F0D8FADC
:108D40000022304B01F0C8FC02000B00300039005B
:108D500001F034FF02F096FA0EAA50510122059B51
:108D6000524418339046059393000EAAD45023E63C
:108D70005346300039009C0002F084FA0EAB1851C3
:108D8000D04619E680230D9A1B06CB18106053605D
:108D90000B0002004A984B9901F010FF4346070070
:108DA0000C00002B00DDD5E680231B069C466444A6
:108DB000E4E62B003A000D9D2A606B600A00030078
:108DC000AA60EB60320023002A616B6188E6099B90
:108DD000DB00009372AB049332E4A49B022B00DD12
:108DE000E8E6002B00DD92E600D079E600270024BB
:108DF0006AE6002600246EE70020002198E600269F
:108E0000340068E7000070410000703EF0B5CE46C7
:108E1000474680B587B000920193474A4B00814690
:108E200088465B08934207DC4146484602F02AFA2E
:108E30004146031E484666D04A4643464846414698
:108E400001F04AFC04000D0002000B0048464146B8
:108E500001F042FC394A3A4B06000F00200029007D
:108E600001F03AFC374A384B01F0A8FE22002B00F3
:108E700001F032FC354A364B00F008FD22002B0091
:108E800001F02AFC334A344B01F098FE22002B00FB
:108E900001F022FC314B324A00F0F8FC0E9B0290AC
:108EA0000391002B34D00098019900222D4B01F042
:108EB00013FC029A039B049005913000390001F0E5
:108EC0000BFC02000B000498059901F077FE2200CC
:108ED0002B0001F001FC009A019B01F06FFE224A79
:108EE00004000D00214B3000390001F0F5FB0200B9
:108EF0000B002000290000F0C9FC02000B004846CE
:108F0000414601F05BFE07B00CBC90469946F0BDAF
:108F100002000B002000290001F0DEFB124A134B77
:108F200001F04CFE32003B0001F0D6FB4A464346BE
:108F300000F0ACFCE7E7C046FFFF3F3E7CD5CF5AD0
:108F40003AD9E53DEB9C2B8AE6E55A3E7DFEB157CA
:108F5000E31DC73ED561C119A0012A3F1111813F10
:108F6000A6F810110000E03F495555555555C53F2D
:108F700049004B0819007047474AF0B54F469146E3
:108F80004B005B0D99444646D6464A46C0B505009F
:108F90000C000E0088460700132A27DC002A4BDB52
:108FA0003E4B13419A460B0052461340034318D0E0
:108FB0003B4A3C4B2800210000F068FC00220023C3
:108FC00000F0AAFA002847D0002C04DA80234A4691
:108FD0005B03134198444646534600279E4338009E
:108FE00031001CBC90469946A246F0BD332A08DDEC
:108FF0008023DB009945F4D102000B0000F046FC11
:10900000EFE7294A9446012263445242DA409246ED
:109010000242E6D0224A234B2800210000F036FC11
:109020000022002300F078FA002815D0002C1EDB67
:10903000534646469F430FE0194A1A4B2800210029
:1090400000F024FC0022002300F066FA002803D080
:10905000002C04DB0027002638003100C1E7640043
:10906000640825430027002DF6D0104EF4E74B4648
:10907000142B0BD03422D21A012393405D19BD4228
:1090800008D201239C462F00E044D1E7133B9C46C5
:10909000E044CDE72F00CBE701FCFFFFFFFF0F000F
:1090A0009C7500883CE4377EEDFBFFFF0000F0BFBD
:1090B000002070474B0070B55B0D14000A00002BB8
:1090C0001AD14B005B08034315D0234B002201F05B
:1090D00003FB224B9C422DDB0A004B005B0D363B11
:1090E0001F4DE318AB422ADC002B0DDD1D4C1B0588
:1090F00022401A43110070BD1B4DAB42F0D102005B
:109100000B0000F0C3FBF6E71D00353519DA174BED
:1091100002009C4209DD0B001548164900F032F8A8
:10912000134A144B01F0D8FAE5E70B001248134933
:1091300000F028F8104A114B01F0CEFADBE70200EC
:10914000E9E7084C363322401B051343190000227F
:109150000B4B01F0C1FACEE700005043B03CFFFFDB
:10916000FE070000FFFF0F80FF07000050C3000054
:109170009C7500883CE4377E59F3F8C21F6EA50148
:109180000000903C30B54A00DB0FDB0752081A4361
:10919000110030BD02B4714649084900095C49001C
:1091A0008E4402BC7047C04603B471464908400073
:1091B0004900095A49008E4403BC70470022430805
:1091C0008B4274D303098B425FD3030A8B4244D38F
:1091D000030B8B4228D3030C8B420DD3FF220902D1
:1091E00012BA030C8B4202D31212090265D0030B90
:1091F0008B4219D300E0090AC30B8B4201D3CB0386
:10920000C01A5241830B8B4201D38B03C01A5241C7
:10921000430B8B4201D34B03C01A5241030B8B42C9
:1092200001D30B03C01A5241C30A8B4201D3CB02B4
:10923000C01A5241830A8B4201D38B02C01A524199
:10924000430A8B4201D34B02C01A5241030A8B429C
:1092500001D30B02C01A5241CDD2C3098B4201D3B4
:10926000CB01C01A524183098B4201D38B01C01A32
:10927000524143098B4201D34B01C01A52410309A9
:109280008B4201D30B01C01A5241C3088B4201D358
:10929000CB00C01A524183088B4201D38B00C01A05
:1092A000524143088B4201D34B00C01A5241411A2C
:1092B00000D20146524110467047FFE701B5002039
:1092C00000F0F0F802BDC0460029F7D076E77047FD
:1092D00003460B437FD4002243088B4274D3030917
:1092E0008B425FD3030A8B4244D3030B8B4228D3B8
:1092F000030C8B420DD3FF22090212BA030C8B42DE
:1093000002D31212090265D0030B8B4219D300E07D
:10931000090AC30B8B4201D3CB03C01A5241830B02
:109320008B4201D38B03C01A5241430B8B4201D3B2
:109330004B03C01A5241030B8B4201D30B03C01ADB
:109340005241C30A8B4201D3CB02C01A5241830A55
:109350008B4201D38B02C01A5241430A8B4201D384
:109360004B02C01A5241030A8B4201D30B02C01AAE
:109370005241CDD2C3098B4201D3CB01C01A524115
:1093800083098B4201D38B01C01A524143098B429E
:1093900001D34B01C01A524103098B4201D30B0187
:1093A000C01A5241C3088B4201D3CB00C01A5241AC
:1093B00083088B4201D38B00C01A524143088B4271
:1093C00001D34B00C01A5241411A00D2014652410A
:1093D000104670475DE0CA0F00D04942031000D329
:1093E0004042534000229C4603098B422DD3030A7E
:1093F0008B4212D3FC22890112BA030A8B420CD38E
:10940000890192118B4208D3890192118B4204D3B6
:1094100089013AD0921100E08909C3098B4201D336
:10942000CB01C01A524183098B4201D38B01C01A70
:10943000524143098B4201D34B01C01A52410309E7
:109440008B4201D30B01C01A5241C3088B4201D396
:10945000CB00C01A524183088B4201D38B00C01A43
:109460005241D9D243088B4201D34B00C01A52411A
:10947000411A00D20146634652415B10104601D3A7
:109480004042002B00D54942704763465B1000D331
:10949000404201B5002000F005F802BD0029F8D0D7
:1094A00016E770477047C046D0400B1C1141203A68
:1094B00003D49C46134118436346524293401843D9
:1094C0007047C0468446101C62468C46191C634691
:1094D00000E0C0461FB501F097F8002801D4002134
:1094E000C8421FBD10B500F0EFFF4042013010BD73
:1094F00010B501F089F8002801DB002010BD012023
:1095000010BDC04610B501F07FF8002801DD002035
:1095100010BD012010BDC04610B501F011F80028A3
:1095200001DC002010BD012010BDC04610B501F0C7
:1095300007F8002801DA002010BD012010BDC04648
:10954000F0B5CE46474615042D0C2E0080B5070415
:10955000140C3F0C9946030C7E435D436743634301
:109560007F19340CE4199C46A54203D980235B0281
:109570009846C4444B4643435143250C3604654446
:10958000360C2404A4195B19591820000CBC904611
:109590009946F0BDF0B54E4657464546DE46E0B525
:1095A00043025B0A450083B00F1C99462D0EC60F7F
:1095B000002D57D0FF2D24D08020DB00C00418439D
:1095C000002381469A469B467F3D7C027A00FB0F32
:1095D000640A120E984623D0FF2A4BD0E300802461
:1095E0000020E4047F3A1C43AD186B1C47460193EE
:1095F000534677403A000F2B48D87D499B00CB5803
:109600009F46002B00D085E008339A46063B9B46D8
:109610007C027A00FB0FFF25640A120E9846DBD10C
:10962000002C00D090E0524601231A4392460120BC
:10963000DBE74C4658461700022824D0032800D107
:10964000CFE00022002301284DD15802D205400A64
:10965000FF071043384303B03CBC90469946A246EE
:10966000AB46F0BD002B5BD104239A46033B00259B
:109670009B46AAE7FF35002C60D1524602231A43CD
:1096800092460220B1E7FF220023DEE74B461B0C87
:109690009C464B462604360C180461463300220CC7
:1096A0006446000C43434E435043544380191A0C04
:1096B0001218964203D9802149028C4664441B0447
:1096C0001B0C1004C01883015E1EB341800E1843AA
:1096D000130C1B199B0103431C00230179D50123A3
:1096E00062081C401443019A7F32002A4DDD630753
:1096F00004D00F232340042B00D00434230103D5CE
:109700003C4B019A1C408032FE2ABCDCA3015B0A60
:10971000D2B29AE70C239A46093BFF259B4654E7B1
:10972000180001F071FE4A46431F76259A40002337
:109730006D4291462D1A9A469B4646E752460323B0
:109740001A439246032050E7200001F05DFE431FBC
:109750002D1A9C40763D002047E780230027DB033D
:10976000FF2272E7424666E74C463200584662E7FF
:1097700080234A46DB031A4222D01C4220D12343D5
:109780005B025B0A4746FF225FE701239A1A1B2A06
:1097900021DC23000199D3409E318C401A00230024
:1097A0005C1EA34113435A0704D00F221A40042A17
:1097B00000D004335A0111D49B015B0A002244E714
:1097C00080234A46DB0313435B025B0A3700FF2218
:1097D0003BE7019587E70022002336E701220023BB
:1097E00033E78023DB0323435B025B0AFF222CE782
:1097F00098E10000FFFFFFF770B500283DD0C317C8
:10980000C5185D40C40F280001F0FEFD9E22121A0B
:10981000962A07DCD2B2082833DD08388540680272
:10982000400A23E0992A0BDD052329001B1AD940A1
:1098300003001B339D402B005D1EAB4119430D00FF
:10984000052801DD431F9D402B000F490B406E078B
:1098500009D00F263540042D05D004335D0102D513
:109860009F220B40121A9B01580AD2B24002D20525
:10987000400AE4071043204370BD0024002200206A
:10988000F4E76802400AF1E7FFFFFFFBF0B54F463F
:109890004646D6460C000903C0B5490A470F5E008C
:1098A00039431F03DB0F9C4665007B0A570F1F439C
:1098B0006D0DE40F760DA146C000B846D200AB1B7B
:1098C00064457BD0002B5FDD002E00D0A4E03E007D
:1098D000164300D112E15E1E002E00D09EE1871AD1
:1098E0004346B84280410125C91A4042091A0B0279
:1098F00000D431E149024E0A002E00D16EE1300061
:1099000001F082FD0300083B1F2B00DD61E12022F6
:109910003900D21A9E40D1409F400E439D4200DD47
:1099200051E15D1B6B1C1F2B00DD7CE12021C91A5E
:109930003D0030008F408840DD40791E8F4131006E
:1099400007222843D940002507433A40002A09D07E
:109950000F233B40042B05D03B1DBB42BF417F4240
:10996000C9191F000B0200D426E26A1CC64B55051C
:109970006D0D9A4200D106E1C44AFF080A40530720
:1099800052023B43120B8EE0002B00D0B8E06B1C60
:109990005B055B0D012B00DC30E1871A4346B842C2
:1099A000B641CB1A76429E1B330200D54CE13B00F8
:1099B0003343A1D100220024002570E0002B00DCFD
:1099C000E5E0002E00D183E0AF4EB54260D08026A6
:1099D00036043743B846382B00DC3EE14346134398
:1099E0001F007A1E97413F18874280414042091864
:1099F0000B0200D4B0E0A44B01359D4200D1C3E07E
:109A0000A24A7B080A4001210F401F435108D30797
:109A100007221F433A4099E79B4EB54238D0802633
:109A200036043743B846382B00DDDCE01F2B00DC62
:109A300030E11E004746203EF740BC46202B04D0B4
:109A40004026F31A46469E403243170063467A1E6C
:109A500097411F43CCE0002B00D104E2434613435F
:109A600000D159E14B07C00818438023C9081B03E4
:109A7000194208D04546ED081D4204D14346D0089E
:109A8000590708432900420FC9007F4D1143C00008
:109A90004B07CA087C49C00803438D4268D01203B3
:109AA0006D05120B6D0D002112031800130B0A0D2A
:109AB00012051A43764B2D0513402B435B00E40738
:109AC0005B08234319001CBC90469946A246F0BD92
:109AD0003E00164312D05E1E002E00D000E1871813
:109AE0008742804141444042091801250B0233D589
:109AF000022585E764463300414610001D00C7E794
:109B0000002D00D0DAE00C000443F3D05C1C00D13F
:109B10009FE15D4CA64200D12FE1DB43382B00DDF5
:109B200066E11F2B00DD83E120240500E41A0F000D
:109B3000DD40D940A0404346A7405B1A441EA041E7
:109B400098462F433843171ABA429241434652422D
:109B5000991A64463500CAE607223A40002A00D026
:109B6000F6E64B07CA084849FF083B438D4296D1A9
:109B70001900114300D19EE1802109030A43120319
:109B8000120B414D8FE71500002200238BE7002BBD
:109B900000D0C7E06B1C5F057F0D012F00DCF1E0FA
:109BA000394DAB4200D1B9E085180A0085428941A0
:109BB0004244494251180722CF076D082F434908F4
:109BC0003A401D00C2E607223049ED1A31403A40C2
:109BD000BCE63E002838864000279FE6380001F0AA
:109BE00013FC20308EE6434613431F007A1E974134
:109BF000C71BB84280414042091A78E60E003B007C
:109C000006431343002D61D1002E00D0F4E0002B59
:109C100000D11BE164463900100039E71A4FBB42FE
:109C20007AD03300FFE630001F3DE840202B03D000
:109C30004021CB1A9E4037437B1E9F41072207439A
:109C40003A400021002589E7171A4346BA42B64137
:109C5000591A76428E1B64464EE61F2B00DDADE09E
:109C600020264746F61AB740B9461700B246DF40ED
:109C70004E463E4337005646B240561EB241174349
:109C80004246DA408918AEE6FF070000FFFF7FFF7B
:109C9000FFFF0F8020264746F61AB740B946170047
:109CA000B246DF404E463E4337005646B240561E4F
:109CB000B24117434246DA40891A99E77F4CA642DF
:109CC0005BD0802424045B42214327E7002E0CD183
:109CD000002B00D1CBE0644639001000774DD7E669
:109CE000764FBB4218D0330075E6002B14D04B07DB
:109CF000C00818438023C9081B03194207D0FC0879
:109D00001C4204D17907D0080843E14621004C46A3
:109D1000420FC9001143C000684DB9E61D00002282
:109D20000023C0E6002D5BD10D00054300D1E2E623
:109D30005D1C00D1B0E0614DAE421FD0DB43382B3B
:109D400071DC1F2B00DD96E020250F00ED1AAF40DF
:109D5000B9460700AA46DF404D463D432F00554611
:109D6000A840D940451EA84188440743BF189742E0
:109D700092415142414435003AE66446350041463D
:109D8000100085E60B000343002D00D063E6002B96
:109D9000F5D04346134300D17AE6871887428041C5
:109DA00007224144404209183A400B0200D4D5E64C
:109DB000434B01351940C9E5380069E61E004746A6
:109DC000203EF740BC46202B04D04026F31A4646DE
:109DD0009E403243170063467A1E97411F4302E6B6
:109DE000364DAE42CAD080252D045B422943A6E7FA
:109DF0000843411E8841A6E6002B00D148E6871A99
:109E00004346B842B641CB1A76429E1B33024BD52D
:109E1000171A4346BA429241591A5242891A0722E6
:109E200064463A4092E501430F00791E8F419DE759
:109E30001C000F00203CE740202B03D04024E31AF5
:109E400099400843411E884138437CE600220024A3
:109E500025E6171A4346BA429241591A5242891AC4
:109E60006446350043E541461000144D10E680225B
:109E70000024120380E61D000F00203DEF40BC4689
:109E8000202B03D04025EB1A994008430700634676
:109E9000781E87411F4369E7871897429B414144D9
:109EA0005B42C9183500A3E53B003343CED00722FF
:109EB00031003A4052E600231A00F4E5FF070000A3
:109EC000FFFF7FFFF0B55746DE464E464546E0B5FC
:109ED000834607000E03480085B092461C00360BEF
:109EE000400DCD0F002800D19DE0954B984239D010
:109EF0008023F6001B041E43924A7B0F334399468E
:109F0000944603006344009300230026FF0002935D
:109F100023031B0B98466300E40F52465B0D01942C
:109F200000D1B3E086498B4200D19EE04246D10089
:109F3000802212040A435146490F11438B4681493E
:109F400052468C4600996344CB1A0021D2000093FC
:109F50002B0063409A460F2E00D905E17A4BB600DC
:109F60009B599F465B463343994600D0B8E0022395
:109F70000826002700900293CAE7CB463A000299D0
:109F80000195019B9A46022927D0032900D180E23E
:109F9000012944D06D49009B8C4663441C00002C71
:109FA00038DD530700D013E2D2085B46DB0109D548
:109FB0005946674B19408B468021C9008C46009B4F
:109FC00063441C00634B9C4207DC5B4664055F07EF
:109FD0005B0217431B0B620D02E000230027584A67
:109FE00000211B031C0B0B0D1B05234314055A4AB0
:109FF000380013401C4353466400DB0764081C43CD
:10A00000210005B03CBC90469946A246AB46F0BD47
:10A010000122524201231B1B382B00DCADE1002240
:10A0200000230027DCE75B46334399465ED0002ED1
:10A0300000D18AE1300001F0E7F903000B3B1C2B53
:10A0400000DD7BE11D22D31A5A460100DA400839AF
:10A050008E4013005F46334399468F403F4B0026A6
:10A060001B1A00930023029352E7414653460B43C9
:10A070003B499B468C46009B634400935B46002B08
:10A080003BD1022300221E43022161E743461343D2
:10A090009B4637D04346002B00D162E1404601F099
:10A0A000B3F903000B3B1C2B00DD53E102004146DA
:10A0B000083A914088461D21CB1A5146D9400B00E1
:10A0C00041460B439B46534693401A00009B25494B
:10A0D0009C46604403008C4663440093002137E7AC
:10A0E0000323B14600900C26029311E7002300934E
:10A0F00001330426002702930AE70323C3461E43C5
:10A10000032125E701331E430022012120E700231C
:10A110009A46802300271B03094A61E780234946AA
:10A120001B03194200D1E2E05946194200D0DEE09B
:10A130000B431B0317001B0BA246014A50E7C04606
:10A14000FF07000001FCFFFFD8E10000FF03000053
:10A15000FFFFFFFEFE070000FFFF0F800DFCFFFF6B
:10A1600001F8FFFFF3030000D94500D9CBE000D18F
:10A17000C6E03C0048460027009B013B00935B463D
:10A18000160E1B021E431302984633041B0C9946FD
:10A19000310C0191FFF798F84A4642430B04210C19
:10A1A000050019438A4207D98919013D8E4203D817
:10A1B0008A4201D9851E8919881A0199FFF784F806
:10A1C00009048C464A46210464464243090C0300B4
:10A1D00021438A4204D98919013B8E4200D8F1E01B
:10A1E0002D041D43AB464346891A4246280C1204EF
:10A1F0001D0C5B46140C22001B041B0C5A430394D9
:10A200006B434443029568431B19150CEB189C42A1
:10A2100003D980246402A44660441C0C15041B046A
:10A220002D0C20185D19814277D373D00C1AA24AE5
:10A230007D1BAF42BF419446009B7F426344E01BBD
:10A240001C00864200D1DBE00199FFF73DF84A4649
:10A2500042430B04290C070019438A4207D9891984
:10A26000013F8E4203D88A4201D9871E8919881A74
:10A270000199FFF729F809044A46894629044D4601
:10A280004243090C030029438A4207D98919013B3B
:10A290008E4203D88A4201D9831E89193F04891A44
:10A2A0003A00039F1A43380013041B0C584381469D
:10A2B0000298150C6F43434345434846000C8446BF
:10A2C000DB1963449F4203D98020400284466544E1
:10A2D00048461F0C00041B04000C7D191818A942E5
:10A2E00000D284E000D17FE001231A4357E68023A7
:10A2F0004A461B0313431B031B0BAA466F4A6FE618
:10A30000BA4200D935E74B46DC0758087B081C43A6
:10A31000FF0734E70024AF4289D247444745A441B0
:10A320005B466442A4196418013BA6421ED2A042B7
:10A330006DD800D1B6E0241A9B4678E703005A4650
:10A34000283B9A400027914688E6584601F05CF881
:10A35000203072E603005246283B9A409346002282
:10A36000B4E6504601F050F820309AE6A642E2D119
:10A37000B845DCD9341A9B4659E71F2B65DC504C95
:10A380000099A4465C46614408008C40110082405C
:10A39000D940501E82410C4314435A46DA40130000
:10A3A000620709D00F222240042A05D02200141D82
:10A3B0009442894149425B181A0262D50122002366
:10A3C00000270DE68A4200D80AE7831E891907E7AD
:10A3D0000F231340042B00D1E6E5171D974292414D
:10A3E00053429B44FA08E0E5002800D1D7E57118F4
:10A3F000531EB14227D3A94215D358D01A0073E790
:10A40000002B00DC04E6012300229B44CDE502235F
:10A410004744474589415B429C46494289190C198A
:10A42000E344241A03E743465F0047459B41B8468F
:10A430005B429E19023A8919A94200D054E740456F
:10A4400000D051E7ABE51A00F6E71F215F4649420D
:10A450000C1BE740202B07D01A49009B8C46634415
:10A4600018005B4683401A43501E82413A43072737
:10A470000023174009D00F210023114014000429A4
:10A4800095D122005F075B021B0BD2081743002205
:10A49000A6E5802359461B030B431B0317001B0B28
:10A4A000064A9DE5BD42B2D89B460024BFE68045E2
:10A4B000B9D31A00C3E7C046FF030000FF0700003E
:10A4C0001E0400003E040000F0B54F464646D64646
:10A4D0008446C0B58046194E18030F034D00000B8B
:10A4E0005C0082463F0B6D0DC90F9146640DDB0F7A
:10A4F0000120B5420AD0B44203D0A54201D157454C
:10A500000CD01CBC90469946A246F0BD66463E4320
:10A51000F7D1AC42F5D154461443F2D10120C845DD
:10A52000EFD1994207D0002DEBD163461F4338008D
:10A53000471EB841E5E70020E3E7C046FF070000FB
:10A54000F0B54F464646D6464D00C0B50E03C90F7E
:10A550008A462C491F035C008046360B6D0D9146E0
:10A560003F0B640DDB0F8D421ED08C4216D0002DA8
:10A570001ED130438446002C01D13A4323D0624699
:10A58000002A1AD09A4529D05146022001390840A4
:10A5900001381CBC90469946A246F0BD39001143D3
:10A5A000E5D002204042F4E73043FAD1AC420FD06C
:10A5B000002C0FD13A43E7D00CE00122013B93433A
:10A5C00018000130E5E763460020002BE1D0DBE70F
:10A5D0003A43E6D19A45D7D1A542D5DCA54205DB61
:10A5E000BE42D1D808D00020BE42D2D2504601236C
:10A5F000013898430130CCE7C845C5D80020C8458C
:10A60000F4D3C6E7FF070000F0B54F464646D646EE
:10A610004D00C0B50E03C90F8A462E491F035C00CA
:10A620008046360B6D0D91463F0B640DDB0F8D425E
:10A6300018D08C4211D0002D18D130438446002C04
:10A640001ED13A431CD163460020002B30D0514626
:10A6500002200139084001382AE039001143EAD0CC
:10A66000022025E03043FBD1AC4226D0002C26D17D
:10A670003A4324D15146022001390840013817E0FD
:10A680006246002A0FD09A45E1D1A54205DBBE42C1
:10A69000DDD819D00020BE420AD25046012301382D
:10A6A0009843013004E00122013B9343180001303C
:10A6B0001CBC90469946A246F0BD3A43D0D19A457B
:10A6C000C5D1A542C3DCE0E7C845C0D80020C845D5
:10A6D000E3D3EDE7FF070000F0B55746DE464E46F0
:10A6E0004546E0B5834606000F03480087B0924612
:10A6F0001D003F0B400DCC0F002800D16FE0DE4B5A
:10A70000984238D08023FF001B041F43730F3B4344
:10A710000193DA4B0027994600239B46F6008144BB
:10A720002B0369001B0B52469846490DED0F00297B
:10A7300000D185E0D04B994200D173E04346DA0066
:10A7400080231B0413435246CC48520F84461343C4
:10A75000524600206144D2008944210069400091A2
:10A760008C46012149448A460F2F00D990E0C44904
:10A77000BF00CF59BF465B463B43019300D06AE11F
:10A7800002230827002681469B46C9E73200584627
:10A79000019B61460091022800D175E0032800D199
:10A7A000FEE1012800D02CE100230027002600252F
:10A7B0003F032A0D3F0BB34812053A4302401B05E5
:10A7C0001343009A5B00D1075B080B43300019006C
:10A7D00007B03CBC90469946A246AB46F0BD5B46EE
:10A7E0003B43019300D12FE1002F00D1A5E13800B8
:10A7F00000F00AFE03000B3B1C2B00DD96E11D223E
:10A80000D31A5A460100DA405E4608398F401300D9
:10A810008E403B4301939C4B00271B1A9946002313
:10A820009B467DE7414653460B4393498C46E144A2
:10A83000002B00D01AE102220220174300228CE7ED
:10A84000134300D10DE14346002B00D181E1404686
:10A8500000F0DAFD02000B3A1C2A00DD72E1010073
:10A86000434608398B4098461D239A1A5346D340D5
:10A870001A004346134352468A404946081A824901
:10A8800089468144002068E77B4B002700268EE73D
:10A89000140C1204120C1100370C3604350C7943D9
:10A8A00028008C462E0060436044834656432100B6
:10A8B000300C80465846794340440291844506D97D
:10A8C0008846802149028C46E04441460291360484
:10A8D000010C360C00048B4681191E0C1B041B0C4A
:10A8E0000391190079438C46280075436544A846B6
:10A8F0005843050C45447743A94203D980214902B6
:10A900008C466744290C8C4639000004000C2D0449
:10A910002D186144AB4405915946049101990F04E7
:10A920003F0C080C390051434243904602008C46CC
:10A93000090C8B4662437C4344445C44A04503D9E4
:10A940008021490288464244210C88466146090418
:10A95000090C8C4639005943434370437E430F0C26
:10A96000F6182404BE19644442448C46B34203D909
:10A9700080235B0298464044029B61469846049BB4
:10A98000370443449B46AB45AD416B420D040599EA
:10A990002D0C8C467F196744FD18A8465D462D197D
:10A9A000A542A44193466442A446C344DC448F427A
:10A9B000BF4198459B4193459241A445A4415B42C8
:10A9C0007F421F43360C52426442BF192243BF18D4
:10A9D000624638184302D20D039913436A020A43B0
:10A9E000501E82416146ED0D2A434E023243D90189
:10A9F00000D4B3E00126500832400243DE07324360
:10AA00005B08224C5444002C62DD510709D00F2012
:10AA10001040042805D0101D9042924152429B18CC
:10AA20000200D90104D580241948E40003405444AD
:10AA30001848844200DD27E75E075B02D2081F0B3F
:10AA4000630516435B0DB2E60023994601330427E4
:10AA500000269B4664E60323019781460C279B460C
:10AA60005EE6012201201743002276E6032303203D
:10AA70001F43434671E6C046FF07000001FCFFFF8D
:10AA800018E20000FFFF0F800DFCFFFFFF03000036
:10AA9000FFFFFFFEFE0700000023802700933F0317
:10AAA0000026434B83E6019B3200A446584670E6DD
:10AAB000AC466EE6802701993F0339422DD03B42D8
:10AAC0002BD11F433F033F0B00951600384B6EE61A
:10AAD00001252D1B382D00DD66E61F2D40DC354895
:10AAE0001C005044160082408440EE40501E8241BB
:10AAF00034431443EB40620709D00F222240042A5A
:10AB000005D02200141D9442804140421B181A02B5
:10AB10003ED501230027002649E68027019B3F03FD
:10AB20001F433F033F0B0094214B40E603005A466E
:10AB3000283B9A40002601926DE6584600F064FCDE
:10AB4000203057E603005246283B9A40130000226B
:10AB500093E6504600F058FC20307BE6CA4650E7AA
:10AB60001F201E004042041BE640202D03D0124C43
:10AB70005444A3401A43501E824132430726002703
:10AB8000164009D00F200023104014000428B9D12A
:10AB900022005E075B021F0BD2081643002306E665
:10ABA00080273F031F433F033F0B1600004BFEE58A
:10ABB000FF0700001E0400003E040000F8B55746E1
:10ABC0004E464546DE460C000903E0B5490A460FED
:10ABD0005F0031431E03DB0F760A9B46530F33435E
:10ABE000C84E6500C000E40FD2006D0DA24681463C
:10ABF0007F0D9C469046B74200D1B9E05B460126E6
:10AC000073409B46EE1BA34500D183E0002E63DD1D
:10AC1000002F00D0B1E06346134300D123E1731E3F
:10AC2000002B00D0BAE1861A6346B042804101256C
:10AC3000C91A4042091A0B0200D447E149024B0AE3
:10AC400098464346002B00D189E1404600F0DCFBEA
:10AC50000300083B1F2B00DD7CE120223000D21ACC
:10AC60004146D040994002009E400A439D4200DD8B
:10AC70006AE15D1B6B1C1F2B00DD94E1202110009D
:10AC80003500C91A8E40DA408840DD40711E8E4181
:10AC9000110007222843002506433240002A09D02C
:10ACA0000F233340042B05D0331DB342B641764207
:10ACB00089191E000B0200D43DE26A1C914B550518
:10ACC0006D0D9A4200D119E18F4AF6080A405707E4
:10ACD00052023743120B9BE0002E00D0C5E06E1CE1
:10ACE0007605760D012E00DC48E16746861ACB1BFF
:10ACF000B042BF417F42B8461F004346FF1A3B00A7
:10AD0000B8461B0200D55FE137439AD100220024E8
:10AD1000002579E0002E00DCFAE0002F00D18DE064
:10AD2000784B9D4267D0802367461B041F43BC4677
:10AD3000382E00DC52E1634613435A1E93411E181D
:10AD400086428041404209180B0200D4BEE06D4BA0
:10AD500001359D4200D1D2E06B4A73080A400121BF
:10AD60000E401E435108D30707221E43324095E789
:10AD70001E00164300D045E740E7624B9D423AD0A3
:10AD8000802367461B041F43BC46382E00DDEBE0E2
:10AD90001F2E00DC3AE133006746203BDF403B00DA
:10ADA000202E05D04027BF1B6646BE40324390464A
:10ADB0004646721E96413343DAE0002B00D114E27E
:10ADC0006346134300D168E180234E07C008C908D9
:10ADD0001B030643194208D06046C008184204D13C
:10ADE00063460100D2085E071643F3009946C90086
:10ADF000720F444D11434B46DE08424B4F07374319
:10AE0000CA089D4200D16EE012036D05120B6D0D54
:10AE100000211203130B0A0D12051A433B4B2D059B
:10AE200013402B435B00E4075B0823433800190001
:10AE30003CBC90469946A246AB46F8BD63461343D8
:10AE400011D0731E002B00D007E186188642804186
:10AE500061444042091801250B0237D502257BE7E2
:10AE60003E00614691463500C5E75C46002D00D0A6
:10AE7000E1E00B000343F3D0731C00D1ACE1214BA4
:10AE80009F4200D13AE1F343382B00DD6FE11F2BE5
:10AE900000DD8CE120250E00ED1AAE40B046060024
:10AEA000AA46DE40454635432E005546D940A840C7
:10AEB0006346451EA8415B1A9C463043161AB242AF
:10AEC000924163465242991A3D00B4E6072232404D
:10AED000002A00D0E4E60B4BF6084F073743CA08B8
:10AEE0009D4200D090E73B00134300D1A6E18023B0
:10AEF0001B031A431203120B024D89E715000022AF
:10AF0000002785E7FF070000FFFF7FFFFFFF0F809F
:10AF1000002E00D0C7E06B1C5E05760D012E00DC14
:10AF2000F0E0C84DAB4200D1B9E085180A00854277
:10AF300089416244494251180722CE076D082E43C9
:10AF4000490832401D00A9E6BF49ED1A1140072209
:10AF50003240A3E6320028388240002686E63000E0
:10AF600000F052FA203073E6634613435A1E9341B1
:10AF7000C61AB04280414042091A5CE60E0067469C
:10AF800006431743002D5ED1002E00D0F3E0002FC2
:10AF900000D11EE15C46614691462CE7A94FBE42B6
:10AFA0007BD01E00F1E610001F3DE840202B03D0AF
:10AFB0004021CB1A9A401643731E9E410722064336
:10AFC00032400021002583E7161A6346B2428041D1
:10AFD000591A40420B1A98465C4632E61F2E00DD95
:10AFE000ABE02027BB1B9A4663465746BB409946B9
:10AFF00013004F46F3401F433B005746BA40571ECD
:10B00000BA4113436246F240891898E62027BB1BD9
:10B010009A4663465746BB40994613004F46F34055
:10B020001F433B005746BA40571EBA41134362467E
:10B03000F240891A9CE7834B9F425FD080252D0404
:10B040007342294320E7002E0CD1002F00D1D0E01D
:10B050005C46614691467B4DCDE67A4FBE421CD0A0
:10B060001E0065E6002F18D0C0084E07064380205A
:10B07000C9080003014208D06346DC08044204D139
:10B080002100DA46D2085E071643F30099460124F0
:10B090005346C900720F11431C406A4DABE61D00B8
:10B0A00000220027B4E6002D59D10B00034300D144
:10B0B000D6E6731C00D1B2E0624B9F421ED0F34330
:10B0C000382B6FDC1F2B00DD97E020250E00ED1ADA
:10B0D000AE40B0460600AA46DE40454635432E0047
:10B0E0005546A840D940451EA8418C440643B61891
:10B0F00096429241514261443D0025E63D00614641
:10B10000914678E60B000343002D00D055E6002B56
:10B11000F5D06346134300D16DE686188642804120
:10B1200061444042091800220B0200D4D0E6464B8D
:10B1300001351940B2E5B1465DE633006746203B74
:10B14000DF403B00202E05D04027BF1B6646BE4097
:10B15000324390464646721E96413343EFE5394BE3
:10B160009F42CBD080252D0473422943A8E7084392
:10B17000411E8841A2E6002F00D13CE66346861AB4
:10B18000CF1AB0429B415B42FB1A98461B024ED538
:10B19000161A6346B2429241591A5242891A5C46C3
:10B1A00000227BE501430E00711E8E419FE71D00CA
:10B1B0000E00203DEE40B046202B04D04025EB1A77
:10B1C00099400843814648464346411E88411843FA
:10B1D00074E60022002417E6161A6346B242924132
:10B1E000591A5242891A3D0025E561469146154D8E
:10B1F00001E680220024120379E61D000E00203DA6
:10B20000EE40B046202B04D04025EB1A994008436D
:10B2100081464E464346711E8E411E4367E786189F
:10B2200096429B4161445B42C9183D008CE547460C
:10B230003743CED007224146324049E600273A0044
:10B24000E6E5C046FF070000FFFF7FFF70B50C4E2C
:10B250000D031C0349005B002D0B490D240B5B0DF6
:10B26000B14208D0064900208B4203D1144320008C
:10B27000441EA04170BD05430120002DFAD1F1E725
:10B28000FF07000030B5144D0A034B00120B5B0D95
:10B29000C90F0024AB4211DD104CA34210DC802406
:10B2A000640322430E4CE41A1F2C0CDD0D48C31A14
:10B2B000DA4013005C42002900D11C00200030BDA0
:10B2C000094BCC18FAE7094DE040AC4663449A407C
:10B2D00013000343EEE7C046FE0300001D04000018
:10B2E0003304000013040000FFFFFF7FEDFBFFFFAE
:10B2F00070B500282DD0C317C5185D40C40F2800B5
:10B3000000F082F8154B1B1A5B055B0D0A2815DD52
:10B310000B38854000222D032D0B002110002D033A
:10B320000A0D2D0B12052A430D4D1B052A40134310
:10B330005B00E4075B082343190070BD020029008D
:10B34000153291400A000B21081AC5402D032D0B20
:10B35000E3E70024002300250022DEE71E040000AE
:10B36000FFFF0F804100090E4B1C70B5DBB2460297
:10B37000750AC40F012B14DDE0239B006D07360B0B
:10B38000CB1800210A0D280012051C4D32435B0525
:10B390002A405B0813435B00E4075B082343190062
:10B3A00070BD002914D1002D1ED0280000F02CF80B
:10B3B0000A281CDC0B232A001B1ADA400300153371
:10B3C0009D400F4B12031B1A5B05160B5B0DD8E754
:10B3D000002D06D0320B802636036D071643094B2D
:10B3E000CFE7084B0026CCE700230026C9E703007F
:10B3F0002A000B3B9A400025E3E7C046FFFF0F8081
:10B4000089030000FF0700001C2101231B04984250
:10B4100001D3000C10391B0A984201D3000A0839E5
:10B420001B09984201D30009043902A2105C40189C
:10B430007047C04604030202010101010000000040
:10B440000000000030B51C00094B05001B6885B0EA
:10B45000D868084B002A01D1074B1A0002920193C9
:10B4600000912B002200054900F026F800F0A6FD0F
:10B470008000002058E200008CD0000065E200004F
:10B48000014B18687047C04680000020084B10B57B
:10B490000400002B02D0002100E000BF054B18681B
:10B4A000836A002B00D09847200001F05DFBC04666
:10B4B0000000000094E200000EB403B5010003ABED
:10B4C000044804CB0068019300F076F802B008BC91
:10B4D00003B018478000002070B500260C4D0D4CBD
:10B4E000641BA410A64209D1002601F03FFB0A4DBF
:10B4F0000A4C641BA410A64205D170BDB300EB58E2
:10B5000098470136EEE7B300EB5898470136F2E76B
:10B510005002002050020020500200206002002053
:10B52000002310B59A4200D110BDCC5CC454013345
:10B53000F8E710B5884202D98B18984203D300234C
:10B5400007E08B5C8354013AFBD210BDCC5CC45441
:10B5500001339A42FAD1F8E703001218934200D15E
:10B56000704719700133F9E7936810B5013B936098
:10B57000002B04DA9469A34207DB0A2905D013687B
:10B58000581C10601970080010BD00F04BFC010041
:10B59000F9E7F8B506000F001400D518AC4201D148
:10B5A000002007E021783A003000FFF7DDFF01348A
:10B5B000431CF3D1F8BD0000F0B59FB002900F001E
:10B5C00016000593002805D083690493002B01D150
:10B5D00000F0F4FD7B4B9F425BD1029B5F68BB890F
:10B5E0001B0762D53B69002B5FD0002306AC63616B
:10B5F000203363761033A37635002B78002B01D0EF
:10B60000252B5CD1AB1B04930CD03200390002987F
:10B61000FFF7BFFF431C00D1C4E06269049B94465E
:10B62000634463612B78002B00D1BBE0012200232F
:10B630005242626002A9543252186E1C2360E360C9
:10B64000A3601370A365317805225F4800F0D4FE33
:10B65000751C002835D12268D30604D5532302A9CE
:10B660005B1820211970130704D5532302A95B1816
:10B670002B21197033782A2B2CD0350000210A2079
:10B68000E3682A786E1C303A092A64D900292ED042
:10B6900026E04E4B9F4202D1029B9F689FE74C4B96
:10B6A0009F429CD1029BDF6899E73900029800F025
:10B6B0000FFC002899D0012040421FB0F0BD013599
:10B6C0009BE7414B2268C01A012383401343236048
:10B6D0002E00B8E7059B191D1B680591002B01DBA7
:10B6E000099304E05B42E3600223134323602B7859
:10B6F0002E2B0AD16B782A2B35D1059B02351A1DCA
:10B700001B680592002B2BDB0793324E297803220E
:10B71000300000F071FE002806D04023801B8340DB
:10B720002268013513432360297806222A486E1CBB
:10B73000217600F061FE00283AD0284B002B25D15D
:10B740000722059B07339343083305936369039AE4
:10B750009B18636150E7434301219B18350090E734
:10B7600001235B42D0E700230A201A000135636001
:10B7700029786E1C3039092903D9002BC5D00792CE
:10B78000C3E74243012352183500F1E705AB0093AC
:10B790003A00134B2100029800E000BF0390039B86
:10B7A0000133D3D1BB895B0600D584E70B9884E7CE
:10B7B00005AB00933A000A4B2100029800F080F894
:10B7C000ECE7C046ECE2000098E200000CE3000069
:10B7D000CCE200009EE20000A2E2000000000000B7
:10B7E00093B50000F7B5150001938A680B690090C6
:10B7F0000C00934200DA130022002B6043321278CF
:10B80000002A01D001332B6023689B0602D52B68E8
:10B8100002332B60062723681F4027D023004333C1
:10B820001B785A1E93412268920630D42200019957
:10B8300043320098089EB047431C25D00623206859
:10B840002A68E16803400025042B03D18D1AEB43DD
:10B85000DB171D40A3682269934201DD9B1AED1896
:10B860000027BD4220D1002010E00137E3682A689C
:10B870009B1ABB42D2DD22000123193201990098A4
:10B88000089EB047431CF0D101204042FEBD30204D
:10B89000E1184331087021005A1C45310978A2187B
:10B8A000433202331170C1E7220001231A32019999
:10B8B0000098089EB047431CE6D00137D1E700004E
:10B8C000F0B589B004920A004332059303900292C6
:10B8D0000A7E0C000E9B6E2A00D186E01FD8632AD8
:10B8E00033D008D8002A00D18CE0582A4DD025004A
:10B8F00042352A7030E0642A01D0692AF7D11968EC
:10B9000025680A1D280629D508681A60002803DA68
:10B910002D23029A404213706B4E0A274FE0732A80
:10B9200074D008D86F2A1FD0702AE0D1202209686D
:10B930000A43226003E0752A16D0782AD7D1220064
:10B94000782145321170614E22E025001A68423597
:10B95000111D196013682B70012365E008681A60D7
:10B960006906D3D500B2D1E719682568081D1860AB
:10B9700008682E0605D5544E08276F2A1BD00A27C3
:10B9800019E06D06F7D580B2F5E745314E4E0A70E5
:10B9900018682268011D00681960150621D5D307B3
:10B9A00002D520231A4322601027002803D1202328
:10B9B00022689A4322602300002243331A7063688E
:10B9C000A360002B58DB04222168914321600028EA
:10B9D00054D1029D002B5AD02500337842352B706C
:10B9E00055E05506DBD580B2D9E71A680D68101D01
:10B9F0004969186013682E0601D5196002E06D06CA
:10BA0000FBD519800023029D23614FE01A68111DA8
:10BA10001960156800216268280000F0EDFC00281C
:10BA200001D0401B6060636823610023029A137099
:10BA30003CE023692A0004990398059DA847431C0C
:10BA40003ED023689B0715D4079BE068984239DAFB
:10BA5000180037E022000123193204990398059E4B
:10BA6000B047431C2CD00135E368079A9B1AAB42C0
:10BA7000F0DCE9E70025F7E70028ADD0029D3900AA
:10BA8000FDF722FC735C013D2B700028F7D1082FD5
:10BA900009D12368DB0706D563682269934202DC7B
:10BAA0003023013D2B70029B5B1B2361059B07AA82
:10BAB00000932100049B0398FFF794FE431CB8D128
:10BAC0000120404209B0F0BDA9E20000BAE2000046
:10BAD0000D4B70B51C680500A36B002B0FD118200F
:10BAE00000F06EFC094BA0630360094B0122436028
:10BAF000084B83600B238381002302614361002292
:10BB0000A36B1D615A6170BD800000200E33CDAB68
:10BB100034126DE6ECDE0500124B10B51C68A36B09
:10BB2000002B0FD1182000F04BFC0F4BA0630360DB
:10BB30000E4B012243600E4B83600B238381002355
:10BB400002614361A46B0B4A206961690A4BFDF7EE
:10BB5000F7FC0122002380185941206161614800EF
:10BB6000400810BD800000200E33CDAB34126DE6CE
:10BB7000ECDE05002D7F954C2DF451580CB430B5FA
:10BB8000164B9DB00C1E1D6808DA8B2301202B601C
:10BB900040421DB030BC08BC02B01847822302A945
:10BBA0009B008B810023029008619C4200D0631EA1
:10BBB0008B604B6101235B42CB81209A21AB280033
:10BBC000019300F055FD431C01DA8B232B60002C00
:10BBD000DFD00023029A1370DBE7C046800000200C
:10BBE0000EB400B50B499CB01DAB029006900791B6
:10BBF00004910948094904CB0591006802A9019301
:10BC000000F036FD0023029A13701CB008BC03B08C
:10BC10001847C046FFFFFF7F800000200802FFFF9B
:10BC2000020010B51378541C002B05D1CC5CD45401
:10BC30000133002CFAD110BD2200F3E7C9B203781A
:10BC4000002B04D08B4200D170470130F7E74B4204
:10BC5000594149420840F7E702780B78002A03D09F
:10BC6000013001319A42F7D0D01A70470023C25CEC
:10BC70000133002AFBD1581E7047002330B59A4289
:10BC80000AD0013AC45CCD5CAC4204D1934202D0EC
:10BC90000133002CF6D1631B180030BD30B5050010
:10BCA000002A00D130BD0C78013A6B1C2C70013198
:10BCB000002C05D19A189A42F4D01C700133FAE78F
:10BCC0001D00EDE710B50378002B0FD10B785A4219
:10BCD00053415B42184010BD0023CA5C002AFAD0D1
:10BCE000C45C944201D10133F7E701300378002BA3
:10BCF000F2D11800EFE70000F0B51F000E0087B08A
:10BD00000590019102920C98347800F0EAFA08222A
:10BD100000194378751C134036D12D2C36D1B51C33
:10BD200074780126002F62D0102F09D1302C07D152
:10BD300020222B789343582B54D110276C7802354E
:10BD40002D4B3900F31818000393FDF7BDFA049149
:10BD500001210023494202008C461800210030399D
:10BD600009291AD80C00A74223DD591C09D06346C3
:10BD7000824206D302D10499A14202DB0123784317
:10BD800020182C780135E9E72E00BCE72B2C01D0D8
:10BD90001E00C7E7B51C7478FAE72100413919295C
:10BDA00001D8373CDFE721006139192901D8573C18
:10BDB000D9E75A1C08D1059A23331360029B0398D4
:10BDC000002B09D107B0F0BD002E00D04042029AEE
:10BDD000002AF7D0002B01D06B1E0193029B019A21
:10BDE0001A60EFE73024002FAAD10827A8E7302CEB
:10BDF0009ED00A27A4E7C046FFFFFF7F37B5130098
:10BE0000064A05001068046A002C00D1044C0A00A0
:10BE100000942900FFF770FF3EBDC046800000205F
:10BE2000E4000020F8B505000E001400002804D03E
:10BE30008369002B01D100F0C1F9224B9C422DD126
:10BE40006C68A369A360A3891B0731D52369002B04
:10BE50002ED023682269F7B2981A6369F6B283423A
:10BE600005DC2100280000F03BF9002826D1A3685A
:10BE70000130013BA36023685A1C22601F70636974
:10BE8000834204D0A389DB071AD50A2E18D12100DA
:10BE9000280000F025F9002812D00FE00A4B9C4240
:10BEA00001D1AC68CDE7094B9C42CAD1EC68C8E728
:10BEB0002100280000F00CF80028CAD001267642A4
:10BEC0003000F8BDECE200000CE30000CCE2000022
:10BED000364B70B51D6806000C00002D05D0AB690F
:10BEE000002B02D1280000F069F9314B9C420FD1A0
:10BEF0006C680C23E25E93B219072DD4D90611D4D5
:10BF000009230120336037331343A381404270BDBE
:10BF1000284B9C4201D1AC68EBE7274B9C42E8D10F
:10BF2000EC68E6E75B0713D5616B002908D02300B6
:10BF30004433994202D0300000F06AFA0023636370
:10BF40002422A3899343A381002363602369236090
:10BF50000823A2891343A3812369002B0BD1A021BD
:10BF60008022A389890092000B40934203D02100D4
:10BF7000300000F0E1F90123A289134011D0002321
:10BF8000A36063695B42A361002023698342BED141
:10BF90000C23E25E1306BAD540231343A381013874
:10BFA000B5E7920700D46369A360EDE78000002045
:10BFB000ECE200000CE30000CCE2000010B506202B
:10BFC00000F090FC012000F0CFFD0000F7B58A8959
:10BFD00005000C00130760D44B68002B04DC0B6CCD
:10BFE000002B01DC0020FEBDE76A002FFAD0002301
:10BFF0002E682B6080235B01216A1A4034D0606D6B
:10C00000A3895B0706D56368C01A636B002B01D058
:10C01000236CC01A0200216A00232800E76AB8478F
:10C02000A189431C06D12B681D2B30D82B4ADA403E
:10C03000D3072CD50023636023692360CB0405D587
:10C04000431C02D12B68002B00D16065616B2E6010
:10C050000029C7D023004433994202D0280000F0C1
:10C06000D7F900206063BEE701232800B847431CCE
:10C07000C6D12B68002BC3D01D2B01D0162B01D1AC
:10C080002E60AFE74023A2891343A381ABE740238F
:10C090000B430120A3814042A5E70F69002FA1D0E7
:10C0A0000B680F60DB1B01930023920700D14B69E3
:10C0B000A360019B002B00DC94E7019B3A00216AFE
:10C0C0002800A66AB047002803DC4023A289134356
:10C0D000DFE7019B3F181B1A0193EAE701004020AC
:10C0E0000B6970B505000C00002B01D1002070BD5C
:10C0F000002804D08369002B01D100F05FF80B4BBE
:10C100009C4209D16C680C22A35E002BEED021006A
:10C110002800FFF75BFFEAE7054B9C4201D1AC68C2
:10C12000F1E7044B9C42EED1EC68ECE7ECE2000056
:10C130000CE30000CCE20000002310B50400036013
:10C140004360836081814366C2810361436183618F
:10C15000190008225C30FFF7FFF9054B2462636287
:10C16000044BA362044BE362044B236310BDC0463F
:10C1700025C900004DC9000085C90000B1C90000F3
:10C1800010B5024900F08CF810BDC046E1C00000B7
:10C1900070B568254A1E55430E002900743100F021
:10C1A00081F9041E08D000212A00016046600C308D
:10C1B000A0606832FFF7D0F9200070BD836913B525
:10C1C0000400002B28D18364C3640365134B144A15
:10C1D0001B6882620193984201D101238361200090
:10C1E00000F020F86060200000F01CF8A060200043
:10C1F00000F018F80022E06004216068FFF79CFF5F
:10C2000001220921A068FFF797FF02221221E068AE
:10C21000FFF792FF0123A36113BDC04694E2000023
:10C2200081C10000F8B51C4B07001E68B369002BE4
:10C2300002D13000FFF7C2FF4836B4687368013B93
:10C2400004D53368002B07D03668F6E70C22A55ECC
:10C25000002D0DD06834F2E704213800FFF798FF75
:10C2600030600028F0D10C2304003B602000F8BDB2
:10C2700020000A4B656625606560A560E360256166
:10C280006561A561082229005C30FFF765F96563E7
:10C29000A563A564E564E9E794E200000100FFFFFF
:10C2A000F7B504000700002601914834002C01D1A5
:10C2B0003000FEBD6368A5680093009B013B0093BE
:10C2C00001D52468F2E7AB89012B08D90E22AB5EB9
:10C2D000013304D029003800019B98470643683594
:10C2E000EBE7EC300068704770B50E001D000E23C0
:10C2F000C95E96B01400002907DA00232B60B389C9
:10C300001B0611D48023DB000FE06A4600F088FB97
:10C310000028F2DBF022019B12021340054A9B1811
:10C320005A4253412B60EDE740230020236016B0B2
:10C3300070BDC04600E0FFFFF7B502268B890500FF
:10C340000C00334206D023004733236023610123CE
:10C350006361F7BD01AB6A46FFF7C6FF00990700AE
:10C36000280000F09FF8002808D10C22A35E9A054F
:10C37000EFD4032293431E43A681E4E70F4BAB6245
:10C380008023A28920601343A381009B2061636105
:10C39000019B002B0DD00E23E15E280000F052FB24
:10C3A000002806D00322A38993431A0001231343D4
:10C3B000A381A0893843A081CBE7C04681C100009A
:10C3C00010B5034B0100186800F06CF810BDC046B2
:10C3D0008000002082B0002900D101A9101E06D0E3
:10C3E000002B06D013780B601078431E984102B0E2
:10C3F000704702204042FAE7C9B28218904201D148
:10C400000020704703788B42FBD00130F6E7000034
:10C4100070B50500002910D00C1F2368002B00DA2E
:10C42000E418280000F034FB1D4A1368002B05D1E6
:10C4300063601460280000F02CFB70BDA34209D992
:10C44000216860188342F3D118685B684118216045
:10C45000EEE713005A68002A01D0A242F9D9196800
:10C460005818A0420BD12068091858181960824248
:10C47000E0D110685268411819605A60DAE7A042AA
:10C4800002D90C232B60D5E721686018824203D1C2
:10C49000106852684118216062605C60CAE7C0465B
:10C4A000241C0020032370B5CD1C9D4308350600D5
:10C4B0000C2D1ED20C25A9421DD8300000F0E8FA40
:10C4C000254A14682100002919D1244C2368002B27
:10C4D00003D1300000F0CAF920602900300000F0DC
:10C4E000C5F9431C2BD10C233000336000F0D1FA86
:10C4F00003E0002DDFDA0C233360002070BD0B68F1
:10C500005B1B19D40B2B03D90B60CC18256003E0FF
:10C510004B688C420DD11360300000F0BAFA200055
:10C5200007220B30231D9043C31AE7D05A42E25032
:10C53000E4E763600C00EFE70C004968C3E70323FE
:10C54000C41C9C43A042E1D0211A300000F08EF9B7
:10C55000431CDBD1C7E7C046241C0020281C002058
:10C56000F8B507000D001600002905D11100FFF7EE
:10C5700099FF04002000F8BD002A03D1FFF748FF0F
:10C580003400F7E700F086FA2C00B042F2D2310016
:10C590003800FFF787FF041EECD029003200FEF7B9
:10C5A000BFFF29003800FFF733FFE3E7F0B58E68DF
:10C5B00085B007000C00039201939E423CD8902363
:10C5C0008A89DB001A4234D00325096923685B1A83
:10C5D0000293636902985D43EB0F5D19019B6D1037
:10C5E00001331B18AB4200D91D00530532D5290079
:10C5F0003800FFF757FF061E09D10C233B6040238C
:10C600000120A28940421343A38105B0F0BD029AE4
:10C610002169FEF785FFA389144A1A40802313433A
:10C62000A381029B2661F61826606561019EED1AC2
:10C63000A560019B9E4200D9019E320003992068AB
:10C64000FEF777FFA36800209B1BA36023689E1959
:10C650002660DAE72A003800FFF782FF061EE0D1E5
:10C6600021693800FFF7D4FEC7E7C0467FFBFFFF14
:10C67000F0B59FB0029005938B890F0016001B0642
:10C6800011D50B69002B0ED14021FFF70BFF38604D
:10C690003861002805D10C23029A013813601FB0BD
:10C6A000F0BD40237B61002306AC636120336376D9
:10C6B0001033A37635002B78002B01D0252B46D1E3
:10C6C000AB1B04930CD0320039000298FFF76EFFC9
:10C6D000431C00D1AEE06269049B944663446361ED
:10C6E0002B78002B00D1A5E001220023524262608A
:10C6F00002A9543252186E1C2360E360A3601370C9
:10C70000A365317805225448FFF776FE751C002892
:10C710001FD12268D30604D5532302A95B18202118
:10C720001970130704D5532302A95B182B21197024
:10C7300033782A2B16D0350000210A20E3682A78A6
:10C740006E1C303A092A4ED9002918D010E0013564
:10C75000B1E7414B2268C01A012383401343236091
:10C760002E00CEE7059B191D1B680591002B01DBF0
:10C77000099304E05B42E3600223134323602B78B8
:10C780002E2B0AD16B782A2B35D1059B02351A1D29
:10C790001B680592002B2BDB0793304E2978032270
:10C7A0003000FFF729FE002806D04023801B83407D
:10C7B00022680135134323602978062228486E1C1D
:10C7C0002176FFF719FE00283CD0264B002B25D1FF
:10C7D0000722059B07339343083305936369039A44
:10C7E0009B18636166E7434301219B183500A6E768
:10C7F00001235B42D0E700230A201A000135636061
:10C8000029786E1C3039092903D9002BC5D007922D
:10C81000C3E74243012352183500F1E705AB00930B
:10C820003A00114B2100029800E000BF0390039BE7
:10C830000133D3D1BB890B985B0600D42FE70120CD
:10C8400040422CE705AB00933A00074B21000298C9
:10C85000FFF736F8EAE7C04698E200009EE20000E3
:10C86000A2E2000000000000ADC50000002370B58A
:10C87000064C05000800236000F060F9431C03D15A
:10C880002368002B00D02B6070BDC046B82F00205D
:10C8900070B504000D001F2904D916230360012080
:10C8A000404270BD436C002B04D08A009B181A686C
:10C8B000002A08D1200000F031F82A0001002000F1
:10C8C00000F01AF8EDE70020012AEAD0511C03D14C
:10C8D000162301302360E4E7002428001C60904701
:10C8E0002000DEE710B5034B01001868FFF7D0FF0A
:10C8F00010BDC04680000020002370B5064C050026
:10C9000008001100236000F001F9431C03D12368E3
:10C91000002B00D02B6070BDB82F002010B500F0A8
:10C92000E5F810BD70B50C000E25495F00F0BAF8AF
:10C93000002803DB636D1B18636570BDA389024A81
:10C940001340A381F9E7C046FFEFFFFFF8B51F00D2
:10C950008B8905000C001600DB0505D50E23C95E8A
:10C960000022022300F080F8A389054A2800134022
:10C97000A38132000E23E15E3B0000F02BF8F8BDEE
:10C98000FFEFFFFF70B50C000E25495F00F06CF85B
:10C99000A389421C03D1054A1340A38170BD8022A4
:10C9A00052011343A3816065F8E7C046FFEFFFFF24
:10C9B00010B50E23C95E00F021F810BD0B1E04D087
:10C9C000FF2A04D98A2303608B3B180070470A7042
:10C9D0000123FAE770B50500080011000022064C9B
:10C9E00022601A0000F0B8F8431C03D12368002B22
:10C9F00000D02B6070BDC046B82F0020002370B55A
:10CA0000064C05000800236000F060F8431C03D1C9
:10CA10002368002B00D02B6070BDC046B82F0020CB
:10CA2000002370B5064C050008001100236000F0DB
:10CA300055F8431C03D12368002B00D02B6070BD38
:10CA4000B82F0020002370B5064C050008002360B5
:10CA500000F054F8431C03D12368002B00D02B6056
:10CA600070BDC046B82F002070B505000800110049
:10CA70000022064C22601A0000F050F8431C03D13B
:10CA80002368002B00D02B6070BDC046B82F00205B
:10CA9000704770470B1F1B68181F002B01DA0B58DB
:10CAA000C018704770B50500080011000022064C40
:10CAB00022601A0000F03AF8431C03D12368002BCF
:10CAC00000D02B6070BDC046B82F00205822012036
:10CAD000014B40421A607047B82F002058220120B5
:10CAE000014B40421A607047B82F002058220120A5
:10CAF000014B40421A607047B82F00205822024B69
:10CB000000201A607047C046B82F0020582201202C
:10CB1000014B40421A607047B82F00205822012074
:10CB2000014B40421A607047B82F00205822012064
:10CB3000014B40421A607047B82F0020044A136826
:10CB4000002B00D1034B1818106018007047C04626
:10CB50002C1C0020C02F002058220120014B4042F5
:10CB60001A607047B82F0020FEE7C046F8B5C046EF
:10CB7000F8BC08BC9E467047F8B5C046F8BC08BC77
:10CB80009E467047646174610000000008CC00009C
:10CB9000EF01000011CC0000E302000019CC0000FE
:10CBA0000909000020CC0000190A000025CC000073
:10CBB0003105000030CC00005303000035CC0000EC
:10CBC000710C000041CC00001F0200004BCC0000A3
:10CBD0001108000059CC0000BD06000066CC000022
:10CBE000F104000072616E646F6D00616C6C006C2A
:10CBF0006173740066616C736500747275650025FD
:10CC00002E3135732E2E2E006D616B654C69737459
:10CC1000006164644C6173740064656C65746500E4
:10CC20006A6F696E00636F707946726F6D546F0042
:10CC300066696E64006A6F696E537472696E6773B9
:10CC400000756E69636F6465417400756E69636F2A
:10CC50006465537472696E67006E657742797465B6
:10CC6000417272617900667265654D656D6F7279AA
:10CC700000000000D9CC0000D9100000DECC00007C
:10CC8000F710000019CC0000FB100000E4CC0000FD
:10CC9000DD100000EECC0000FF100000F7CC00001B
:10CCA0000311000001CD0000071100000CCD0000B1
:10CCB0000B11000018CD0000E110000021CD000094
:10CCC000EF1000002BCD0000E510000036CD000075
:10CCD000F310000066696C65006F70656E00636C30
:10CCE0006F736500656E644F6646696C65007265BA
:10CCF00061644C696E650072656164427974657344
:10CD000000617070656E644C696E6500617070657D
:10CD10006E6442797465730066696C6553697A65FF
:10CD20000073746172744C697374006E6578744931
:10CD30006E4C6973740073797374656D496E666FB8
:10CD400000000000381300004813000062130000C8
:10CD5000E0130000181400004E14000086140000B8
:10CD6000AC140000E81400002A1500008015000033
:10CD7000C415000030160000781600009E16000052
:10CD8000D61600001C1700004217000070170000A4
:10CD90009E170000D417000058180000201900004A
:10CDA00096190000061A0000521A0000721A0000BC
:10CDB000941A0000461B00008C1B0000041C00009D
:10CDC000321C0000621C0000981C0000001D0000C6
:10CDD000801D0000C61D00000E1E0000841E000005
:10CDE000FA1E0000421F0000881F0000BE1F000046
:10CDF000042000004A20000092200000E6200000ED
:10CE00004421000082210000EC21000022220000C9
:10CE10006A220000B2220000FA220000342300003F
:10CE20007C230000C42300003025000070170000A0
:10CE3000381300002C240000381300006224000086
:10CE40008E240000C4240000F024000038130000E9
:10CE5000381300003813000038130000AA25000022
:10CE6000EC2500003226000082260000AE260000DD
:10CE7000FE2600002427000052270000381300007F
:10CE80003813000076270000A6270000D6270000F0
:10CE90000C280000362800006C28000096280000AE
:10CEA000BE280000E62800004C2900007C29000074
:10CEB000A6290000D0290000002A00002A2A00002C
:10CEC0003813000038130000381300003813000036
:10CED000381300005A2A0000862A0000B22A0000F7
:10CEE000DE2A00000A2B0000402B0000762B0000F9
:10CEF000AC2B0000E22B00000E2C00003A2C0000AE
:10CF0000702C0000381300003813000038130000A4
:10CF100038130000381300003813000038130000E5
:10CF200038130000381300003813000038130000D5
:10CF30003813000038130000381300009C2C000048
:10CF4000D22C00005B2564206974656D206C6973C8
:10CF5000745D002825642062797465732900286F48
:10CF6000626A65637420747970653A2025642900CB
:10CF7000537461636B20756E646572666C6F7700C5
:10CF8000626F6F6C65616E006E756D6265720073C5
:10CF90007472696E67006C697374006279746520DD
:10CFA0006172726179000000070000000300000058
:10CFB00002D00000F52D00000AD00000A52E0000D0
:10CFC00013D000004F2F00001CD00000F92D0000EE
:10CFD00025D00000532F00002DD000003D2F000071
:10CFE000000000000100000002000000030000003B
:10CFF000040000000A0000006D6963726F3A626904
:10D000007400686173546F6E6500706C6179546F61
:10D010006E6500686173536572766F007365745353
:10D020006572766F00646163496E69740064616360
:10D03000577269746500474320746F6F6B202564D5
:10D040002075736563733B206672656520256420D7
:10D05000776F726473003C496E74656765723E0059
:10D060003C4C6973743E003C4F626A6563743E00D9
:10D070003C4279746541727261793E000D0A564DE9
:10D080002050616E69633A2025730D0A006D697343
:10D0900063000000C9D00000113C0000D2D00000A5
:10D0A000A13B0000D6D00000F53A0000DED0000021
:10D0B0009B3A0000E8D00000313A0000F4D00000B4
:10D0C000333900006E756C6C00686578546F496E7A
:10D0D000740073696E006A736F6E476574006A73DB
:10D0E0006F6E436F756E74006A736F6E56616C7508
:10D0F000654174006A736F6E4B657941740000007E
:10D100005CD100007D3C000064D10000813C000047
:10D110006ED100009F3C000077D10000A93C0000C8
:10D1200082D10000B33C00008ED10000BD3C000065
:10D13000A3D10000C73C0000B8D10000D13C0000E2
:10D14000C4D10000DB3C0000D4D100008B3C0000C7
:10D15000E0D10000953C00006E6574006861735773
:10D160006946690073746172745769466900737423
:10D170006F705769466900776966695374617475A1
:10D1800073006D794950416464726573730068740B
:10D190007470536572766572476574526571756512
:10D1A000737400726573706F6E64546F487474703A
:10D1B000526571756573740068747470436F6E6E38
:10D1C00065637400687474704973436F6E6E656351
:10D1D0007465640068747470526571756573740069
:10D1E00068747470526573706F6E7365001A1B1CDF
:10D1F00003040607090A17181900000000000808B0
:10D200000800080A4A4000000A5FEA5FEA0ED92EC9
:10D21000D36E19324489330C924C924D08080000A9
:10D220000004880808040804848488000A448A40AA
:10D2300000048EC480000000048800000EC00000BE
:10D240000000080001224488100C9252524C048CB9
:10D2500084848E1C824C901E1EC244924C06CA527C
:10D260005FE21FF01EC13E02448ED12E1FE24488B1
:10D27000100ED12ED12E0ED12EC488000800080029
:10D2800000048004880244880482000EC00EC00896
:10D29000048244880ED126C0040ED135B36C0C92A2
:10D2A0005ED2521C925C925C0ED010100E1C9252F8
:10D2B000525C1ED01C901E1ED01C90100ED01371FC
:10D2C0002E12525ED2521C8808081C1FE242524C99
:10D2D0001254981492101010101E113B75B1311198
:10D2E0003935B3710C9252524C1C925C90100C92D6
:10D2F000524C861C925C92510ED00C825C1FE484CE
:10D300008484125252524C1131312A44113135BBAE
:10D310007112524C9252112A4484841EC488101EE9
:10D320000EC808080E10080482410EC242424E0484
:10D330008A400000000000001F0804800000000E6A
:10D34000D2524F10101C925C000ED0100E02424EB2
:10D35000D24E0C925C900E06C81C88080ED24EC2AB
:10D360004C10101C92520800080808024002424C5F
:10D3700010149814920808080806001B75B13100B3
:10D380001C925252000C92524C001C925C90000E67
:10D39000D24EC2000ED010100006C8049808080E25
:10D3A000C807001252524F0011312A440011313582
:10D3B000BB00124C8C9200112A4498001EC4881E97
:10D3C00006C48C8486080808080818080C88180009
:10D3D000000C83600000000001000000020000005B
:10D3E000030000000400000005000000060000002B
:10D3F0000700000008000000090000000A0000000B
:10D400000B0000000C0000000D0000000E000000EA
:10D410000F000000100000001200000014000000C7
:10D4200016000000180000001A0000001C00000098
:10D430001E00000020000000230000002600000065
:10D44000290000002C0000002F0000003200000026
:10D45000360000003A0000003E00000042000000DC
:10D46000460000004B000000500000005500000086
:10D470005A00000061000000680000006F0000001A
:10D48000760000007D000000840000008B0000009A
:10D490009200000099000000A0000000A70000001A
:10D4A000AE000000B5000000BC000000C30000009A
:10D4B000CA000000D1000000D8000000DF0000001A
:10D4C000E6000000ED000000F4000000FB0000009A
:10D4D000FF00000024D50000FD3C00002FD5000017
:10D4E0009142000039D50000B93E000046D5000049
:10D4F000014100004DD500005141000056D500000B
:10D50000A141000062D500009940000073D50000E1
:10D51000293F000080D50000294000006469737035
:10D520006C6179006C696768744C6576656C006D38
:10D5300062446973706C6179006D62446973706CE8
:10D5400061794F6666006D62506C6F74006D625554
:10D550006E706C6F74006D624472617753686170B5
:10D5600065006D625368617065466F724C657474D6
:10D570006572006E656F506978656C53656E640006
:10D580006E656F506978656C53657450696E004EB6
:10D590006F7420656E6F75676820726F6F6D2065A0
:10D5A00076656E20616674657220636F6D7061636D
:10D5B00074696F6E00436F6D7061637465642046BB
:10D5C0006C61736820636F64652073746F72650AA1
:10D5D000256420627974657320757365642028253D
:10D5E00064252529206F662025640042616420722D
:10D5F00065636F726420666F756E6420647572690E
:10D600006E6720696E697469616C697A6174696FAB
:10D610006E00256420256420256420282564207759
:10D620006F72647329002564207265636F7264737E
:10D630002C20256420776F7264732C206D617849EB
:10D64000442025642C20636F6D70616374696F6E74
:10D65000206379636C657320256400526573746F71
:10D66000726564202564207363726970747300535B
:10D6700074617274656400726164696F0000000017
:10D6800010D70000614C00001DD70000FD4E0000C7
:10D690002DD700007D4E00003BD7000091500000C8
:10D6A00046D70000894C000056D70000114D0000FD
:10D6B0006AD70000F94C000079D7000073520000CF
:10D6C00085D70000F15100008ED700009551000071
:10D6D00099D70000DD500000A4D7000019510000C8
:10D6E000ADD700004D510000B6D70000994C0000A6
:10D6F000C5D70000794C0000CED70000A94C00002F
:10D700006E6F6E65006F746865720070616972009B
:10D7100064697361626C65526164696F006D657301
:10D7200073616765526563656976656400706163FE
:10D730006B657452656365697665007061636B65DE
:10D740007453656E64007265636569766564496EDD
:10D7500074656765720072656365697665644D65B9
:10D760007373616765547970650072656365697686
:10D770006564537472696E670073656E64496E7494
:10D78000656765720073656E6450616972007365E8
:10D790006E64537472696E67007365744368616E7A
:10D7A0006E656C0073657447726F75700073657495
:10D7B000506F776572007369676E616C5374726540
:10D7C0006E677468006465766963654944006C61DE
:10D7D00073744D657373616765494400556E6B6E74
:10D7E0006F776E207072696D6974697665205B254C
:10D7F000733A25735D000000000000009630077743
:10D800002C610EEEBA51099919C46D078FF46A7034
:10D8100035A563E9A395649E3288DB0EA4B8DC7954
:10D820001EE9D5E088D9D2972B4CB609BD7CB17ED4
:10D83000072DB8E7911DBF906410B71DF220B06AA4
:10D840004871B9F3DE41BE847DD4DA1AEBE4DD6DB4
:10D8500051B5D4F4C785D38356986C13C0A86B64B4
:10D860007AF962FDECC9658A4F5C0114D96C0663D4
:10D87000633D0FFAF50D088DC8206E3B5E10694CB4
:10D88000E44160D5727167A2D1E4033C47D4044BF4
:10D89000FD850DD26BB50AA5FAA8B5356C98B242D4
:10D8A000D6C9BBDB40F9BCACE36CD832755CDF4554
:10D8B000CF0DD6DC593DD1ABAC30D9263A00DE5184
:10D8C0008051D7C81661D0BFB5F4B42123C4B35674
:10D8D0009995BACF0FA5BDB89EB802280888055FF4
:10D8E000B2D90CC624E90BB1877C6F2F114C685854
:10D8F000AB1D61C13D2D66B69041DC760671DB0142
:10D90000BC20D2982A10D5EF8985B1711FB5B60613
:10D91000A5E4BF9F33D4B8E8A2C9077834F9000F53
:10D920008EA8099618980EE1BB0D6A7F2D3D6D08F3
:10D93000976C6491015C63E6F4516B6B62616C1CE3
:10D94000D83065854E0062F2ED95066C7BA5011B13
:10D95000C1F4088257C40FF5C6D9B06550E9B712B3
:10D96000EAB8BE8B7C88B9FCDF1DDD62492DDA1573
:10D97000F37CD38C654CD4FB5861B24DCE51B53A93
:10D980007400BCA3E230BBD441A5DF4AD795D83D93
:10D990006DC4D1A4FBF4D6D36AE96943FCD96E34D3
:10D9A000468867ADD0B860DA732D0444E51D0333B3
:10D9B0005F4C0AAAC97C0DDD3C710550AA410227C3
:10D9C00010100BBE86200CC925B56857B3856F2093
:10D9D00009D466B99FE461CE0EF9DE5E98C9D929F3
:10D9E0002298D0B0B4A8D7C7173DB359810DB42E33
:10D9F0003B5CBDB7AD6CBAC02083B8EDB6B3BF9A7F
:10DA00000CE2B6039AD2B1743947D5EAAF77D29D0A
:10DA10001526DB048316DC73120B63E3843B6494EA
:10DA20003E6A6D0DA85A6A7A0BCF0EE49DFF0993EA
:10DA300027AE000AB19E077D44930FF0D2A308875A
:10DA400068F2011EFEC206695D5762F7CB6765800A
:10DA500071366C19E7066B6E761BD4FEE02BD3890A
:10DA60005A7ADA10CC4ADD676FDFB9F9F9EFBE8E6A
:10DA700043BEB717D58EB060E8A3D6D67E93D1A1AA
:10DA8000C4C2D83852F2DF4FF167BBD16757BCA68A
:10DA9000DD06B53F4B36B248DA2B0DD84C1B0AAF2A
:10DAA000F64A0336607A0441C3EF60DF55DF67A8AA
:10DAB000EF8E6E3179BE69468CB361CB1A8366BC3A
:10DAC000A0D26F2536E2685295770CCC03470BBB8A
:10DAD000B91602222F260555BE3BBAC5280BBDB28A
:10DAE000925AB42B046AB35CA7FFD7C231CFD0B52A
:10DAF0008B9ED92C1DAEDE5BB0C2649B26F263EC1C
:10DB00009CA36A750A936D02A906099C3F360EEB29
:10DB10008567077213570005824ABF95147AB8E2E9
:10DB2000AE2BB17B381BB60C9B8ED2920DBED5E5C9
:10DB3000B7EFDC7C21DFDB0BD4D2D38642E2D4F119
:10DB4000F8B3DD686E83DA1FCD16BE815B26B9F6A9
:10DB5000E177B06F7747B718E65A0888706A0FFF09
:10DB6000CA3B06665C0B0111FF9E658F69AE62F8C9
:10DB7000D3FF6B6145CF6C1678E20AA0EED20DD7C9
:10DB80005483044EC2B30339612667A7F71660D0E9
:10DB90004D476949DB776E3E4A6AD1AEDC5AD6D929
:10DBA000660BDF40F03BD83753AEBCA9C59EBBDE49
:10DBB0007FCFB247E9FFB5301CF2BDBD8AC2BACAF9
:10DBC0003093B353A6A3B4240536D0BA9306D7CD69
:10DBD0002957DE54BF67D9232E7A66B3B84A61C489
:10DBE000021B685D942B6F2A37BE0BB4A18E0CC349
:10DBF0001BDF055A8DEF022D416C6C207461736B35
:10DC0000732073746F70706564007630383900204B
:10DC10002573202573004D656D6F727920636C65E7
:10DC200061726564004E6F20667265652074617371
:10DC30006B20656E747269657300000084DC0000FF
:10DC4000FD65000091DC0000396200009DDC0000F1
:10DC5000CD650000A3DC0000DD650000A9DC00004C
:10DC6000ED650000AFDC00006D620000B9DC000073
:10DC700059660000C1DC0000AD63000073656E737F
:10DC80006F727300616363656C65726174696F6E56
:10DC90000074656D70657261747572650074696C8D
:10DCA00074580074696C74590074696C745A007407
:10DCB0006F756368526561640069326352656164BF
:10DCC00000693263577269746500000040DD00002E
:10DCD000E56600004EDD0000E966000057DD00004B
:10DCE000F566000061DD0000F96600006ADD0000F5
:10DCF000FD6600006FDD00000167000074DD0000BC
:10DD00000567000080DD00000967000087DD000076
:10DD10000D67000090DD00001167000095DD000038
:10DD200015670000A0DD000019670000AADD0000F3
:10DD3000ED660000B4DD0000F1660000746674005A
:10DD4000656E61626C65446973706C6179006765CA
:10DD500074576964746800676574486569676874B6
:10DD600000736574506978656C006C696E6500724B
:10DD700065637400726F756E6465645265637400E8
:10DD8000636972636C6500747269616E676C6500CB
:10DD90007465787400746674546F756368656400A4
:10DDA000746674546F7563685800746674546F7544
:10DDB00063685900746674546F7563685072657354
:10DDC000737572650076617273000000ECDD00000F
:10DDD000A96B0000F6DD0000896B0000FFDD00008C
:10DDE000656B00000BDE0000F16A00007661724591
:10DDF0007869737473007661724E616D6564007347
:10DE000065745661724E616D6564007661724E6133
:10DE10006D65466F72496E6465780057656C636F17
:10DE20006D6520746F204D6963726F426C6F636B18
:10DE3000732100705F73706920213D204E554C4C5A
:10DE4000002F686F6D652F6769742F2E706C617479
:10DE5000666F726D696F2F7061636B616765732F99
:10DE60006672616D65776F726B2D61726475696E34
:10DE70006F6E6F726469636E7266352F6C69627261
:10DE800061726965732F5350492F5350492E637047
:10DE90007000535049436C6173733A3A535049438D
:10DEA0006C617373284E52465F5350495F547970CA
:10DEB000652A2C2075696E74385F742C2075696E24
:10DEC00074385F742C2075696E74385F7429000093
:10DED0000000000000000000B56D0000716D000042
:10DEE000976D0000A16D0000AB6D0000956D000006
:10DEF0000300000002000000010000000400000018
:10DF000005000000110000000C0000000B000000E4
:10DF1000120000000A000000060000001A000000C5
:10DF2000140000001700000016000000150000009B
:10DF300010000000FFFFFFFFFFFFFFFF00000000D9
:10DF40001E0000001900000018000000070000007B
:10DF500008000000090000000D0000000E00000095
:10DF60000F0000001C0000001B0000001D0000004E
:10DF700013000000000000000000000065720000B7
:10DF800095790000E5720000F9720000EF72000060
:10DF9000617200005572000005730000817200007C
:10DFA000517200000000000000000000000030433B
:10DFB00000000000000030C37371727400000000A4
:10DFC000FB21F93FFB2109407CD91240FB2119407C
:10DFD0007A6A1F407CD92240BBFD2540FB212940A5
:10DFE0003A462C407A6A2F405C4731407CD9324017
:10DFF0009C6B3440BBFD3540DB8F3740FB21394003
:10E000001BB43A403A463C405AD83D407A6A3F40B9
:10E010004C7E40405C4741406C1042407CD94240BD
:10E020008CA243409C6B4440AC344540BBFD454012
:10E03000CBC64640DB8F4740EB584840FB21494068
:10E0400083F9A200444E6E00FC291500D157270029
:10E05000DD34F50062DBC0003C999500419043003F
:10E060006351FE00BBDEAB00B761C5003A6E240011
:10E07000D24D42004906E00009EA2E001C92D10070
:10E08000EB1DFE0029B11C00E83EA700F53582001B
:10E0900044BB2E009CE98400B4267000417E5F00E2
:10E0A000D6913900538339009CF439008B5F84008A
:10E0B00028F9BD00F81F3B00DEFF97000F98050010
:10E0C000112FEF000A5A8B006D1F6D00CF7E3600B6
:10E0D00009CB2700464FB7009E663F002DEA5F0040
:10E0E000BA277500E5EBC7003D7BF100F739070063
:10E0F00092528A00FB6BEA001FB15F00085D8D0041
:10E10000300356007BFC4600F0AB6B0020BCCF0018
:10E1100036F49A00E3A91D005E619100081BE60039
:10E1200085996500A0145F008D40680080D8FF00CD
:10E1300027734D0006063100CA561500C9A87300A2
:10E140007BE260006B8CC00000000040FB21F93FC7
:10E15000000000002D44743E000000809846F83C0A
:10E160000000006051CC783B00000080831BF03938
:10E170000000004020257A38000000802282E3362B
:10E18000000000001DF369350200000003000000DC
:10E1900004000000060000008C9600003696000087
:10E1A0003696000064970000329600003296000018
:10E1B0005A97000064970000329600005A970000BA
:10E1C000329600006497000068970000689700008E
:10E1D000689700007097000068A10000DA9F0000B7
:10E1E0001EA00000829F00001EA000000EA10000E3
:10E1F0001EA00000829F0000DA9F0000DA9F00004E
:10E200000EA10000829F00007A9F00007A9F00000C
:10E210007A9F00001CA1000090A8000092A70000B7
:10E2200092A70000B0AA00008CA700008CA70000F5
:10E2300098AA0000B0AA00008CA7000098AA0000CD
:10E240008CA70000B0AA0000A6AA0000A6AA0000A1
:10E25000A6AA0000B4AA00002C2066756E6374693B
:10E260006F6E3A2000617373657274696F6E20225D
:10E27000257322206661696C65643A2066696C6565
:10E2800020222573222C206C696E6520256425735D
:10E2900025730A0084000020232D302B2000686C99
:10E2A0004C006566674546470030313233343536B9
:10E2B00037383941424344454600303132333435F2
:10E2C000363738396162636465660000000000001B
:10E2D000000000000000000000000000000000003E
:10E2E000000000000000000000000000000000002E
:10E2F000000000000000000000000000000000001E
:10E30000000000000000000000000000000000000D
:10E3100000000000000000000000000000000000FD
:10E320000000000000000000000000004300504F0B
:10E330005349580000202020202020202020282879
:10E3400028282820202020202020202020202020B5
:10E3500020202020208810101010101010101010F5
:10E360001010101010040404040404040404041025
:10E3700010101010101041414141414101010101B3
:10E38000010101010101010101010101010101017D
:10E390001010101010104242424242420202020289
:10E3A000020202020202020202020202020202024D
:10E3B00010101010200000000000000000000000FD
:10E3C000000000000000000000000000000000004D
:10E3D000000000000000000000000000000000003D
:10E3E000000000000000000000000000000000002D
:10E3F000000000000000000000000000000000001D
:10E40000000000000000000000000000000000000C
:10E4100000000000000000000000000000000000FC
:10E4200000000000000000000000000000000000EC
:0CE43000000000000000000000000000E0
:08E43C00CC1CFF7F0100000071
:10E44400FFFFFFFF4006000001000000E803DC05B9
:10E45400DC05DC05DC050000FFFFFFFFFFFFFFFF1D
:10E464001800000019FCFFFFFFFFFFFFFF00000082
:10E474000200000003000000FFFFFFFF0000000097
:10E48400010000000000020001000000FFFFFFFF88
:10E494000000000002000000000004000200000070
:10E4A400FFFFFFFF00000000030000000000080061
:10E4B400030000000A000000080000000100000042
:10E4C4008400002000000000ECE200000CE30000E7
:10E4D400CCE200000000000000000000000000008A
:10E4E4000000000000000000000000000000000028
:10E4F4000000000000000000000000000000000018
:10E504000000000000000000000000000000000007
:10E5140000000000000000000000000000000000F7
:10E5240000000000430000000000000000000000A4
:10E5340000000000000000000000000000000000D7
:10E544000000000043000000000000000000000084
:10E5540000000000000000000000000000000000B7
:10E564000000000043000000000000000000000064
:10E574000000000000000000000000000000000097
:10E584000000000043000000000000000000000044
:10E594000000000000000000000000000000000077
:10E5A4000000000043000000000000000000000024
:10E5B4000000000000000000000000000000000057
:10E5C4000000000043000000000000000000000004
:10E5D4000000000000000000000000000000000037
:10E5E40000000000430000000000000000000000E4
:10E5F4000000000000000000000000000000000017
:10E6040000000000BDC90000D5C3000000000000E8
:10E6140034E3000006CC00008CD000008CD0000055
:10E624008CD000008CD000008CD000008CD0000076
:10E634008CD000008CD000008CD00000FFFFFFFFC6
:10E64400FFFFFFFFFFFFFFFFFFFF0000010041533B
:10E6540043494900000000000000000000000000E1
:10E664000000000000000000000000000000415312
:10E6740043494900000000000000000000000000C1
:10E684000000000000000000000000000000000086
:10E69400E9000000416D000089700000B1750000C0
:04E6A400C1000000B1
:040000030000712563
:00000001FF
